:1000000000560020316D0000916C0000A16C0000D2
:10001000B96C0000D16C0000E96C00000000000029
:10002000000000000000000000000000016D000062
:10003000116D000000000000216D0000196E00002D
:10004000796C000000000000000000007116010043
:10005000AD1501001D1601000000000000000000A9
:10006000F14D000051F8000031F80000E9160100E0
:10007000000000000000000000000000091701005F
:100080002DE9F843054689464FF00108154E164CF8
:10009000164F12E0236943F00403236187F832808E
:1000A000BFF34F8F00BF30BF87F83200236923F0C2
:1000B00004032361BFF34F8F62B600F01DF872B6E0
:1000C000735D33B900F014F80028E3D000BF30BFEF
:1000D000F2E700237355B9F1000F00D0C84762B6AC
:1000E000BDE8F8831024002000ED00E0000010506F
:1000F0005FF800F0214D00005FF800F091FB000078
:10010000FFFFFFFFFFFFFFFFFFFFFFFFFFFFFFFFFF
:10011000FFFFFFFFFFFFFFFFFFFFFFFFFFFFFFFFEF
:10012000FFFFFFFFFFFFFFFFFFFFFFFFFFFFFFFFDF
:10013000FFFFFFFFFFFFFFFFFFFFFFFFFFFFFFFFCF
:10014000FFFFFFFFFFFFFFFFFFFFFFFFFFFFFFFFBF
:10015000FFFFFFFFFFFFFFFFFFFFFFFFFFFFFFFFAF
:10016000FFFFFFFFFFFFFFFFFFFFFFFFFFFFFFFF9F
:10017000FFFFFFFFFFFFFFFFFFFFFFFFFFFFFFFF8F
:10018000FFFFFFFFFFFFFFFFFFFFFFFFFFFFFFFF7F
:10019000FFFFFFFFFFFFFFFFFFFFFFFFFFFFFFFF6F
:1001A000FFFFFFFFFFFFFFFFFFFFFFFFFFFFFFFF5F
:1001B000FFFFFFFFFFFFFFFFFFFFFFFFFFFFFFFF4F
:1001C000FFFFFFFFFFFFFFFFFFFFFFFFFFFFFFFF3F
:1001D000FFFFFFFFFFFFFFFFFFFFFFFFFFFFFFFF2F
:1001E000FFFFFFFFFFFFFFFFFFFFFFFFFFFFFFFF1F
:1001F000FFFFFFFFFFFFFFFFFFFFFFFFFFFFFFFF0F
:10020000FFFFFFFFFFFFFFFFFFFFFFFFFFFFFFFFFE
:10021000FFFFFFFFFFFFFFFFFFFFFFFFFFFFFFFFEE
:10022000FFFFFFFFFFFFFFFFFFFFFFFFFFFFFFFFDE
:10023000FFFFFFFFFFFFFFFFFFFFFFFFFFFFFFFFCE
:10024000FFFFFFFFFFFFFFFFFFFFFFFFFFFFFFFFBE
:10025000FFFFFFFFFFFFFFFFFFFFFFFFFFFFFFFFAE
:10026000FFFFFFFFFFFFFFFFFFFFFFFFFFFFFFFF9E
:10027000FFFFFFFFFFFFFFFFFFFFFFFFFFFFFFFF8E
:10028000704700BF034613F8012B002AFBD1181A50
:100290000138704700487047A0DA010041207047DC
:1002A0000120704708B506F07FFC08BD08B506F0D0
:1002B000DFFC43690148984708BD00BFA0DA010090
:1002C00010B50C4611461A46012807D010B1022875
:1002D0000BD010BDE0B200F047F8FAE7BDF80830E7
:1002E000C9B2E0B200F082F8F3E7E0B200F046F9FC
:1002F000EFE700BF054B00229A80DA805A819A818D
:10030000B42119811A765A769A7670473C250020D6
:10031000014B1878704700BF3C25002010B40446FC
:10032000034B0FCB84E80F00204610BC704700BF82
:10033000402500200346054901F114024869186070
:10034000098B927999809A71184670473C25002054
:10035000044B187E012803D0987E003018BF01207E
:10036000704700BF3C25002010B504461D4B1B788C
:1003700013F0030F02D010F00C0F15D114F0030F7F
:100380001CD113F0080F02D014F0040F22D113F087
:10039000040F15D014F0080F12D0124B00229A80CF
:1003A000DA80B4221A810BE006F0FEFB02690D4BE5
:1003B0001A61FFF79FFF00F019F901E0FFF79AFFBC
:1003C000084B1C70084C204600F08AFE204600F0C6
:1003D00037FB10BD034B00229A80DA80B4221A81C9
:1003E000EEE700BF3C250020A8DA010010B5044666
:1003F00000F09EFF042C00D010BDFFF789FF10F025
:100400000C0F05D000F0A5FF4368984700F0F8F8FE
:10041000564C204600F0B2FE204600F0B7FB544B8D
:100420001A78042A30D0082A46D0514B5B89B3F59C
:10043000616F05D34E4B0021598199890131998112
:100440004B4B99894EF66023994250D0484BD9883E
:100450004EF6602399424ED0454B99884EF6602364
:1004600099424CD012F0080F4DD1414B1B8BB3F584
:10047000807F76D03E4B9B7E13B1013B3C4A937606
:100480003B4B1A7E5A76B7E73949CB8801339BB28A
:10049000CB803849A1FB0301490901EB8101A3EBA2
:1004A000C1039BB2002BC0D1314B59890131598115
:1004B000196901311961B8E72D490B89013B0B819D
:1004C0008B8801339BB28B802B49A1FB0301490927
:1004D000C1EB0111A3EB81039BB2002BA5D1244BEF
:1004E0005989013159811969013119619DE7204B01
:1004F00000219981AAE71E4B0021D980ACE71C4B53
:1005000000219980AEE700F024FF43689847036814
:10051000984760B9164B1B7813F0080FA5D0134805
:1005200000F066FE78B1124BB4221A819DE700F00C
:1005300010FF4368984700F0ACFD0128EAD10C4B4E
:10054000B4221A81E6E70A4B1B7813F0080F8CD00F
:10055000074B1B89002B88D106F08AFB036898475C
:1005600083E7034B06229A768AE700BFA8DA0100E8
:100570003C250020CDCCCCCC8988888810B50728B4
:1005800019D8DFE800F019041D201823262C06F0E6
:100590000BFB044606F06CFBC3684FF4806200213D
:1005A00020469847FFF7A6FE0E4800F099FD04F19B
:1005B000F00000F032FA10BD0A4800F0B5FDFAE78D
:1005C000094B1975F7E7084B5975F4E7064B997510
:1005D000F1E7054BD975034800F082FDEBE7024BCC
:1005E0001976E8E7A8DA01003C25002008B5882242
:1005F0000021024819F01BF908BD00BF5825002052
:100600002DE9F04F85B080460022904911F8323034
:100610006FF3C71301F8323001EBC20358786FF360
:10062000C710587098786FF3C7109870D8786FF328
:10063000C710D87018796FF3C710187158796FF315
:10064000C710587198796FF3C7109871D8796FF304
:10065000C710D8710132112AD8D1D8F80030984784
:100660000390002302934FF04C0A42E04FF0010E3A
:100670001427B54238D8CDF804B0334676469E46A6
:100680002AE04FF0010E1427F3E7425C42F08002AB
:10069000425402F07F0202EB0709B9F14C0F0FDD63
:1006A000425C6AF30602425401339BB29C420FD370
:1006B00019461CF80320D209E7D0002EF4D0E4E755
:1006C0003A4410F8019062F3060900F80190EBE754
:1006D0000135ADB2AE4507D3A345F9D8019B5B4ABE
:1006E00002EBC50C6046E3E7029B013302930A2B41
:1006F00064D09DF80890D8F82830484698470128DB
:1007000005D0D8F82830484698470228ECD1D8F8C8
:100710000C30484698470446D8F810304846984769
:10072000074600EB00134A4A82FB0325DB17C3EBA5
:1007300025250194E300474A82FB03241C44DB1770
:10074000C3EBA424D8F8183048469847D8F80830A6
:1007500048469847002814BF11230323AEB2F51A68
:1007600025EAE575ADB21E44102EA8BF1026B6B21C
:10077000A4B2E21A22EAE2721FFA82FB1C44072C9E
:10078000A8BF0724A4B2D8F8083048469847019B70
:10079000A3F146091FFA89F9B9F56B7F3FF666AFF9
:1007A0009A2F7FF66EAF002814BF14270127002868
:1007B00014BF4FF0010E4FF0000E5AE70026234FF2
:1007C0001FE0043AE55C62F30605E55404E0013AF3
:1007D000E55C62F30605E5540133082B0ED0C25CDC
:1007E000D209F9D1C25C02F07F02122AEFD8032AA3
:1007F000E7D8E25C6FF30602E254EDE70136112E12
:1008000004D0002307EBC6000446E8E7039B1BB1B6
:10081000002421460D4D05E0FFF7E8FEF8E701341E
:10082000112C0DD0002305EBC400C25C02F07F0246
:10083000092A84BF013189B20133082BF5D1EEE7D3
:10084000024BA3F8881005B0BDE8F08F58250020B2
:10085000B5814E1B49D6B9F22DE9F04F83B006465B
:10086000019114460368984770B13E4A92F88A3065
:10087000013382F88A30A146002C5ED00027B846AA
:100880009346DFF8E8A037E0FFF7B0FE4FF000082E
:10089000019B83F8008055E0F3682046984740B3F9
:1008A00033692046984720B3F368204698470546A9
:1008B00033692046984700EB00108AFB0023C017DD
:1008C000C0EB232080B2ED00274B83FB05232B4494
:1008D000ED17C5EBA325ADB20BEBC000435D03F0F4
:1008E0007F03122B05D808F101085FFA88F8019BF5
:1008F0001C7001374F4510D0FCB2B36A20469847B0
:100900000128C9D0B36A204698470228C4D0B36AE8
:10091000204698470328ECD1BEE7B8F1000F0CD071
:10092000104BB3F88830442B10D8B8F1010F09D020
:1009300012D90023019A137004E04FF00008019BC4
:1009400083F80080404603B0BDE8F08F4FF0000808
:10095000019B83F80080F5E74FF00008019B83F8C6
:100960000080EFE75825002049D6B9F2B5814E1B2B
:10097000431E9BB24FF6FD7293421BD84B1E9BB297
:10098000934219D801EB01110C4B83FB0131090A89
:10099000C0000B4B83FB00231844C0F38F20094B8E
:1009A00003EBC101085C00F07F0013288CBF00201E
:1009B000012070470120704701207047B5814E1B10
:1009C00049D6B9F258250020F8B506460F4C2568DF
:1009D000238903EB83035B00F4336B8006F048F953
:1009E0000435238903EB830307690A22314605EBAB
:1009F0004300B847238901339BB223812268527890
:100A00009A4201D800222281F8BD00BFE4250020CF
:100A1000704708B5FFF7D8FF08BD10B5044606F0CB
:100A200027F9C3684FF44472002120469847034BCE
:100A30001C60462363700A23237010BDE425002048
:100A400030B5A5B00446436898474F4B1B7913F067
:100A5000030F09D0A368984710F0080F21D1A368AD
:100A6000984710F0040F1CD1474B1B7913F00C0F63
:100A700009D0A368984710F0020F41D1A3689847A6
:100A800010F0010F3CD1A36898473F4D2871E368EF
:100A900004A89847BDF81830EB8000236B8125B07F
:100AA00030BD002501950295ADF80C5006F0E0F838
:100AB000C3680A22294601A898479DF804300222FB
:100AC00062F302038DF80430E36810A89847BDF87C
:100AD0000430BDF8462062F30F13ADF80430E3682C
:100AE0000CA89847BDF83E30ADF80630E36808A87A
:100AF00098470B9BADF8083001A8FFF765FFB3E7F7
:100B0000002501950295ADF80C5006F0B1F8C368C8
:100B10000A22294601A898479DF80430032262F36F
:100B200002038DF8043063689847BDF804300288EA
:100B300062F30B13ADF80430134A52891209C3F360
:100B4000072362F307138DF80530E36820A8984760
:100B5000BDF88230ADF80630E3681CA89847BDF8B0
:100B60007030ADF80830E36818A89847BDF86E30CB
:100B7000ADF80A30E36814A89847179BADF80C301D
:100B800001A8FFF721FF7EE7E42500202DE9F04FC3
:100B9000A9B0044643689847A368984710F0080F27
:100BA00004D1A368984710F0040F39D02368984700
:100BB00043689847054600F06CFA80B1236898476F
:100BC000436898478146002704970597ADF8187049
:100BD00002460A2104A800F048FAB846EEE028468A
:100BE00000F05BFA0028E9D163689847B0F86030FC
:100BF000002B40F07381B84BDD880135E36818A8FD
:100C00009847BDF868309D4200F0D781E3680EA890
:100C10009847B14BBDF84020DA805A8901325A8199
:100C200029B0BDE8F08FF368284698473369284615
:100C300098472368984743689847834600F035FAF9
:100C4000B0F1000AC0F2448163689847C388ADF8E8
:100C50000830636898470389ADF80A30636898479D
:100C60004388BDF808201344ADF80C3063689847FA
:100C70008388BDF80A201344ADF80E305FFA8AFA73
:100C8000DBF80C30504698470190DBF810305046A6
:100C9000984702AA0146019800F0C0F9002840F0E8
:100CA00019814FF4C973ADF8083040F66A03ADF806
:100CB0000A3040F2A623ADF80C3040F62413ADF80C
:100CC0000E30DBF80C30504698470190DBF81030BE
:100CD0005046984702AA0146019800F09FF900305B
:100CE00018BF01209DF8223060F345138DF82230A3
:100CF0006368984790F86330C3F302039DF824209B
:100D000063F302028DF824206368984790F866A088
:100D10000AF0FD0A6369984701280ED14AF0020AD9
:100D20006368984790F86830FF2B06D0636898474F
:100D300090F86830013380F868306368984780F82D
:100D400066A063689847BDF8243090F8662062F387
:100D5000C803ADF82430B368284698479DF825307D
:100D600060F382038DF82530B369284698471F2821
:100D700028BF1F20BDF8223060F38A13ADF822305F
:100D8000F369284698471F2828BF1F209DF8233065
:100D900060F3C7038DF82330336A28469847C0F3C1
:100DA0008F001F2828BF1F209DF8253060F3C70340
:100DB0008DF8253007A8FFF707FE0137D9F8003076
:100DC0009847FBB28342BFF40FAFFBB228AA13448B
:100DD00013F8905CCDF81C80CDF82080ADF824800D
:100DE000D9F8283028469847012805D0D9F8283066
:100DF000284698470328E0D12368984743689847D6
:100E00000646E3680AA89847BDF82CA005F030FF15
:100E1000C3680A22414607A898479DF81C306FF323
:100E200002038DF81C30B36A28469847012814BF86
:100E3000002001209DF81C3060F3C3038DF81C30A6
:100E4000BDF81C30BDF82E2062F30F13ADF81C3036
:100E50004FEA1A129DF81E3062F303038DF81E301C
:100E60009DF820306AF303038DF82030F36828469C
:100E70009847BDF81E3060F30F13ADF81E3033698C
:100E800028469847BDF8203060F30F13ADF82030A6
:100E9000236912A898479DF822309DF8482062F3F4
:100EA00001038DF82230736A284698479DF8223056
:100EB00060F383038DF8223003F00C030C2B7FF4D6
:100EC000B2AE9DF8223043F00C038DF82230AAE632
:100ED000404607E7012005E7E425002000230A93A8
:100EE0000B93ADF83030236898474368984706461F
:100EF00000F0DBF8051E4FDB05F0BAFEC3680A22DE
:100F000000210AA898479DF82830012262F30203C5
:100F10008DF82830E36814A89847BDF82830BDF84C
:100F2000562062F30F13ADF828306368984790F8A5
:100F3000603013F0020F3AD16368984790F8603040
:100F400013F0040F35D16368984790F8603013F0C0
:100F5000080F30D16368984790F8603013F0100F95
:100F600014BF062200229DF82A3062F303038DF895
:100F70002A30EDB2F36828469847BDF82A3060F36E
:100F80000F13ADF82A30336928469847BDF82C3046
:100F900060F30F13ADF82C300AA8FFF715FD636856
:100FA00098470023A0F860301B4A538123E60122B2
:100FB000D9E70422D7E70522D5E700250A950B9546
:100FC000ADF8305005F054FEC3680A2229460AA83D
:100FD00098479DF82830042262F302038DF82830E8
:100FE000E36824A89847BDF82830BDF8962062F33E
:100FF0000F13ADF82830E36820A89847BDF88E306D
:10100000ADF82A30E3681CA898471F9BADF82C3038
:101010000AA8FFF7D9FCF9E5E4250020134672B1D0
:10102000128882420DD89A8882420CD3DA888A428A
:101030000BD3588888428CBF0020012070470020C5
:10104000704700207047002070470020704710B59F
:101050000446084611460023224600F0BBF9002151
:10106000204600F0E4F9C0B210BD08B5002300F03E
:10107000B1F908BD08B500F0ADF908BD08B500210B
:1010800000F0D5F9C0B208BD08B500F0D0F9C0B283
:1010900008BD08B500F076F908BD08B500F086F97E
:1010A00008BD08B500F05AF908BD08B500F0E6F92A
:1010B00008BD000010B5436898470488003418BF85
:1010C000012405F0D5FD83682246032102209847BC
:1010D00005F0CEFD8368224603210420984710BD09
:1010E000F8B507460F4B1B68BBB1002425460D4ED3
:1010F00056F8253053B156F82530984703682BB180
:1011000056F8253098470368384698470134E4B2CA
:10111000254656F82430002BEAD13846FFF7CAFF9F
:10112000F8BD00BF2C100020F8B50746124B1B6815
:10113000F3B100242546104E56F825308BB156F8F1
:101140002530984743683846984750B156F82530BF
:101150009847C3682BB156F825309847C36838467E
:1011600098470134E4B2254656F82430002BE3D1E9
:101170003846FFF79FFFF8BD2C1000202DE9F04105
:1011800007461A4B1B68002B2DD000242646174D0E
:1011900005E00134E4B2264655F824301BB355F877
:1011A0002630002BF5D055F826309847436838464E
:1011B00098470028EDD055F82630984790F81480CD
:1011C000BB68984718EA000FE3D055F826309847D7
:1011D0008368002BDDD055F8263098478368384661
:1011E00098470028D5D0BDE8F08100BF2C10002022
:1011F0002DE9F04107461C4B1B68002B32D0002420
:101200002646194D05E00134E4B2264655F824304F
:101210002BB355F82630002BF5D055F826309847DB
:101220004368384698470028EDD055F8263098474F
:1012300090F81480BB68984718EA000FE3D055F87F
:10124000263098470369002BDDD055F826309847A3
:101250000369384698470028D5D0012000E00020D7
:10126000BDE8F0810020FBE72C10002008B54368A2
:1012700098470078C0F3400008BD704730B587B08C
:101280000446036898474368984702461F4903A8E5
:1012900000F0D9FE9DF8153013F0020F2ED0BDF8E6
:1012A0000C30CD3B9BB240F29D22934229D8BDF831
:1012B0000E2040F6B7039A4225D99DF81430043B1E
:1012C000DBB2382B01D9002019E0002301930293EF
:1012D0004FF00203012565F387138DF8043005F004
:1012E000C7FC436801A898476368984790F8603046
:1012F00043F0020380F86030284600E0002007B089
:1013000030BD0020FBE70020F9E700BFF0250020FA
:1013100008B540F2411354224021024800F07EFEFD
:1013200008BD00BFF025002000487047C0DA01006A
:1013300010B51446012802D0022805D010BD1A4667
:10134000204601F04DF8F9E71946104601F006F87D
:10135000F4E70148704700BFD8DA010038B5054608
:101360000368984748B10024AB68E0B29847034649
:1013700030B901340A2CF7D100E00023184638BDFB
:101380000123FBE738B505460368984750B10024B0
:10139000AB6AE0B29847012806D001340A2CF7D195
:1013A000002000E0002038BD0120FCE738B50546EC
:1013B0000368984750B10024AB6AE0B2984703280D
:1013C00006D001340A2CF7D1002000E0002038BDFF
:1013D0000120FCE72DE9F84F8246894616469846DB
:1013E00000252F4609E07B1CDBB20AF807404B457D
:1013F0001BD01F4601350A2D17D0ECB2B36A204628
:1014000098470028F6D0F36820469847834633690A
:1014100020469847B8F1000FE5D0424601465846AD
:10142000FFF7FCFD0028DED1E4E7BDE8F88F2DE9E9
:10143000F843074688460024264604E00136F6B203
:1014400001340A2C17D0E5B2BB6A28469847002819
:10145000F6D0FB682846984781463B69284698475E
:10146000B8F1000FEAD0424601464846FFF7D6FDE4
:101470000028E3D1E4E770B2BDE8F88338B505464B
:101480000368984760B10024AB6AE0B2984728B976
:1014900001340A2CF8D14FF0FF3038BD60B2FCE7C0
:1014A0004FF0FF30F9E7000008B54368984700782F
:1014B000C0F3C00008BD064B46221A809B225A800A
:1014C00040F2F2329A8040F6D902DA80704700BFCB
:1014D0000C260020F0B585B0044643699847244D9A
:1014E000A8762368984743689847024605F10801A3
:1014F00002A800F068FC9DF80830022B03D00025FC
:10150000284605B0F0BDBDF80A70BDF80C602A464B
:1015100031463846FFF782FD05460028F0D000230B
:10152000009301934FF00203042262F38503012527
:1015300065F387138DF8003047FA02F38DF8023017
:1015400046FA02F38DF8033006F00F0646EA071656
:101550008DF8046005F08CFB436868469847636823
:10156000984790F8603043F0080380F86030C7E790
:101570000C26002030B585B00C4C4625039564231D
:1015800002931E230193032200921223012104F1EE
:10159000080000F0F1FB25809B23638040F2F233CA
:1015A000A38040F6D903E38005B030BD0C260020AF
:1015B00000487047E0DA010008B5436898470378AF
:1015C00013F0240F14BF0120002008BD38B5436874
:1015D0009847C58804894188294482882244034B5E
:1015E0005D809C80D9801A8138BD00BF44260020D0
:1015F0002DE9F04784B08046436898470378C3F3E9
:101600008009C3F34017D8F8143098473F4D85F848
:101610002600D8F80030984743689847024605F1FD
:10162000140102A800F0CFFB9DF808A0BDF80A60E5
:10163000BDF80C40AA1C21463046FFF7EFFC30BB3A
:1016400005F10A0221463046FFF7E8FC0346002870
:101650005AD1184604B0BDE8F0872C4B1A7000230D
:10166000F7E71FB3294B1B78012B1FD00023F0E7AE
:10167000D8F80430984790F8603043F0040380F8BD
:1016800060300123E5E70023E3E70023E1E70022E0
:10169000BAF1010FE1D0BAF1020FF4D1B9F1000FA4
:1016A000DFD01FB9194B1B78002BEED1002301931B
:1016B0004FF00203012262F3850362F387138DF872
:1016C0000030124D2B788DF8013033118DF8023037
:1016D00023118DF8033004F00F0444EA06168DF848
:1016E000046005F0C5FA4368684698472B78002BDC
:1016F000BED0D8F80430984790F8603043F020030B
:1017000080F860300123A4E70122C1E744260020CD
:1017100030B587B00546036904A898479DF8133093
:1017200053BB254C462303935D230293242301934B
:101730000523009312230222114604F1140000F045
:101740001BFB6B689847C588018942882A448388B7
:101750000B446580A180E28023819B22164B4621A9
:1017600059819A8140F2F232DA8140F6D9021A8226
:1017700000221A7007B030BD0F4C0A2303935D237B
:1017800002932423019307230093122303220221AF
:1017900004F1140000F0F0FA6B689847C5880189DD
:1017A00042882A4483880B446580A180E28023819B
:1017B00040F2DE42D2E700BF4426002000487047D6
:1017C000F8DA010070B5064600242546736898478C
:1017D000204445760134182CF8D170BDF8B5036863
:1017E00098474368984705460C4CC368A07A9847C9
:1017F00006462B69A07A98470746AB6AA07A9847B5
:10180000022801D00020F8BD04F114023946304608
:10181000FFF704FC003018BF0120F4E78826002001
:1018200038B5044643689847037D012B0CBF01215E
:101830000321244800F0D1FC63689847B0F84B407E
:1018400040F2A513002C18BF23461E4A9382B0F81D
:101850004D1040F2D573002918BF0B46D382B0F863
:101860004F2040F29323002A18BF1346154D2B83B7
:10187000B0F8513040F6C200002B18BF18466883FC
:101880009CB1503CA4B20F48848389B1503989B2CD
:101890000C48C1837AB1503292B20A490A846BB1C2
:1018A00050339BB2074A538438BD40F25514EAE7DF
:1018B00040F28571ECE740F2E322EEE740F61213C6
:1018C000F0E700BF882600202DE9F04F8DB00646D6
:1018D00003689847436898470446914901F1140307
:1018E000024609A800F088FCBDF824300093BDF83A
:1018F00026A09DF82D509DF82EB0BBF1010F13D0FE
:10190000874B93F82430012B40F00881A36A2846C6
:10191000984703280DD060B102283DD0BBF1010FDC
:1019200000F0C080002433E07D4B012283F82420A6
:10193000ECE77B4B002483F8244083F825403046B5
:10194000FFF740FF0494022343F00C02012464F3E8
:1019500087128DF80C208DF80D30009A13118DF838
:101960000E304FEA2A138DF80F300AF00F0A4AEAB8
:10197000021A8DF810A005F07BF9436803A8984778
:101980007368984790F8603043F0100380F8603037
:1019900020460DB0BDE8F08F614B93F82530002B49
:1019A000BCD1E368284698470746236928469847EC
:1019B0005C4A01463846FFF731FB60BB0121584BBA
:1019C00083F82510002304934FF00203032262F3EF
:1019D000850361F387138DF80C308DF80D20009A84
:1019E00013118DF80E304FEA2A138DF80F300AF0DC
:1019F0000F0343EA02138DF8103005F039F94368FC
:101A000003A898477368984790F8603043F0100334
:101A100080F8603082E700270397049705970697C0
:101A20000797089716234FF00109CDF804A09A46AE
:101A300024E00135102D19D07C19A4B233689847E1
:101A400003680320984703684146E8B298471E2878
:101A5000EFDD0CAB03EBD40304F0070409FA04F444
:101A600013F8242C144303F8244CE2E71037BFB2D8
:101A70000AF1010A1FFA8AFAC02F03D000255FFA83
:101A80008AF8D9E7DDF804A003AF0DF124083C463D
:101A9000E51B7368984714F8013B28444376A0453A
:101AA000F6D13BE7204ABDF82A10BDF82800FFF721
:101AB000B5FA044600283FF46BAF73689847027D7F
:101AC000012A14BF00220122002304934FF00203D5
:101AD000032161F38503012464F387138DF80C302F
:101AE0008DF80D20009A13118DF80E304FEA2A134D
:101AF0008DF80F300AF00F0343EA02138DF810300F
:101B000005F0B6F8436803A898477368984790F8BB
:101B1000603043F0100380F8603039E7002437E785
:101B200088260020A42600209C26002010B54368AB
:101B300098470478C4F300140CB9204610BD05F092
:101B400097F883680122032110469847F5E770B59E
:101B5000044643689847037D012B114E4FF0500314
:101B60000CBF012203221946304600F038FB002545
:101B700086F8245086F825502046FFF723FE636838
:101B8000984710234375636898470C2383756368EF
:101B900098471823C37563689847057670BD00BFE2
:101BA000882600200048704710DB010010B504466D
:101BB000028B038A9A4202D90123C375037594F8F4
:101BC0002730012B12D0A37C012B14D0A27D0D4B0A
:101BD00053F8223020469847012811D0022814BF1C
:101BE00000200220A38D0133A38510BD0423E375DB
:101BF00001232375E7E70523E37501232375E5E753
:101C00000120EFE740100020C289B0F91A30B0F986
:101C100022105B1A002BB8BF5B42934218DCB0F96C
:101C20001C30B0F924105B1A002BB8BF5B429A42FB
:101C300010DBB0F9282043889A4207DCB0F92C3039
:101C400040898342CCBF00200120704700207047AC
:101C5000002070470020704770B5044690F8265069
:101C6000012D05D9AB1EDBB2012B08D9002070BDB8
:101C7000012303750020A0750323E375F7E7068DA4
:101C8000013636B20685FFF7BFFF08B90123237579
:101C9000032D01D00020EAE723889E42BCBF012328
:101CA000237563889E42C4BF012323750023A37557
:101CB000627D237B9A4201D00020D8E7B4F92A3014
:101CC000A2889342BCBF01222275E2889342C4BF1E
:101CD00001232375B4F92C3022899342BCBF012221
:101CE000227562899342C4BF012323750023638553
:101CF000237D4BB100202075A685E38B6383238C65
:101D0000A38301236375B2E7002363750220AEE766
:101D100010B5044690F8263023B9438D013343852E
:101D2000002010BD012B25D1FFF76EFF18B902234B
:101D3000E3750123237501222285637D1344DBB201
:101D40006375A275B4F92210E183B4F924202284CA
:101D50003BB1237D2BB9607D012814BF00200120F9
:101D6000DFE7002020750123A38560856183A283BE
:101D70006375F0E70020D4E730B4BDF80850BDF833
:101D80000C400280438001FB02F292B2AB1A8380C6
:101D9000A21AC280058144810173BDF81030C3814D
:101DA000BDF8143003820023037543754385838592
:101DB0000385C3754FF6FF7242838283C283028418
:101DC000837530BC7047F0B585B005460C461646A5
:101DD000002301930293ADF80C30898B608BFEF7E2
:101DE000C7FDD0B10A2201A93046FEF735FD012812
:101DF00022D90023237563756385A3852385E37545
:101E00004FF6FF726283A283E2832284A3752B7054
:101E10006B80AB80284605B0F0BD00232375637549
:101E20006385A3852385E3754FF6FF726283A283E2
:101E3000E2832284A375D5E79DF8047000B3F368AC
:101E4000384698476084336938469847A084B36A17
:101E50003846984784F82600B36938469847208367
:101E60003046FFF71EF9A0B9002384F8273020463A
:101E7000FFF79CFE628BA38B28706A80AB80C9E75A
:101E80004FF6FF736384A384002384F826302383F2
:101E9000E6E7012384F82730E9E700BF70B5044680
:101EA0000E4615788B6A28469847012801D00120F4
:101EB00070BD002323806380A380E380238163813E
:101EC000A381E38123746374227E02F0F80263F33A
:101ED000C3022276F36828469847A08133692846D2
:101EE0009847E081237C01332374E0E72DE9F0413A
:101EF00004460F461678CB683046984780463B69C3
:101F0000304698470546BB6A30469847032841D07B
:101F1000A389A8EB03031BB22380B4F902209A42E1
:101F2000B8BF1A4616466280B4F904709F42A8BF33
:101F30001F46A780E089281A00B2E080B4F9082083
:101F40008242B8BF02462281B4F90A108142A8BF7A
:101F500001466181B4F9125001EB050C604553DA7A
:101F6000491B884250DD521B904203DC227E42F026
:101F700002022276EA1993424BDA7F1BBB4248DD0C
:101F8000721B9342DEBF237E43F0080323760120B9
:101F9000BDE8F08100232374B4F90020E38A9A425B
:101FA00022DB217E01F00801002914BF002010204F
:101FB00059428A4206DC227E12F0040F04BF40F030
:101FC0000800C0B2B4F9062093420FDC237E13F060
:101FD000020F0BD140F00400C0B29142D8DB237E47
:101FE00013F0010F08D0D3E70020E1E7914207DBAF
:101FF000237E13F0010F03D140F00200C0B2C7E707
:10200000002808BF0120C3E7217E41F001012176AD
:10201000A9E7227E42F004022276B1E74182828261
:10202000C3820023038043808380C3800381438174
:102030008381C38103744374027E02F0F80263F368
:10204000C302027670472DE9F04186B004460D4682
:10205000164600238DF81730314903AA03C982E8D8
:10206000030000930193ADF808300A226946304618
:10207000FEF7EDFF80469DF800708DF81770B36A8B
:1020800038469847002831D0B8F1010F2ED1B369F6
:1020900038469847AB8A834228D3B3683846984776
:1020A00020BBF3689DF817009847804633699DF878
:1020B0001700984707462B7C06AA02EB830353F8C8
:1020C0000C3C0DF11702314628469847A989EA8948
:1020D0006B7C5E1C6E7421806280A4F80480E780B3
:1020E00023726072204606B0BDE8F08100232B8089
:1020F0006B80AB80EB802B816B81AB81EB812B7490
:102100006B742A7E02F0F80263F3C3022A762380FE
:102110006380A380E380237201236372E2E700BF40
:1021200028DB010070B504460E4615468B6A104642
:102130009847012801D0002070BD0023237223801E
:102140006380A380E3806372A372E372F36828461E
:10215000984720803369284698476080A572637A43
:1021600001336372E7E7F8B504460E4615468B6AFD
:10217000104698470746F36828469847A080336979
:1021800028469847E080238A9BB9A289B4F9003099
:10219000B4F904105B1A002BB8BF5B42934213DC06
:1021A000B4F9023000B2181A0028B8BF4042824287
:1021B0000ADB227AE3899A4209D300236372E07A28
:1021C000B0FA80F04009F8BD0123E372F1E7032F74
:1021D0004FF0000008BF6072F5E7C1817047818150
:1021E000C281038200230372038043808380C38003
:1021F00043728372C37270472DE9F04186B0044682
:102200000D4617461E460023036043608360039318
:102210000493ADF814300B8A3288D21AADF804203A
:102220007288D21AADF80620B2881A44ADF8082098
:10223000F2881344ADF80A3001A93846FEF724FFAE
:10224000804631463846FEF71FFFB8F1010F0DD02A
:10225000AA7A00236B7223806380A380E3802372B9
:102260006272A372204606B0BDE8F08108B900236F
:102270002B7201AB3A460A2103A8FEF7FBFE6A7AED
:102280000D4B53F822309DF80C20394628469847CC
:10229000B5F800C06F88AE88E9882B7AAA7A03F176
:1022A000010E85F808E0A4F800C06780A680E180F0
:1022B00023726272A072D5E748100020014B188883
:1022C000704700BFB02600200A207047024B5B68B1
:1022D00003EB0010807B7047B0260020024B5B6848
:1022E0000001185C704700BFB0260020024B5B68FD
:1022F00003EB001040887047B0260020024B5B685B
:1023000003EB001080887047B0260020024B5B680A
:1023100003EB0010C0887047B0260020024B5B68BA
:1023200003EB001000897047B0260020024B5B6869
:1023300003EB001040897047B0260020024B5B6819
:1023400003EB001080897047B0260020024B5B68C9
:1023500003EB001040787047B0260020014B198035
:1023600058607047B02600200048704730DB0100FD
:10237000C0F10F0000EB001001EB4000024B1B68A6
:1023800033F91000704700BFB8260020C0F10F00DD
:1023900000EB001001EB4000024B5B6833F91000CA
:1023A000704700BFB8260020C0F10F0000EB0010FE
:1023B00001EB4000024B9B6833F91000704700BFEF
:1023C000B8260020C0F10F0000EB001001EB400028
:1023D000024BDB6833F91000704700BFB8260020BD
:1023E000014B43F821007047B8260020014B03EB56
:1023F000800070475CDB0100704700BF2DE9F043AF
:10240000054683B0092002F003FC80460A2002F052
:10241000FFFB07460DF088F90446194E98F80000B6
:10242000184902F007FCDFF86C9032462046002184
:1024300003F052FCEDB298F80000134902F0FAFBE9
:102440002B4642462046494600960EF0C7FC387897
:102450000E4902F0EFFB32462046002103F0F2FF66
:1024600038780B4902F0E6FB00962B463A4609F114
:10247000240120460EF000FD03B0BDE8F08300BF4C
:10248000CD4C0000BD5E0000815E0000A56600002E
:10249000AD650000500E002030B50024134B144DE4
:1024A00083B01A6829466320009400F009FD0120DA
:1024B000FFF7A4FF0F4B29461A68632000F000FDC8
:1024C000012320468DF80030009BDAB262F307004A
:1024D000C3F3072262F30F20C3F3074262F31740EE
:1024E0001B0E63F31F6003B030BD00BFA0040020CB
:1024F0009C9A0100A404002038B50B4B0B491A68C4
:10250000632000F0DDFC0A4C04F1180554F8043B8C
:102510001B699847AC42F9D1064B04491A686320FD
:10252000BDE8384000F0CCBCA0040020D89A0100DF
:1025300028000020A404002010B50B4B0B4C1A6897
:102540002146632000F0BCFC094A0A4B127853F87C
:102550002230DB689847084B2146BDE810401A68D6
:10256000632000F0ADBC00BFA0040020CC9A0100A5
:102570005010002028000020A404002010B50B4BB0
:102580000B4C1A682146632000F09AFC0021094B8D
:10259000094A1B6811705B689847084B2146BDE8E3
:1025A00010401A68632000F08BBC00BFA00400201C
:1025B000C09A01002800002050100020A404002030
:1025C0000023F0B55F4C8DB003A8019307F0AEF97E
:1025D0002378002B00F082805B4A5C4B127853F822
:1025E00022309B689847237801909DF81B209A42DF
:1025F0006AD09DF81B30DBB2002B23700CBF022485
:102600000124534B9DF82E201978914205D09DF856
:102610002E00C0B21870002853D09DF8243013B19A
:1026200001238DF804309DF825301BB10122494B60
:1026300083F822209DF81330EBB9434B1B78032B12
:102640001CD0012C1FD0022C31D09DF80420002A70
:1026500049D10020019BDAB262F30700C3F30722DD
:1026600062F30F20C3F3074262F317401B0E63F3BC
:102670001F600DB0F0BD07F04FF938BB0123012CEE
:102680008DF80430DFD106232F4C8DF804302378E9
:10269000042BDED0042637462C4D55F82330DB685A
:1026A000984755F8273026705B689847D1E707238D
:1026B000254C8DF804302378052BCAD005263746E3
:1026C000EAE709F0DBFDA8E700249AE71E4B1B7838
:1026D000012BB6D804238DF80430B2E79DF81B20F7
:1026E000002A82D178E7184C013A21780B46062A55
:1026F000AFD801A050F822F0152700002D270000C8
:1027000053260000232700005326000091260000D6
:10271000B926000000299CD001290CD0002637469C
:10272000BAE7032995D003263746B5E7012990D0AB
:1027300001263746B0E700220748164602701746C2
:10274000AAE700BF521000205010002028000020EF
:1027500051100020E40D0020E00D002038B5114B91
:1027600011491A68632000F0ABFB0AF013FB10B9A3
:102770000E4B1A789AB90E4C04F1180554F8043B24
:102780001B689847AC42F9D100240A4B0A4A1C70D6
:10279000126805496320BDE8384000F091BB18700D
:1027A000E9E700BFA0040020B49A01005210002005
:1027B0002800002050100020A404002030B4184D40
:1027C0000022D5F8014001322346186802EBC2010D
:1027D000294480B1586898B19868B0B1D868C8B138
:1027E000042A1BD0D1F801300132186802EBC20173
:1027F00029440028EED12068186058680028EBD1E1
:102800006068586098680028E8D1A0689860D86827
:102810000028E5D1E068042AD860E3D130BC7047D5
:102820004004002030B4184D0022D5F80140013298
:102830002346186802EBC201294480B1586898B158
:102840009868B0B1D868C8B1042A1BD0D1F801305B
:102850000132186802EBC20129440028EED1206839
:10286000186058680028EBD16068586098680028A4
:10287000E8D1A0689860D8680028E5D1E068042A0B
:10288000D860E3D130BC70477004002010B502F06E
:1028900073F8094B1B689847084B1B689847084B0F
:1028A0001B689847BDE81040064A074B127853F85A
:1028B00022305B68184700BF14000020A80D0020DC
:1028C000700D002054100020E0A20100F0B500249B
:1028D000A3B017AE214630462C2211ADCDE91144EC
:1028E000CDE913441594ADF8584016F0A0FF0BAB9A
:1028F000CDE90333CDE90844CDE90644CDE90056DE
:10290000074F05930EA80C940B94CDF833402B463B
:102910003C682A46029029460B20A04723B0F0BD10
:10292000C02700200B4A08B512780B4B53F8223011
:10293000DB689847FFF7CAFF084B1B699847084BAD
:102940001B699847074B1B699847BDE8084001F091
:10295000AFBF00BF54100020E0A20100140000200F
:10296000A80D0020700D002070B505468AB007F054
:102970008DFA022D24D0032D20D0012D044614BF42
:1029800004460024274D2B78A34215D001A806F059
:10299000CDFF2B78012B15D0234E56F82330DB6862
:1029A000984756F824302C705B68984728780AB00E
:1029B000BDE8704007F070BA0AB070BD0224E1E7CC
:1029C0000124DFE7002CE7D19DF826309BB90AF0FF
:1029D000E1F9D8B100242A78134B53F82230DB6890
:1029E0009847124B2C705B68984722461049642028
:1029F00000F066FADAE709F083FB044609F01AFBF7
:102A00000AF0C8F90028E5D1002CE3D10024FFF733
:102A100089FF2C70FFF73AFF22460649642000F038
:102A20004FFAC3E754100020E0A201001400002078
:102A30008CA20100B8A201002DE9F04790B006F089
:102A400051FF07A806F072FF584A594B1278594DAA
:102A500053F822309B6898470690C0F30729C0F3CB
:102A6000074404F08BF807F021FA2A789DF8223009
:102A700082469A4206D09DF8220005F0D7FE9DF8C6
:102A800022302B70012500264B4BDFF84C819868D3
:102A900005F006FA49484A4F2A462946434603901C
:102AA000CDE901660095642000F0BEF93B6898F816
:102AB0000020997891420FD0CDE901662E46414A17
:102AC0000233039200952A462946642000F0ACF9AF
:102AD0003B689B7888F800300DF08AF93B688DF8E8
:102AE0001700DB7883421BD1BAF1000F29D146BB16
:102AF0005CB39DF83530002B9DF8343018BF0024AE
:102B00003BB3002007F0C8F94FF00109012C2DD08C
:102B100074BB4846FFF728FF012010B0BDE8F087DE
:102B2000012200232848CDE9013303900DF117035A
:102B300064200092114600F077F93B68D8780DF0D8
:102B400043F9002007F0B8F902249DF83430002B37
:102B5000D7D19DF82B30FBB99DF82330002BD5D071
:102B600007F094F90228CCD0012CD1D10EF01CFF33
:102B7000164B17491A68632000F0A2F9FFF7D2FE3E
:102B8000FFF784FE134B12491A68632000F098F98E
:102B9000012010B0BDE8F08707F078F90228B0D026
:102BA0009DF82330002BB1D0DAE700BF541000208D
:102BB000E0A20100531000207406002058A201007A
:102BC000A806002064A2010080A20100A004002049
:102BD00044A20100A4040020D40400202DE9F04701
:102BE0009CB0044603A8884606F0A0FE00235B4E76
:102BF0009DF82320C6E90033C6E902333382002A58
:102C000058D094F82B0094F82AA094F829905045B5
:102C100094F828E03AD8A0F11D01A0F11007821E17
:102C2000C9B2FFB2D2B2F14526D84B4614E0A3F1A7
:102C30000B04022C41D803EB031400EB440438F9D5
:102C40001450002436F914C0AC45B8BF26F814500F
:102C50000133DBB29E450FD3022AE8D9022F37D8C1
:102C6000A3F10B04022C47D803EB031400EB44043C
:102C700038F914500324E5E70130C0B201310137BF
:102C800001328245C9B2FFB2D2B2CCD23E2200217B
:102C90000DF1320016F0CBFD002340F60115822421
:102CA00000961A460CA91E20ADF830508DF835401C
:102CB00007F0AAFA1CB0BDE8F087DC1F022C29D867
:102CC00003EB031400EB440438F914500124B9E772
:102CD0000229BDD8A3F10B04022C26D9DC1F022C3B
:102CE00033D99C1E022CB3D803EB031400EB44042D
:102CF00038F914500824A5E7DC1F022C1DD99C1EAE
:102D0000022CA5D803EB031400EB440438F914504B
:102D1000052497E79C1E022C9AD803EB031400EBC2
:102D2000440438F9145002248CE703EB031400EB3D
:102D3000440438F91450062484E703EB031500EB30
:102D40004505042438F915507CE703EB031400EB28
:102D5000440438F91450072474E700BF58100020C9
:102D6000F0B5204E83B0054601F1200014461F4601
:102D70007160FDF787FA1C4B1C4A99682130376057
:102D80004860946060782278E37802FB00F203F0F8
:102D90007F0303FB02F3164C22790B60D3B2012BA5
:102DA00001D003B0F0BD7721FF221E46114F3970CC
:102DB00022712379FF2B10D120222946684616F074
:102DC00007FD009B032B04EB830206DC019BD2F87A
:102DD000052006FA03F31342EBD105233B7003B041
:102DE000F0BD00BF401A0020CC060020B008002033
:102DF000EC1C00207C07002070B5154600F1200473
:102E00002046DF220E4616F0D1FD45B13046FDF7D3
:102E100039FA2946C0F1DF02204416F0C7FD2046EA
:102E2000BDE87040FDF72EBAF0B5C3B004460E46BB
:102E300015460146202202A81F4616F0C9FC029B37
:102E4000032B0EDC01221D48039900EB8303D3F80A
:102E500005C002FA01F313EA0C0F02D00379934282
:102E600001D043B0F0BD4FF48072002102A816F0EB
:102E7000DEFC00234B99DF220AA8CDE9003316F0CF
:102E800095FD0AA8FDF7FEF99DF803C0489B499AF5
:102E90008DF8070063F3060C20464A9C62F3C71CBA
:102EA0003B4602A96A468DF800608DF801508DF806
:102EB00006408DF803C0FFF753FFD2E7EC1C00205B
:102EC000F0B5C3B004460D4616460146202202A8BE
:102ED00016F07EFC029B032B0DDC012216490398A1
:102EE00001EB8303D3F8057002FA00F33B4202D0F2
:102EF0000B79934201D043B0F0BD00274FF48072AC
:102F0000394602A816F093FC3246294602A8CDE9BC
:102F10000077FFF771FF3B468DF807006A4602A96C
:102F20002046ADF800708DF803708DF804708DF8B0
:102F30000670FFF715FFDEE7EC1C0020F0B585B04A
:102F4000654601F0C3FE01F0F3FE0021084601F0E2
:102F50009DFBD5E901210446002701200426CDE987
:102F6000010705482346039000967220FFF75CFF97
:102F7000204605B0F0BD00BF9CA401002DE9F0473C
:102F800090F815C082B0BCF1000F2BD01C46002574
:102F90004FEA4C0606EB8C0603EB0616216294F80A
:102FA000247084F8245094F8257084F8255094F8FF
:102FB000267084F8265094F8277084F8275094F8E7
:102FC000287084F8285094F8297084F8295094F8CF
:102FD0002A7084F82A5094F82B7084F82B503034DF
:102FE000A642DBD1BCF1000F2FD098469146824615
:102FF00000269AF814301BB300257700DAF8003069
:1030000006225C5D68466110013116F0E1FB9AF81A
:10301000142004F0010406FB0291009B3C449B0039
:1030200004EB440403EB041401984B5D4444216A0F
:1030300000EB8000834001350B43AA422362DDDCB4
:103040009AF815300136B342D3DC02B0BDE8F08700
:103050002DE9F04100241962196593F8241083F8D2
:10306000244093F8251083F8254093F8261083F820
:10307000264093F8271083F8274093F8541083F8DC
:10308000544093F8551083F8554093F8561083F840
:10309000564093F8571083F8574093F8281083F858
:1030A000284093F8291083F8294093F82A1083F8D0
:1030B0002A4093F82B1083F82B4093F8581083F88C
:1030C000584093F8591083F8594093F85A1083F8F0
:1030D0005A4093F85B1083F85B40017D82B019B3CE
:1030E00006461D46571E3368062213F804806846BC
:1030F0004FEA6801013116F06BFB08F001080099F6
:103100004FEA480290448A0002EB081201992A44CF
:1031100017F8013F106A01EB81018B4003431362F2
:10312000337D0134A342DEDC02B0BDE8F08100BF94
:103130002DE9F04F95B004AFD1F801300446386363
:10314000022100203B6101F0A1FA0021386208460B
:1031500001F09CFA01F0E2FBEC46257D647D80469F
:1031600004FB05F2D01DC008ACEBC0008546EC4660
:10317000960006F10A03DB08ACEBC30C04A8E54695
:1031800000210DF1100CC7F824C0FC62FE607861CC
:1031900016F04DFB3246FF21786A16F048FB0423F7
:1031A00007F1400202F8043D114601207A6001F067
:1031B000DFFC3B699A68AB009178FB61D3781278A9
:1031C0005B1A01339A4240F32F810A234FF0000922
:1031D0002E46BB626300BB60BB6A98491F2B40F35D
:1031E00010811A4601FB03F103EB431302EB431377
:1031F00003EBC33301F1404103F140432031904AD6
:10320000013341F01F018F489362C2E90813303245
:103210008242F8D1012204248B4B0192CDE9029322
:103220000094BD6A11467B686420FD63FFF7FCFDD6
:103230003D6AFA680021284616F0F9FAFB6A002B6D
:1032400000F0D38000234FF0405B7D63BB614FF003
:10325000000A01254FF4FA74BB693A6953441377A5
:1032600001F034FD01F064FD8BF8F350D6B1D7E9DD
:103270000C3C186806EB000E10F8013B03F001024D
:1032800052450BD15B1008EBC313B3F840201988EB
:10329000DCF80030521A1344CCF8003070450CF1C1
:1032A000040CE9D1013C8BF8F390D9D1BAF1000FAD
:1032B00002D14FF0010ACDE77A6BF969BB690A4484
:1032C0007A63BA6802339342BB61C0D104235F4A78
:1032D000CDE90034CDE902423D6A32462B46F96A17
:1032E0006420FFF7A1FD7B6AD7F814A0D7F828B0B7
:1032F000A5F1040CA3F1040E86B1724660460023CA
:1033000050F8041F52F8045FA94238BF0AF803B00E
:1033100003F1010338BF11609E42F1D1FB69013412
:103320009C449E44FB6AB244A342E5D10123484A2F
:10333000CDE90039CDE90292FD6A7B693246294622
:103340006420FFF771FD0423BA6A2946013214464E
:10335000BA62404ACDE90039CDE9029264207B6A25
:103360003246FFF761FD3E2C7FF436AFFB6A3546EF
:10337000B3B100227B6A384E191F5DB10C460020A4
:1033800054F8043F0130A6FB03C385424FEA5313B0
:103390002360F5D1FB6901321944FB6A9342ECD1F9
:1033A000002400222D496420FFF78AFD0122284BCA
:1033B000642003937B69CDE901440092FE6A2A46AA
:1033C0003146FFF731FD224625496420FFF778FD9D
:1033D0000420CDE901441F4B2A4603937B6A314602
:1033E00000906420FFF720FD23E0184B3246039342
:1033F000F96A0094CDE9011164203B6AFFF714FDDE
:1034000094E7BB6A1A4601FB03F103EB431302EB9B
:1034100043130B4A03EBC3330A489362C2E9081310
:1034200030328242F8D1F5E600220E496420FFF7DF
:1034300047FD4437BD46BDE8F08F00BF2084100231
:103440009800046098060460D4A30100E0A3010082
:10345000F4A3010000A40100D34D62100CA40100EC
:1034600020A4010030A401002DE9F043437D8646ED
:10347000007DF3B1002601F1FF3C0F494FEA4308FC
:1034800098B16446DEF80020871812F8019B14F802
:10349000015F09F00103334403EB430301EB031322
:1034A00003EB59039742DD73EFD10236464584445E
:1034B000E6D1BDE8F08300BF9800046070B56446B3
:1034C00084B0DCF800000E460125FFF7CDFFD4E9FB
:1034D00001210020054CCDE90100334600950394FD
:1034E0006420FFF7A1FC04B070BD00BFA0A30100E1
:1034F000427D02B3F0B40026037DDFF83CC0ABB1DF
:1035000000247700056806FB03122D5D05F001031A
:103510003B4403EB43030CEB031303EB5503DB7B4F
:103520001355037D0134A342ECDC427D0136B242E7
:10353000E5DCF0BC70477047980004602DE9F04F5F
:103540008146A5B0049160220F460CA8002116F018
:103550006EF94FF4C0620021864816F068F999F8B8
:103560001480B8F1000F21D000230125D9F80060A4
:103570007C7F9C4217DCBA7F9A4214DBF25C02F03B
:10358000010E4FEA4E0171441F2A0DF1900E05FA0B
:1035900002FC0EEB011100F3578251F85C2C42EA59
:1035A0000C0241F85C2C01334345E2D199F81550E7
:1035B000002D00F0598200210124D9F80420A81818
:1035C00012F8013B04FA03F3904241EA0301F7D1F8
:1035D000C1F3130200234FF0405C9DF83E00049EAF
:1035E0009DF86E707668140C20F00F0092B22043A4
:1035F000ADF83C20ADF86C209DF8312027F00F0786
:103600008DF83E0030783C436FF3C3028DF86E4076
:103610008DF85F00BDF838408DF88F008DF83120AF
:103620009DF83A009DF85E2004F0030420F03F006E
:1036300022F01F029DF86170ADF838408DF83A0015
:10364000BDF868409DF86A008DF85E209DF88E20D8
:1036500063F3C30722F01F0204F0030420F03F00CD
:103660008DF88E200696ADF85C308DF83B30ADF8C5
:103670008C308DF86B308DF86170ADF868408DF846
:103680006A00049E3269CCF84810002D00F0CF810A
:103690004FF0010B4746CDE901329A46354B039373
:1036A00041F480130B932AF003031A464FF0000EE7
:1036B000D9F804C007931CF80A3004320BFA03F857
:1036C000C8F31308C8F30D039B000993CDF81480C9
:1036D0004FEA9833039CDDF8188008920A93264637
:1036E0004FEA4E0524AB754403EB0515603D0FCD45
:1036F0000FC60FCD0FC695E80F0086E80F00019AA0
:10370000238862F309032380002F00F08E81029941
:103710006FF000420B460F4413F8011B8A42A8BF0A
:103720000A469F42F8D1D2B2E27298F80630002BD6
:1037300040F05B812368059A62F31F33236094F89D
:103740002E3098F8052023F01F0399F8151084F8FF
:103750002E304FF00003501EA385062800F287810B
:10376000DFE810F01C010901E300E100DF00DD00EB
:103770000A0000BF980004600B1F534540F372819C
:103780000CEB0A031D7994F82E300BFA05F5C5F3FE
:10379000044023F01F030343A58584F82E30C5F3AE
:1037A0001405BAF1030F12DD0CEB0A0313F8040C35
:1037B00094F82E300BFA00F00543C5F3044023F0D3
:1037C0001F030343A58584F82E30C5F31405CB1ED3
:1037D000534511DD0CEB0A03D87894F82E300BFA20
:1037E00000F00543C5F3044023F01F030343A58500
:1037F00084F82E30C5F31405BAF1020F12DD0CEB7C
:103800000A0313F8030C94F82E300BFA00F005436A
:10381000C5F3044023F01F030343A58584F82E302D
:10382000C5F314058B1E534511DD0CEB0A03987884
:1038300094F82E300BFA00F00543C5F3044023F052
:103840001F030343A58584F82E30C5F31405BAF190
:10385000010F08DD0CEB0A0313F8023C0BFA03F32B
:103860001D43C5F31405236894F82E0045EA13356B
:1038700045F48015C5F3140320F01F00013940EA18
:1038800013405145A58584F82E000FDD0CEB0A038B
:103890005B78C1B20BFA03F32B43C3F3140321F09B
:1038A0001F0141EA1341A38584F82E10BAF1000FDD
:1038B00007D0D4441CF8011C0BFA01F10B43C3F3ED
:1038C000140383F4FF130B9883F4FF5394F82E1022
:1038D00083F01F030340C3F3044021F01F010143A1
:1038E000012AA38584F82E100BD0DB43E268A17B6C
:1038F000C2F31302134021F00F0242EA1342A381E4
:10390000A2733034BEF1000F57D1049BD9F804C024
:10391000D3F8048099F814704FF0010EDFE600250B
:1039200055E700257EE700259DE70139514540F325
:1039300081800CEB0A035B7894F82E100BFA03F3EA
:10394000C3F3044221F01F011143A385C3F3140202
:1039500084F82E10BAF1000F70D0D4441CF8013C4A
:103960000BFA03F313430B9AC3F314031340C3F38B
:103970001401DB4308E0404A236882EA13330B9AC0
:103980001340C3F31401DB4394F82E20A18522F0E9
:103990001F0242EA114284F82E20A7E74FF00002EE
:1039A00094F82E30A28523F01F0343F0100384F80F
:1039B0002E303034BEF1000FA7D0019A99F815309F
:1039C0002232C2F309020192039A0AF1010A60321B
:1039D0000392029A534502F12202029227DD049BD0
:1039E00099F814705B6806935DE6079B0CEB030186
:1039F000089B0CEB030511F8013B20680BFA03F35D
:103A0000226843EA103363F31F328D422260F2D101
:103A10002389099A03F0030313432381A37A0A9AA3
:103A200023F03F031343A37289E6FF227CE625B00F
:103A3000BDE8F08F0022BAF1000F8ED10B9B13402E
:103A4000C3F31401DB439FE711F8580C203A844676
:103A500005FA02F2C0F30100024362F3010C01F81F
:103A600058CCA0E500259CE62A462946B2E54FF051
:103A7000FF33002188E700BFFFFF0F00002900F09F
:103A80009F802DE9F04FD1F80120ADF5117D0CCAD2
:103A900093F8009093F801B01278884609EB0B0771
:103AA00008A9064605929D7893F804A0DC78FFF7F4
:103AB0001FFD444BF9B2481C83F8290009F1010CA1
:103AC00009F1FF3083F8221083F824C083F8250021
:103AD000059A002A6FD1A9F10A0983F827904FF0BF
:103AE0000009384B4A469E460AF03F0C05F01F007D
:103AF00004F00F0183F8289002F114030EEB430346
:103B00009C7801326CF305049C705C88112A60F388
:103B10008A14C4F3072561F3C6055C80DD70EBD120
:103B20004FF04050002280F8A720347DBCB14FF008
:103B3000010C3168234D013911F8013F1C2BEA5467
:103B400002F1010209DD90F8A7E01D3B0CFA03F336
:103B500043EA0E03DBB280F8A730A242ECD1D8F8DA
:103B600001103046FFF7EAFC08A93046FFF77CFC5D
:103B7000D8F8013030465968DA68C979124BFFF736
:103B8000FDF949F640437F00012400200422033759
:103B900093FBF7F70D490290CDE90024039107ABA1
:103BA0002246214664200797FFF73EF920460DF58F
:103BB000117DBDE8F08F0BF1010B83F827B08EE784
:103BC0000846704700000460980004608CA401005F
:103BD000F0B50C4699B0602200210746684615F002
:103BE00026FE30220021544815F021FE4FF40870C3
:103BF0009DF80130626843F008038DF80130BDF88C
:103C00000010537960F30901013BADF80010032B5C
:103C100003D8DFE803F07F6D02024FF0FF344FF06E
:103C2000405100209DF82E30ADF82C4043F01F038A
:103C30008DF82E30C1F830014FF0013300216D4670
:103C40001278CDF813308DF82F20CDF81730CDF83D
:103C50001B308DF81F30CDF80F308DF80B100CACE9
:103C60000FCD0FC40FCD0FC495E80F0084E80F00EF
:103C70003D7D3DB33C680126254407E052F85C3C9D
:103C8000A54243EA070342F85C3C1BD014F8013B11
:103C900003F00100420002441F2B18A806FA03F7A4
:103CA00000EB0212EADD12F8581C203B084606FA27
:103CB00003F3C1F301010B4363F30100A54202F8D2
:103CC000580CE3D16C461C4F0FCC0FC70FCC0FC75D
:103CD00094E80F0087E80F00184E0CAD0FCD0FC60B
:103CE0000FCD0FC695E80F0086E80F0019B0F0BDA4
:103CF0004FF0FF344FF0405100209DF82E30ADF8CA
:103D00002C4023F01F0343F00F038DF82E30C1F831
:103D1000300191E700204FF040519DF82E30ADF872
:103D20002C0023F01F03064843F010038DF82E30BB
:103D3000C1F8300180E700BF98060460C80604603F
:103D4000FFFF0F00002900F086802DE9F84FD1F821
:103D50000160424AD6E900531C7893F8018095F837
:103D600000A004EB0805EDB204F1010993F802C0CC
:103D700093F804E0DF7805F1010B5FFA89F9631E1F
:103D800082F829B082F8225082F8253082F82490F7
:103D9000BAF1000F5AD10A3C82F8274000242F4B79
:103DA000224698460EF03F0E0CF01F0C07F00F074E
:103DB00083F8284002F1140308EB43039C78013296
:103DC0006EF305049C705C88112A6CF38A14C4F3AA
:103DD000072567F3C6055C80DD70EBD14FF04055D9
:103DE00000221F4C1F4B85F8A72084F82F9083F8E2
:103DF0002F90077DCFB14FF0010E0468DFF85CC053
:103E0000013C14F8013F1C2B0CF8032002F10102C5
:103E100009DD95F8A7801D3B0EFA03F343EA08037A
:103E2000DBB285F8A730BA42EBD10D4604463146E5
:103E3000FFF7CEFED5F8013020465968DA68C97917
:103E4000074BFFF705F90120BDE8F88F08F10108DD
:103E500082F82780A2E70846704700BF4C00046044
:103E600098060460C8060460F0B400254FF0405383
:103E70000326D0F8011001248A684D7417780420B5
:103E800083F82C7157784FF4C07C83F82D719779A3
:103E900083F82A71177A83F82B71977883F82E713B
:103EA000D27883F82F21D1E90021177883F8257182
:103EB00083F88E60C9780F27491B18BF012183F84A
:103EC000841083F8814083F8805083F8AE0083F833
:103ED000AF00557893F8891085EA040666F305115A
:103EE000022683F8891093F8A11065F3041183F872
:103EF000A11083F88D0083F8B04083F8C570A3F853
:103F0000C8C083F8CC60507A517983F8000190786A
:103F100083F80501D07883F80A0183F80D1111792F
:103F200083F81011117A83F8DA10D27983F8A0207F
:103F3000F0BC00F0FFBD00BF012138B54FF0405389
:103F4000D0F80140084693F8415100F09FFB637C94
:103F5000074903EB0313EDB200EBC30001EB05418E
:103F6000882215F059FC637C0133637438BD00BFAF
:103F700080080160D0F801305B689B794BB3F0B4E6
:103F80004FF0C04784B0DFF84CC004AE002568464F
:103F90006A463B46002153F82540883342F8044BDB
:103FA00096422144F7D13C4650F8043BA1EB430331
:103FB0005B10904244F8253004F18804F4D10135B7
:103FC000222DE4D107F508776745DFD104B0F0BCB6
:103FD0007047704780080060F0B5D0F8016085B088
:103FE00073689B7923B34FF0C04CDFF8D8E004AF7F
:103FF000002568466A466346002153F82540883309
:1040000042F8044B97422144F7D1644650F8043BF0
:10401000A1EB43035B10904244F8253004F188047F
:10402000F4D10135222DE4D10CF5087CF445DFD123
:1040300096F82170717F1FBB3A46214C4FF0220C3D
:10404000A4F505050023994209DCB07F984206DB00
:10405000F07FB84203DC96F82000B84203DA44F857
:10406000232045F823200133222BECD1BCF1010C95
:10407000E8D10137102F04F18804DFD105B0F0BD7D
:1040800000273A460E480023A0F50505994209DCB1
:10409000B47F9C4206DBF47FBC4203DC96F82040F0
:1040A000BC4203DA40F8232045F823200133222BB9
:1040B000ECD10137102F00F18800E4D105B0F0BD3C
:1040C00000008560800800604FF04053F0B5032584
:1040D0000021D0F80100012682680424177883F8B3
:1040E000E07092F801C00F2783F8E1C092F802C097
:1040F00083F8E2C092F803C083F8E3C092F806C0E8
:1041000083F8E6C0127A83F8E720426883F88E507D
:10411000D278521A18BF012283F8842083F8816074
:1041200083F8801083F8AE4083F8AF40026893F8BC
:10413000891092F801C08CEA060E6EF3051183F81F
:10414000891093F8A1106CF3041183F8A11083F87F
:104150008D4083F8B06083F8C57083F88750C17FC5
:1041600001EB4101A940A3F8C81090F820101029D4
:1041700028BF1021B140C9B283F8CC10517A83F81E
:104180000011917883F80511D17883F80A1111791B
:1041900083F81011117A83F8DA10D27983F8A0200D
:1041A000BDE8F04000F0C6BC4FF04053F0B4032629
:1041B0004FF0000CD0F8010001258268017F1478CF
:1041C00001EB410183F8E040547883F8E1409778AF
:1041D0008C0083F8E270D178042783F8E31091799A
:1041E00083F8E610127A83F8E720426883F88E603D
:1041F000D278B2EB0C0218BF012283F8842083F836
:10420000815083F880C0026893F88910507880EA62
:10421000050C6CF305114FF00F0C83F8891093F81F
:10422000A11060F3041183F8A11083F88D7083F856
:10423000B05083F8C5C083F88760A3F8C84083F8FE
:10424000CC50517A83F80011917883F80511D17818
:1042500083F80A11117983F81011117A83F8DA10B2
:10426000D27983F8A020F0BC704700BF2DE9F04F51
:1042700093B004AF07F13805654C664E45F8300D34
:1042800007F1240807F1140A94E80F008AE80F00E8
:1042900007F1600350464146CAE902567B63FBF7CB
:1042A000EFFF94E80F005C4C88E80F00404607F1F0
:1042B0003401C8E90254FBF7E3FF012000F0A8FC39
:1042C000002800F09E800021E9460A46BB680546AA
:1042D000D0F801005E7D1C7D0368D0F804C004FBAB
:1042E00006FBC7E903465C789CF802607C604B4C97
:1042F000597002F1140304EB43035988013241F46D
:10430000F861112A5980F4D16A460BF10703DB08E2
:10431000A2EBC3039D469CF8013004AC01695A46E8
:1043200020463B6015F078FA3B68BBF1000F09D0DE
:10433000224604EB0B0012F8011B0431824202F802
:10434000011CF8D148F001024AF00101CDE9002139
:1043500001205A461946234602F02EFED7E90321D2
:104360004FF0000A0123DFF8B8800093CDE901AADD
:10437000CDF80C8023466420FEF756FDD7F810B028
:10438000D34542DDD646D7E9020ABAF1000F0EDD69
:104390000023027DD5F801100EFB0232496914F8A2
:1043A00002C0C95C013361445345A154F1D10EF1FF
:1043B000010EDE45E9D12146FFF756F8D7E9032182
:1043C0004FF0000A012023460090CDE901AA6420A5
:1043D000CDF80C80FEF728FD5246104806F01F0667
:1043E00002F1140300EB43035988013266F38A118A
:1043F000112A5980F4D1D5F801303A791B685A70E6
:10440000CD463C37BD46BDE8F08FB868D3E700BF66
:10441000009A01003D2F0000BD3400000000046040
:10442000A0A301002DE9F04FADF5137D04AF786036
:1044300001200C4600F0ECFB0026D0F80130D4F847
:1044400001201B6854685A78B8605E70012191465B
:1044500007F118004FF4087294F801A015F0E7F97D
:10446000ADF6880D0DF1100B584631464FF4086239
:1044700015F0DDF9BAF1010F53DD0124A046384DE6
:10448000FE60ABF1040B374E304611222146303628
:1044900015F0CDF9AE42F7D101220426324B07F1D7
:1044A00014000393FB681146CDE90183009603468F
:1044B00064207C61FEF7B8FC00F008FC00F038FCDA
:1044C000FB682A4ACDE9018303924FF0C0432222C0
:1044D000102100967220FEF7A7FC59464FF0C0430A
:1044E000DFF894C007F11802186851F8046F04331C
:1044F0008642BCBF14700860634502F10102F3D12B
:104500001B4BCDF800800393FB680134CDE90133E8
:10451000222207F1180310216420FEF785FCA24532
:10452000B1D1786807F11801FEF79EFF0124002140
:10453000BB681048D3F801301A6807F1180382F8F5
:104540000190CDE9011103902222009410216420F2
:10455000FEF76AFC07F50F77BD46BDE8F08F00BF98
:10456000A7060460A7000460ACA3010030C50100E9
:10457000A0A30100BCA301008008006030B585B095
:1045800000F0D6FB0021084600F080F80025044624
:1045900004210120064ACDE901050091039223463A
:1045A000222210217220FEF73FFC204605B030BDCC
:1045B00030C50100012170B50446084600F066F8D8
:1045C00000210546012000F061F8D4F801202B1FDE
:1045D000147C011F05F1840653F8042F02FB04F23A
:1045E000B3424FEAE21241F8042FF5D100F1840101
:1045F00005F5867053F8042F02FB04F298424FEA47
:10460000E21241F8042FF5D170BD00BF704700BF22
:104610004FF0405393F84121002082F0010283F8CB
:10462000412193F8432182F0010283F8432170472E
:104630004FF0405310B593F82430CBB172B60E4A08
:1046400014689CB90D490E4B08681160027803EBA1
:10465000C2035B68984701230A4A1375BFF34F8F63
:104660004FF0405208490C721370937062B610BD3F
:104670000BF068FCE2E700BF6C10002094100020F3
:10468000D8040020000010501024002001290CD074
:1046900007D3022903D1074B53F8200070470020AD
:1046A0007047054B53F820007047044B53F8200027
:1046B000704700BFBC100020D4100020EC10002078
:1046C0004FF0C04370B5584C584E594D5949626827
:1046D0002360336029601AB15749201D07F008FB99
:1046E00073681BB15549564807F002FB6B681BB154
:1046F0005449554807F0FCFA4F4A4FF48871534823
:1047000007F086FA4D4A4FF488714D4807F080FA59
:104710004C4A4FF488714C4807F07AFAA3681BB1F1
:104720004B494C4807F0E4FAB3681BB14A494B487F
:1047300007F0DEFAAB681BB149494A4807F0D8FADE
:10474000434A8821434807F063FA434A8821434893
:1047500007F05EFA424A8821424807F059FAE368B6
:104760001BB14149414807F0C3FAF3681BB1404906
:10477000404807F0BDFAEB681BB13F493F4807F0DE
:10478000B7FA394A5021394807F042FA384A5021DD
:10479000384807F03DFA384A5021384807F038FACF
:1047A00023691BB13649374807F0A2FA33691BB1B8
:1047B0003549364807F09CFA2B691BB13449354816
:1047C00007F096FA2E4A88212E4807F021FA2E4A41
:1047D00088212E4807F01CFA2D4A88212D4807F021
:1047E00017FA63691BB12C492C4807F081FA7369E9
:1047F0001BB12B492B4807F07BFA6B691BB12A4987
:104800002A4807F075FA244A5021244807F000FA94
:10481000234A5021234807F0FBF9BDE87040224AA3
:104820005021224807F0F4B9D4100020EC100020E9
:10483000BC10002000008560F0A4010004A5010068
:10484000F010002020A50100C0100020D81000208A
:104850003CA50100DC10002058A50100F410002048
:1048600078A50100C410002098A50100E0100020E8
:10487000B4A50100F8100020D4A50100C810002044
:10488000F4A50100E410002010A60100FC10002097
:1048900030A60100CC10002050A60100E810002036
:1048A0006CA60100001100208CA60100D010002091
:1048B0002DE9F047114C124E124DDFF84CA0DFF8F5
:1048C0004C90DFF84C8004F1140754F8043F1BB1FE
:1048D0005146204607F00CFA55F8043F1BB14946F3
:1048E000284607F005FA56F8043F1BB1414630460A
:1048F00007F0FEF9BC42E8D1BDE8F087D4100020F3
:10490000BC100020EC100020B0A40100C0A40100E5
:10491000D8A4010000487047000084600048704738
:1049200000000230F8B516461D4604460F46FFF754
:10493000A5F808B10F4B1F6031462046FFF702FA79
:1049400008B10C4B5E60069A2946204601F0C4FC73
:1049500018B1084B069AC3E90225DDE90712204683
:1049600001F0D4FC20B1034B089A1A61079A5A61EE
:104970000120F8BD741000202DE9F04F8DB004AF78
:104980000AF0D2FE02240546B860982200215F4852
:1049900014F04DFF5E4B2A7D2968D3F80100009486
:1049A0005C4B00F0C9FC5C4B6A7D6968D3F8010080
:1049B0005A4B009400F0C0FC242200215848C7F84C
:1049C00004D014F034FF0AF0AFFE437D544D1A4674
:1049D0007B612B46073202F4FC72ADEB020D42689C
:1049E000067D3A61046804AAFA60A5F124011A7FE1
:1049F000093B42F00A0283F825208B42F7D17B69FC
:104A0000002B77D03869F96802460139184412F84A
:104A1000013BC3F12103824201F8013FF7D100F0CD
:104A200083FC814600F084FC8246002E6BD0A319E3
:104A30004FF0010B984607F11806C7F800A014F8CC
:104A400001AB08224FEA4A01304614F0C1FE19F9C1
:104A50000A30B96903EBC3032B44FA69585C0BFABB
:104A600002F20243A0455A54E9D17B69D7F800A06D
:104A700013B34FF0010B7B69FC6823447B613B69F6
:104A800003F1FF3814F8011B18F8019F49000822B0
:104A9000304614F09DFE1AF90930B969023303EB70
:104AA000C303FA692B44585C01320BFA02F2024349
:104AB0005A547B69A342E5D1D7F804D00EF01AFD11
:104AC0000EF062FD0EF0D0FCFDF778FEFDF7AAFEB9
:104AD0001149144A144B0091B8681449CDE90132C8
:104AE0000B4B134AFFF71EFFFFF7EAFD2437BD46C5
:104AF000BDE8F08F00F018FC814600F019FC8246FA
:104B0000002ED9D093E707F11806B2E70000046041
:104B100040040020C4310020700400202C29002013
:104B2000F42900206404002018020020840A0020D8
:104B3000D00A002008B50BF041F9054B1B789842CC
:104B400004D01846BDE808400BF0F0B808BD00BF1F
:104B5000D404002010B50BF031F904460BF0F8F83E
:104B6000844203D0BDE810400BF0E0B810BD00BF98
:104B70002DE9F04100248046104B0E4620222146AC
:104B80000F481C6014F053FEA04514DD2146013E81
:104B90000C4D0B4F06EB080C16F8014F0A4B53F85F
:104BA000042F1078A04204BF47F821200131AB4206
:104BB000F5D16645F0D1BDE8F08100BF6C10002052
:104BC00094100020901000207010002070B50E4D41
:104BD0002C68B4B1206803780A2B12D80B4E56F813
:104BE00033309847636863B12B682268191D2960C8
:104BF0003AB15868037806EBC306736898470120FA
:104C000070BD0020286070BD6C100020D80400200A
:104C1000074B10B403F1200453F8042F117881429C
:104C200002D0A342F8D10022104610BC704700BF4A
:104C300070100020044B11B143F820107047034A54
:104C400043F82020704700BFA80400200D46000054
:104C500070B5094C094E04F1200554F8040F03788F
:104C60005A1E092A02D856F823309847AC42F4D18C
:104C7000BDE87040FFF76EBF90100020A804002030
:104C800010B572B60C4A1468A4B90C490C4B0868EC
:104C90001160027803EBC2035B6898470422094B5A
:104CA0001A75BFF34F8F4FF04053012206490C7223
:104CB0001A709A7062B610BD6C100020941000201B
:104CC000D80400200000105010240020FFF7B0BCD2
:104CD000FFF7D6BF002208B5054B1A720BF0CEFCC9
:104CE000044B054A1A60BDE80840FFF7A1BC00BFAD
:104CF00010240020B41000203146000008B50BF04D
:104D0000DDFC002303480449044A03600B60136080
:104D100008BD00BFB4100020B8100020041100200E
:104D2000024B1868003018BF012070476C1000203B
:104D300008B5084908200AF0FBFEFFF789FF0BF0D1
:104D4000BDFC002304480549054A03600B6013605D
:104D500008BD00BF11460000B4100020B8100020AC
:104D60000411002038B572B60BF0A8FC00200E49E3
:104D70000E4A0F4B08601060186062B60D4B1C683D
:104D800084B10D4BA3F1200553F804292168914209
:104D900018BF5860AB42F7D1BDE83840074908203A
:104DA0000AF0C6BE38BD00BFB4100020B810002005
:104DB000041100206C100020B010002011460000EB
:104DC00008B5044908200AF0B3FEBDE80840FFF723
:104DD0003FBF00BF1146000008B50449082014F089
:104DE0000BFEBDE80840FFF733BF00BF11460000CF
:104DF000082270B5304C314D23682A60B3B1186871
:104E00000278022A31D05A6882B1FFF7DFFE00280B
:104E10003FD001232A4A1375BFF34F8F4FF0405202
:104E20000020284908721370937012E001260020B8
:104E3000244A23491672244A087512680AB1904719
:104E400023681868214B027853F8323098470023C2
:104E5000236010221E4B2A60D3F8002112071CD4B5
:104E60004FF0405300225A7070BDD0F80120567C9C
:104E7000002EC8D1154B1B6998470123104A1375A2
:104E8000BFF34F8F4FF040520E490E721370937064
:104E9000DFE701220B4B1A72DBE7002208240D48E2
:104EA0000D49C3F8804102704FF04053C1F84021D2
:104EB00000225A7070BD00BF6C1000202009002035
:104EC000000010501024002030240020D8040020BE
:104ED00000E100E01C09002000000250F0B5012AAA
:104EE00083B0164605460C461F462DDC0146684633
:104EF00014F06EFC36B3009B3F2B1D46A8BF3F2528
:104F0000019A002B134405F03F05B8BF00253F2B45
:104F10001A46A8BF3F22002B4FF0000102F03F03CA
:104F2000B8BF002304F1100207EB420C09B30A19C1
:104F3000103207EB4202907965F305009071013160
:104F4000B142F3DB03B0F0BD104606F02BFE044186
:104F500006FB04F40F2C294606DD0122684614F0F6
:104F600037FC0126009BC7E73246684614F030FC48
:104F7000C1E79CF8062063F305028CF80620DEE703
:104F8000F0B5012A83B0154604460E461F462DDCB7
:104F90000146684614F01CFC009B2DB33F2B1C46B9
:104FA000A8BF3F24019A002B134404F03F04B8BF6C
:104FB00000243F2B1A46A8BF3F22002B4FF00001D0
:104FC00002F03F03B8BF002306F1100207EB420CCA
:104FD000F1B18A19103207EB4202907964F30500AF
:104FE000907101318D42F3D103B0F0BD104606F04F
:104FF000D9FDF30744BF06416E4321462A46684661
:1050000054BF06F1FF36013614F0E2FB009BC5E702
:105010009CF8062063F305028CF80620E1E700BF48
:1050200030B5DCF8103085B064469847FFF780FE55
:10503000D4E9023200200121042502900448CDE980
:10504000005103907220FDF7EFFEA06805B030BD5F
:10505000C8A6010030B5DCF8103085B0644698472A
:10506000FFF766FED4E902320020012104250290F8
:105070000448CDE9005103907220FDF7D5FEA068E9
:1050800005B030BDC8A6010030B5DCF80C3085B0E5
:10509000644600259847FFF74BFE01210420064A8D
:1050A000A36800900392CDE9011514227220FDF748
:1050B000BBFEA06805B030BDC8A6010030B5DCF865
:1050C0000C3085B0644600259847FFF731FE01217A
:1050D0000420064AA36800900392CDE9011514222A
:1050E0007220FDF7A1FEA06805B030BDC8A6010082
:1050F0002DE9F04F0D46CC1D890087B024F0070440
:105100000A3121F0070106AFADEB040D0DF11808CF
:10511000ADEB010D9B4606AEBC6A9DB10023013884
:1051200000EB050E10F8011F1AB112F801C008F8C3
:1051300003C01CB154F8211046F82310704503F148
:105140000103EFD1EAB14FF0010A4FF000092B4BF8
:10515000514603932A464346CDE90199CDF800A074
:105160006420FDF761FEFB6AFA6AD3F8013011781A
:10517000D3E9002312780A299B79524414D00629D6
:105180002CD06CB14FF0000C012104241C48334694
:1051900003902A46CDE9011C00946420FDF744FEEB
:1051A0000437BD46BDE8F08F009340F64A30CDE9A4
:1051B000036BCDE9015840F235234FF4487102F0FA
:1051C0007FF804200F4A00900392CDE901995B46D5
:1051D00051462A466420FDF727FED2E7009340F6A9
:1051E0004A30CDE9036BCDE9015882234FF4487171
:1051F00002F066F80420044AE5E700BF44A7010076
:1052000060A701004CA7010058A701002DE9F04F4D
:105210000D46CC1D890087B024F007040A3121F027
:10522000070106AFADEB040D0DF11808002DADEB35
:10523000010D9B4606AEBC6A13DD0023013800EB6E
:10524000050E10F8011F1AB112F801C008F803C0CA
:105250001CB154F8211046F82310704503F10103E6
:10526000EFD1EAB14FF0010A4FF000092A4B514645
:1052700003932A464346CDE90199CDF800A0642066
:10528000FDF7D2FDFB6AFA6AD3F801301178D3E951
:105290000023127809299B79524414D005292CD077
:1052A0006CB14FF0000C012104241C4833460390DC
:1052B0002A46CDE9011C00946420FDF7B5FD0437B2
:1052C000BD46BDE8F08F009340F64A30CDE9036B50
:1052D000CDE9015840F235234FF4487101F0F0FF59
:1052E00004200F4A00900392CDE901995B46514694
:1052F0002A466420FDF798FDD2E7009340F64A3035
:10530000CDE9036BCDE9015882234FF4487101F0D8
:10531000D7FF0420034AE5E71CA7010038A70100D6
:1053200024A7010030A7010000487047C4310020C5
:10533000004870472C2900202DE9F04F85B04068C7
:1053400004AFD7F828904578D01D20F0070009FB5E
:1053500005F5ADEB000D0DF1100A0E46504600218B
:1053600090461C4614F063FAA94540DB4FF0000B51
:1053700008F1FF3922224FF0FF31204614F057FA8E
:1053800033784FFA8BF0B8F1010FE0542CDD4FF079
:10539000000E6FEA060C711C11F8012BA356B3F135
:1053A000FF3F05D1431CAB42ACBF00235BB2A3540B
:1053B000984219D092FBF5F005FB1020012814BF8C
:1053C00001204FF0FF30204482569A420CD00CEB63
:1053D00001029145A1EB06027BD0904501DD184604
:1053E000DAE7BEF1000F40D1BBF1000F3AD0002246
:1053F0003B496420FDF764FDB8F1000F5CDD013E20
:10540000B14606EB080119F8013F93FBF5F205FBE5
:1054100012324945E254F6D101210022314BCDE947
:10542000011203930091234642466420FDF7FCFCE1
:105430000AF1FF3316F8012FA256B14503F8012FE8
:10544000F8D10121002428485346039042466420A5
:10545000CDE901140091FDF7E7FC20460437BD4675
:10546000BDE8F08F4FF0010B84E7012100221D4BB6
:10547000CDE9011200910393424623466420013E88
:10548000FDF7D2FC06EB08010AF1FF3316F8012FF5
:10549000A256B14203F8012FF8D10124002112488D
:1054A000CDE90141039053466420424600942146D1
:1054B000FDF7BAFC2046D1E701210020094ACDE9D9
:1054C000011003922346009142466420FDF7ACFC94
:1054D000B7E79045C9DD4FF0010E18465CE700BF05
:1054E000E4A6010008A70100D4A601002DE9F047B9
:1054F000D2F8017006467A680D4652789846012A1D
:1055000019D9002815DD00244FF04C094D1E01E08B
:105510007B685A78510094FBF1F301FB134315F8B3
:10552000010F611009FB03830134FFF7D7FCA6428A
:10553000EED1BDE8F0870028FBDD00244FF04C0AD7
:10554000DFF8249019F904306110002B06DB7A682B
:105550000AFB03835278285DFFF7C0FC0134A642A2
:10556000F0D1BDE8F08700BFC431002010B564461B
:1055700084B0DCF80420084BFFF7B8FF01210020BD
:105580002368E268054CCDE9010000910394722084
:10559000FDF74AFC04B010BD90070460BCA60100F2
:1055A00010B5644684B0DCF80420084BFFF79EFF7A
:1055B000012100202368E268054CCDE9010000913B
:1055C00003947220FDF730FC04B010BDC0080460E5
:1055D000BCA601002DE9F047D2F801601F467268B1
:1055E0005278012A1ED900281ADD4D1E21244FF0C1
:1055F0004C0805EB000901E073685A78510094FBF0
:10560000F1F301FB134315F8010F04EBD47108FB10
:1056100003734910FFF7B4FCA94504F1FF34EBD143
:10562000BDE8F0870028FBDD0D464FF04C0A0D4C1D
:1056300001EB000904F1220814F9013BA8EB040175
:1056400001EBD171002B4FEA610106DB72680AFBA6
:10565000037352782878FFF793FC01354D45EBD161
:10566000BDE8F0872C29002010B5DCF8042084B0B8
:10567000084B6446FFF7AEFF01210022064823686D
:10568000CDE901220390009114227220FDF7CCFB9A
:1056900004B010BDF8060460BCA6010010B5DCF82B
:1056A000042084B0084B6446FFF794FF01210022D8
:1056B00006482368CDE9012203900091142272204C
:1056C000FDF7B2FB04B010BD28080460BCA60100C1
:1056D000F0B403268C68012527784FF0060C80F87B
:1056E000E8706778002B80F8E970A778B8BF0333BB
:1056F00080F8EA70E778C3F38F0380F8EB70A7793E
:10570000D2B280F8EE70247A072780F8EF4080F854
:105710008E60002690F88940096844F0300480F8D3
:10572000894090F8A1406FF3041480F8A1400C78F0
:1057300080F8A94080F8985090F88B406FF30004EF
:1057400080F88B4080F88D7080F8B05080F8C5608C
:1057500080F8815080F8805080F8AEC080F8AF703B
:1057600080F884604C7A80F89F408C7A80F89E4064
:1057700080F89C60A0F8CA3080F8CD204B7BF0BC4C
:1057800080F800318B7880F80531CB7880F80A31C9
:105790000B7980F810310B7B80F8DA3090F8A33069
:1057A000CA7962F3061380F8A33090F8A3300A7A1E
:1057B00062F3020380F8A330CB7A80F8A030704700
:1057C000D0F8011008B54A684FF4F26352784FF0F0
:1057D00040505200FFF77CFFBDE80840FFF7BAB920
:1057E000D0F8011008B54A684FF40C6352784FF0B6
:1057F00040505200FFF76CFFBDE80840FFF7AAB920
:1058000049F64043014411440331490030B50122B7
:1058100093FBF1F10025042487B0074806AB43F859
:10582000041D0390CDE90125114600946420FDF785
:10583000FBFA07B030BD00BFACA601002DE9F04F68
:105840004FF04C09984609FB03F909F1070383B0AF
:1058500023F0070300AFADEB030D78603A600C4610
:1058600068464A46002113F0E2FFB8F1000FEA460D
:1058700071DD6B465C200DEB09015A78187002F05F
:10588000EC0242F002025A704C339942F5D13A6868
:1058900014F0FF011369566964D053EA06020CBF85
:1058A0004FF0010E4FF0000E00224FF0010C05E00A
:1058B000BEF1000F10D101328A421FD0C2F1200583
:1058C00006FA05F523FA02F0A2F12004284326FA8D
:1058D00004F42043C007EBD54FF04C0B7868234C01
:1058E000805C24561F280CFA00F50BFB04A425DC71
:1058F0006069013205438A426561DFD13B68B8F1D6
:10590000000F5B6858780FDD00234C2555240228D2
:1059100007D105FB03A2D17C547421F001019474DA
:10592000D17401339845F2D14A465146386B13F091
:1059300073FF386B0C37BD46BDE8F08F257E2038ED
:10594000AB460CFA00F0C5F30105054365F3010B06
:1059500084F818B0AFE73A6814F0FF01136956698C
:105960009BD1E1E73B685B685878CDE7C431002004
:105970002DE9F04F85B01546D0F801800A7DD8F8A2
:10598000044002AF6678086803FB06F603EBC30A1F
:105990001146334600954246FFF750FF0AF10703D0
:1059A000D8F8044023F00703C7F804D0ADEB030D8B
:1059B00094F805B00DF10809484652460021647874
:1059C00013F035FFBBF1020F00F0CC80BBF1040FE8
:1059D00000F0B180BBF1010F00F08380524600213E
:1059E000484613F024FF002E40F3DD802C464FF094
:1059F000000C4A460023E11812F8010B0133092B71
:105A00000872F8D10CF1010C664509F1090904F19D
:105A10004C04EEDC4FF0000E2846F146D8F8048026
:105A2000D7F804D098F8064004F01F0404F0030CE3
:105A30004FEA8C1CA408002101F1100300EB430382
:105A400093F806A0DA790AF03F0A22F00702013142
:105A50004AEA0C0A2243112983F806A0DA71EBD135
:105A600090F84A300EF1010E23F01F03764580F8BE
:105A7000489080F8499080F84A3000F14C00DADC18
:105A8000002398F8049098F803A098F802B05046C4
:105A900049465A469846012409EB0A0E0BEB090CBD
:105AA000AEF10A0E0CF1010C5FFA8EFE5FFA8CFC6F
:105AB00001339E4285F802A02C7185F803C085F859
:105AC000059085F806B085F807E085F81980AC7672
:105AD00005F14C05ECDCFFF793FE0C37BD46BDE845
:105AE000F08F002E5FDDCB464FF0000EDFF8E0A018
:105AF0005946DFF8D4C00023022C03D0012C03D177
:105B0000012B01DC9E4506D003EBC30208781CF88C
:105B1000022002430A700133042BEDD10CF1010C79
:105B2000E24501F10101E6D10EF1010E76450BF1DE
:105B3000090BDDD15AE7002E35DDCC4606EBC60E4B
:105B40001F4CCE4461461F4B13F8012F587AA342D5
:105B500042EA000201F8012BF6D10CF1090CF445E0
:105B6000F0D143E7002E1EDD4C46174806EBC60C6D
:105B700090F801E0837ACC444EEA030E08300EF030
:105B8000F50E2146114B13F8012F93F809A083421B
:105B900042EA0A0201F8012BF5D184F801E0093448
:105BA0006445EED122E7D8F80430D7F804D0D8788D
:105BB00019799A78FFF724FE0C37BD46BDE8F08FBF
:105BC0000E2A0020052A0020F4290020F3290020B5
:105BD000FD2900202DE9F04792B0DFF8F0C002AFB8
:105BE000DFF8ECA007F12C0407F11C0907F1080607
:105BF00005468846BA619AE80F0089E80F002146F9
:105C000007F16003C9E9026C4846FB63FAF738FB09
:105C10009AE80F00DFF8BCC084E80F00C4E9026C0A
:105C2000204607F13C01FAF72BFB0520FEF7F0FFB9
:105C3000034600210220D3F80160FB60FEF726FD39
:105C40000523AA7E07F1400101F83C3DD31D03F472
:105C5000FC73ADEB030D02AB386101207A61BB60D0
:105C6000FEF786FFBB699847FFF762F8736844F058
:105C700001045878800105F095FFB26849F00106EB
:105C80005189BB68CDE900467A6901F051FA79691A
:105C900028688B000A3323F00703ADEB030D02AD38
:105CA000D7E90343BA68CDE900342B46FFF7AEFAD3
:105CB000B8F1000F05D07A6929464046920013F0EA
:105CC000ABFD4037BD46BDE8F08700BF2150000066
:105CD000109A01006D5500002DE9F04792B0DFF8F1
:105CE000F0C002AFDFF8ECA007F12C0407F11C09AB
:105CF00007F1080605468846BA619AE80F0089E868
:105D00000F00214607F16003C9E9026C4846FB63B6
:105D1000FAF7B6FA9AE80F00DFF8BCC084E80F0083
:105D2000C4E9026C204607F13C01FAF7A9FA092000
:105D3000FEF76EFF034600210420D3F80160FB60EC
:105D4000FEF7A4FC0923AA7E07F1400101F83C3DBF
:105D5000D31D03F4FC73ADEB030D02AB38610120DE
:105D60007A61BB60FEF704FFBB699847FEF7E0FF6E
:105D7000736844F001045878800105F013FFB2689D
:105D800049F001065189BB68CDE900467A6901F006
:105D9000CFF9796928688B000A3323F00703ADEB4C
:105DA000030D02ADD7E90343BA68CDE900342B46B1
:105DB000FFF72CFAB8F1000F05D07A692946404662
:105DC000920013F029FD4037BD46BDE8F08700BFC3
:105DD00055500000109A0100A1550000F8B59B0035
:105DE00003F10A0424F0070400AF002AADEB040D10
:105DF000EC460CDDBC69ACF10405013C224414F80E
:105E0000016F51F82660944245F8046FF7D11A46A5
:105E1000614613F001FDBD46F8BD00BF70B582B00C
:105E200009F082FC012104460220FEF72FFC00212C
:105E300006460220FEF72AFC0546A27E3146920065
:105E400013F0EAFC2168A37E227D284600912946B2
:105E5000FFF7C4FF02B070BD38B509F065FC012141
:105E600005460220FEF712FC044600210220FEF740
:105E70000DFCAA7E2146BDE83840920013F0CCBC50
:105E800070B582B009F050FC012104460420FEF7F1
:105E9000FDFB002106460420FEF7F8FB0546A27E26
:105EA0003146920013F0B8FC2168A37E227D28467B
:105EB00000912946FFF792FF02B070BD38B509F096
:105EC00033FC012105460420FEF7E0FB04460021D7
:105ED0000420FEF7DBFBAA7E2146BDE83840920095
:105EE00013F09ABCD0F8011008B54A684FF4DF638C
:105EF00052784FF040505200FFF7EAFBBDE80840EF
:105F0000FEF728BED0F8011008B54A6840F628030D
:105F100052784FF040505200FFF7DAFBBDE80840DE
:105F2000FEF718BE2DE9F04F4C261C4606FB03F683
:105F3000F31D85B023F0070300AFADEB030DF86050
:105F4000BA600D4668463246002113F070FC002C02
:105F5000E8467BDD6B4642200DEB06015A7818704F
:105F600002F0EC0242F012025A704C339942F5D121
:105F7000BB68002DD3F810E0D3F814C06EDD5EEAE4
:105F80000C030CBF4FF0010A4FF0000A2346002219
:105F900054464FF001097E609A4603E084B901320D
:105FA000954222D0C2F120000CFA00F02EFA02F342
:105FB000A2F1200103432CFA01F10B43DB07EDD5DD
:105FC0004C26FB6827499B5CC3F12100C9561F285A
:105FD00009FA00FB06FB01812ADC4B69013243EA26
:105FE0000B0B9542C1F814B0DCD15446BB68002CB1
:105FF0005B687E68587811DD00234FF04C0C6FF021
:106000005505022807D10CFB0382D17C557421F081
:1060100001019574D17401339C42F2D1324641465C
:10602000B86B13F0F9FBB86B1437BD46BDE8F08FC1
:10603000087EC3F10103834609FA03F3C0F30100AC
:10604000184360F3010B81F818B0A8E7BB68002D76
:10605000D3F810E0D3F814C091DCDFE7BB685B68CD
:106060005878C9E72C2900202DE9F04F87B01C464D
:1060700094460B46D0F8016002AFFA607268497D21
:106080005578586804FB05F5CDF800C02B4632461C
:10609000FFF748FF04EBC402D31D746823F0070325
:1060A000C7F808D0ADEB030D94F805900DF1080882
:1060B00040460021647813F0BAFBB9F1020F00F0FA
:1060C000D480B9F1040F00F0B980B9F1010F7ED08E
:1060D000002D40F3EB804FF0000CFC68424600239B
:1060E000E11812F8010B0133092B0872F8D10CF1F9
:1060F000010C654508F1090804F14C04EEDC4FF091
:10610000000ED7F80CC0F1466046D6F80480D7F8E8
:1061100008D098F8064004F01F0404F00306B60106
:10612000A408002101F1100300EB430393F806A03B
:10613000DA790AF03F0A22F0070201314AEA060A38
:106140002243112983F806A0DA71EBD190F84A3086
:106150000EF1010E23F01F03754580F8489080F87A
:10616000499080F84A3000F14C00DADC002398F8BE
:10617000049098F803A098F802B0504649465A4651
:106180009846012409EB0A0E0BEB0906AEF10A0E44
:1061900001365FFA8EFEF6B201339D428CF802A002
:1061A0008CF804408CF803608CF805908CF806B0ED
:1061B0008CF807E08CF819808CF81A400CF14C0C24
:1061C000EADCFFF71DFB1437BD46BDE8F08F002D5C
:1061D0006CDDAB1C7D60C3464FF0020EA4461D462D
:1061E000DFF8F0905846374CAEF1020A0023BCF1BC
:1061F000020F20D0BCF1010F07D1012B05DD022BCE
:106200000CBF00220122524505D003EBC3020178E6
:10621000A25C0A4302700133042BE8D10134A1458A
:1062200000F10100E2D10EF1010EAE450BF1090BB8
:10623000D8D17D684FE79E45E7D1ECE7002D35DDED
:10624000C44605EBC50E204CC64461461F4B13F8EF
:10625000012F587AA34242EA000201F8012BF6D13D
:106260000CF1090CF445F0D135E7002D1EDD444654
:10627000144805EBC50C90F801E0837AC4444EEA5B
:10628000030E08300EF0F50E2146114B13F8012FC6
:1062900093F80990834242EA090201F8012BF5D1F3
:1062A00084F801E009346445EED114E77368D7F847
:1062B00008D0D87819799A78FFF7A2FA1437BD4632
:1062C000BDE8F08FF42900200E2A0020052A0020C6
:1062D000F3290020FD29002089B182B138B5054697
:1062E0001446084602232946064AFFF741FB20468A
:1062F00029460223044AFFF7B7FE012038BD0020DB
:10630000704700BF90070460F806046089B182B14D
:1063100038B505461446084602232946064AFFF7C3
:1063200027FB204629460223044AFFF79DFE012051
:1063300038BD0020704700BFC00804602808046012
:106340002DE9F04F91B0DFF8F0A002AFDFF8ECC01C
:1063500007F1240407F114053E1D804689463A6181
:106360009AE80F0085E80F00C5E9026C284621462F
:1063700007F160037B63F9F783FF9AE80F00DFF80A
:10638000C0C084E80F00C4E9026C204607F1340164
:10639000F9F776FF0620FEF73BFC034600210320B9
:1063A000D3F801B0BB60FEF771F9062398F819A085
:1063B00007F1380101F8383D0AF1070303F4FC73D3
:1063C000ADEB030D02ABF86001207B60FEF7D0FB64
:1063D000DBF8043045F00105587844F001048001F1
:1063E00005F0E0FBDBF808207B6851894FEA8A065C
:1063F000CDE90045524600F09BFE06F10A0303F486
:10640000FF63ADEB030D02ACD7E9025398F815100A
:10641000D8F804007A68CDE900352346FEF768FE17
:10642000B9F1000F04D032462146484613F0F4F982
:106430003C37BD46BDE8F08F109A0100895000003E
:10644000695600002DE9F04F91B0DFF8F0A002AFDF
:10645000DFF8ECC007F1240407F114053E1D804667
:1064600089463A619AE80F0085E80F00C5E9026C99
:106470002846214607F160037B63F9F701FF9AE89C
:106480000F00DFF8C0C084E80F00C4E9026C2046AA
:1064900007F13401F9F7F4FE0A20FEF7B9FB0346D1
:1064A00000210520D3F801B0BB60FEF7EFF80A2306
:1064B00098F819A007F1380101F8383D0AF10703EF
:1064C00003F4FC73ADEB030D02ABF86001207B60BD
:1064D000FEF74EFBDBF8043045F00105587844F038
:1064E0000104800105F05EFBDBF808207B68518920
:1064F0004FEA8A06CDE90045524600F019FE06F142
:106500000A0303F4FF63ADEB030D02ACD7E90253BA
:1065100098F81510D8F804007A68CDE900352346BC
:10652000FEF7E6FDB9F1000F04D032462146484699
:1065300013F072F93C37BD46BDE8F08F109A0100A8
:10654000BD5000009D56000070B582B009F0ECF817
:10655000012104460320FEF799F800210646032096
:10656000FEF794F80546627E3146920013F054F926
:106570006168637E627D284600912946FFF72EFC04
:1065800002B070BD38B509F0CFF8012105460320EF
:10659000FEF77CF8044600210320FEF777F86A7EB8
:1065A0002146BDE83840920013F036B970B582B08C
:1065B00009F0BAF8012104460520FEF767F800212A
:1065C00006460520FEF762F80546627E31469200D7
:1065D00013F022F96168637E627D284600912946A6
:1065E000FFF7FCFB02B070BD38B509F09DF84FF025
:1065F0004053054693F8414101210220FEF746F839
:10660000E4B2AA7E0349240421449200BDE8384044
:1066100013F002B97009016038B509F085F84FF040
:106620004053054693F8414101210320FEF72EF81F
:106630006A7E0449E4B201EB04419200BDE83840AF
:1066400013F0EAB80809016038B509F06DF84FF0A9
:106650004053054693F8414101210420FEF716F806
:10666000E4B2AA7E0349240421449200BDE83840E4
:1066700013F0D2B87009016010B509F055F84FF069
:106680004053012193F841410520FDF7FFFF0449E4
:10669000E4B201EB04415022BDE8104013F0BCB855
:1066A0000809016038B509F03FF8012105460520C9
:1066B000FDF7ECFF044600210520FDF7E7FF6A7EA9
:1066C0002146BDE83840920013F0A6B808B5FEF7A1
:1066D0002FFBBDE8084000210220FDF7D7BF00BF17
:1066E00008B5FEF725FBBDE8084000210420FDF7B2
:1066F000CDBF00BF08B5FEF71BFBBDE80840002179
:106700000320FDF7C3BF00BF08B5FEF711FBBDE8CE
:10671000084000210520FDF7B9BF00BF704700BF4A
:10672000F0B5B5B03A9E0546F8B1421E022A01D92D
:1067300035B0F0BD6427194602A8442213F06CF866
:1067400030687168B268F36813AC0FC4306971695E
:10675000B269F369184E0FC4009702AB2A46346839
:1067600000210120A04735B0F0BD0F461446014678
:10677000C82202A813F05BF8396802A8882213F037
:106780004BF8246824AE04F1400735462068616860
:10679000A268E3681034BC4206F110060FC5F4D1BC
:1067A0000022C82104480091046802AB1146012070
:1067B000A04735B0F0BD00BF84DA0100F8B5002372
:1067C000114C1946236063603C22104813F02FF8E7
:1067D00000F0EAF94FF480620D4B0E490E4E0F4C5B
:1067E0009B68886030689A606368851C9847A368D6
:1067F0000746984739460246284613F00DF82369A4
:1068000034689847E080F8BD0C270020342A002027
:10681000CC060020401A00207406002084DA010013
:10682000F0B51E4C85B02678174686421946DDE93C
:106830000A230546DDF830C018D0A378AB4201D05A
:1068400005B0F0BDE378002BFAD0CDB94FF4086065
:1068500001210A902A460846114B1B680393039CAA
:10686000104BA44605B0BDE8F04060476678002EA6
:10687000E3D0CDF800C010321031FFF751FFDCE754
:106880006B1E022BDCD84FF488600121044C0A9067
:1068900024683B462A4608460394E2E70C2700207A
:1068A00084DA0100980004602DE9F04F5A4C85B05D
:1068B0000E9D64790295DDE90F56019614B905B075
:1068C000BDE8F08F914600240090A02288465348EE
:1068D00000219A46DFF850B112F0A9FFA646504AAF
:1068E0004E4805F1FF3CCDF80C904FE0002B0CBF5B
:1068F000012302234FF487664370009B047033F931
:106900001430029D06FB03F38BFB03761E44DB175A
:10691000C3EBE6234FF4166655F82450438038F94C
:106920001430C5F3072706FB03F38BFB03961E44C5
:10693000DB17C3EBE6238380039B33F81460EBB2D1
:10694000FF1AC5F30743C3EB1565AF42C6804FF08E
:106950004D034BDD03FB07F7BF1107814581019B09
:106960003AF814501B5D85818373009B0EF1010E74
:1069700033F91430138038F91430538001340A2C61
:10698000117100F1100002F1060235D01CF8011F50
:1069900013790029AAD1002BF0D04FF48766B2F901
:1069A0000050B2F9023006FB05F54FF4166606FBFF
:1069B00003F38BFB05678BFB03964FF003091E4423
:1069C000DB17C3EBE623019E047080F80190365D6F
:1069D0002F44ED17C5EBE725C180018141818181FD
:1069E0000EF1010E458083808673C7E703FB05F532
:1069F000AB1103814781B2E70A4B03221B680221D6
:106A00000093009C0120A446044BCDF838E005B06B
:106A1000BDE8F04F604700BF0C2700201411002094
:106A2000342A002084DA01008100088010B584B087
:106A300003F038FA0E4A4379117899420CD0437921
:106A40000C49DBB213700A6803923BB90221009330
:106A500008461A46039CA04704B010BD002302213B
:106A6000009308460122039CA04704B010BD00BF5C
:106A70000811002084DA010010B582B003F012FA88
:106A8000437F43B10023054C43771A4600931946D0
:106A900024680220A04702B010BD00BF84DA0100C4
:106AA00030B583B003F0FEF9084CC37F22789A42D8
:106AB0000AD00023C07F0649C0B202460D6820708C
:106AC000009306210220A84703B030BD0A11002020
:106AD00084DA010030B583B091B1838B028B194900
:106AE0001A44782A0B781FDDB0F924001BB3002468
:106AF000154A1460013BDBB202200B70106004E009
:106B00000846114A0F4B11601970104C23788342CC
:106B100008D000230E49024600930D68207007211B
:106B20000220A84703B030BD0020074A1060002BA8
:106B3000E0D11068E9E70123034AA0281360F8DDDB
:106B40002323D9E7101100200C1100200911002087
:106B500084DA0100002300B583B0019300F024F82B
:106B60000378054A8DF80430019BC3F300131370BA
:106B700003B05DF804FB00BF0B11002010B582B01C
:106B8000FFF77AFFFFF752FFFFF78AFFFFF7E2FFF9
:106B90000023044900930C681A4604210120A047F1
:106BA00002B010BD84DA010000487047B411002023
:106BB0004FF48060704700BFF9F764BB12F02CBE41
:106BC00012F035BE10B40124034B00221C7003499F
:106BD000642010BCFCF774B9C6240020E8A70100AB
:106BE00070B505460E46144688B010490022642050
:106BF0000794CDE90556FCF763F901210020042232
:106C00000B4BCDE9011000920393032205AB6420E6
:106C1000FCF70AF9003418BF0124064B03EB4502C8
:106C200003F81560547008B070BD00BF8CA7010058
:106C3000C0A701000C27002038B5002204460A49ED
:106C40006420FCF73DF9094A40F2F121134623F88C
:106C5000021B25686468C2F802505C601046BDE8FB
:106C600038400C2103F052B96CA70100D03000204D
:106C70000048704704A801001EF0040F0CBFEFF39A
:106C80000880EFF309808169004A104715FE000073
:106C9000684620F007018D4601B401BC8546704767
:106CA00072B61EF0040F0CBFEFF30880EFF30980FB
:106CB000004A1047396E000072B61EF0040F0CBF78
:106CC000EFF30880EFF30980004A10473D6E0000A3
:106CD00072B61EF0040F0CBFEFF30880EFF30980CB
:106CE000004A1047416E000072B61EF0040F0CBF40
:106CF000EFF30880EFF30980004A1047456E00006B
:106D0000684620F007018D4601B401BC85467047F6
:106D1000684620F007018D4601B401BC85467047E6
:106D2000684620F007018D4601B401BC85467047D6
:106D3000684620F007018D4619B507232B4CB0207B
:106D4000237308F0F3FF0021294A2A4BA1709A42CD
:106D50000CD2111D03335B1A23F0030326480B44A6
:106D600050F8041B42F8041B9A42F9D1234A244BE1
:106D70009A420CD2111D03335B1A23F003032148FE
:106D80000B4450F8041B42F8041B9A42F9D11E4AE6
:106D90001E4B9A420AD20020111D03335B1A23F0C6
:106DA00003030B4442F8040B9342FBD1EFF3088238
:106DB000174B9A4205D94FF0CD3143F8041B9A4244
:106DC000FBD84FF6FF72094B1A8708F063FE08F0F4
:106DD0006DFE1049002008F009FE044600F05EF840
:106DE000844200D0FEE70AF0BFFCFBE70000105031
:106DF0000056002080560020800000000000002087
:106E0000501000206CDB010050100020CC26002028
:106E10000C320020FCFB0100684620F007018D4683
:106E2000002201B5034B1A6009F06CFABDE801407D
:106E30008546704710E000E0704700BF704700BF14
:106E4000704700BF704700BF014B93F821007047A7
:106E5000C0FB0100014B187E704700BFC0FB010062
:106E6000014B587E704700BFC0FB0100014B987E6C
:106E7000704700BFC0FB0100014BD87E704700BFC8
:106E8000C0FB0100014B986A704700BFC0FB0100C6
:106E9000014BD86A704700BFC0FB0100014B186866
:106EA000704700BFFCFB01002DE9F04F4FEA820B59
:106EB00083B00BF10A0525F0070500AFADEB050D1A
:106EC0006D463B604B68D1F80080064614468A4602
:106ED0007B60C0475A462846002112F0A8FC0122D8
:106EE00002FA06FB1BF1FF3B17D37B6898478146EC
:106EF000BBF1000F00D0C047002CF3DDAC460021F1
:106F00005CF8043B59F8042B013113448C424CF8D3
:106F1000043CF5D11BF1FF3BE7D2002C09DD2946EB
:106F2000002251F8043B01323341944241F8043CC1
:106F3000F7D1DAF808302946204698473A68DAF857
:106F40000C302946204698470C37BD46BDE8F08FE7
:106F500001322DE9F04191FBF2F404FB121282B0F0
:106F6000DDE90A67DDE90C4512B102B0BDE8F08148
:106F70002022804600921846DDE90812012304F021
:106F800077FDB8F1000FF0DD04EB48020FFA87FE41
:106F90000FFA86FC08E0634655F8041B944203FB95
:106FA000101345F8043CE0D034F9023BB342F2DC64
:106FB000BB42B8BF7346EFE72DE9F04F1446984641
:106FC000D31D85B023F0070300AFADEB030D950093
:106FD00079608346002168463A6012F028FC05F18A
:106FE0000A0323F0070341462046EA46ADEB030DB2
:106FF000BB6B9847FB6B9847E94601462A464846D3
:1070000012F00AFC002C40F38880434608EB040190
:1070100013F8012B01328B4203F8012CF8D14146C1
:107020003868BB6B9847FB6B9847043D04384D4468
:10703000A9F10403514642464FF0FF0C4FF0010EF8
:1070400008E0AB4281F800E01C6001F1010102F1AF
:10705000010211D050F8044F53F8046FA642F0DB40
:107060001478AB4204F1FF3481F800C0147001F1D0
:10707000010102F10102EDD13B685E1E56440AF1A6
:10708000FF334FF0000A1D46C4461C46012209E0AA
:10709000786888420FDB00228CF80010B4420CF1B3
:1070A000010C0ED014F9011F0029F7D09CF8000044
:1070B00001448B45ECDDB44284F800A00CF1010CD6
:1070C000F0D182BBC7E9023241463868BB6B9847B2
:1070D000FB6B9847D7E9023284469E4605E049F8A3
:1070E0002200AC4202F1010215D015F9011F00295E
:1070F000F7D05CF8220059F822308342EFDB18F811
:107100000200AC42A0EB010108F8021085F800A0D3
:1071100002F10102E9D17346B5E7BB6B414638681D
:107120009847FB6B98471437BD46BDE8F08F00BF0A
:107130002DE9F04F012683B00138B2F100080D4669
:1071400000AF9B4606FA00F640F39880013B03EB44
:107150000800F1B203F8011F8342FBD1761000F062
:107160009D804FEA880AAAF10409C7F804A07C6B45
:10717000D7F830A059464046D047A047B8F1000F95
:1071800013DD5B465FFA86FC011F00EB090E51F828
:10719000040F1A78A842A2EB0C00D6BF6244187004
:1071A0001A70714503F10103F1D17610E2D159460D
:1071B00040463B6BD7F804A098477B6B98470AF191
:1071C0000A0323F00703ADEB030DB8F1000F0246ED
:1071D0006C465CDD043C161F20463146AAF1040AC9
:1071E00002EB0A0C51F8043F5B1B8C4540F8043F4E
:1071F000F8D1D9465B46304602EB0A0E50F804CF70
:107200001978AC4501F1FF3CD6BF013183F800C0CD
:107210001970704503F10103F0D1594640463B6BAC
:107220007A6098477B6B98477A68924456F8043F97
:1072300054F8042F5B1B002A83EAE371A1EBE3718E
:10724000B8BF52428A420ADA99F80020002B02F1B4
:10725000FF31D6BF013289F8001089F80020B2450D
:10726000236009F10109E1D1594640463B6B98473B
:107270007B6B98470C37BD46BDE8F08F76107FF4E6
:1072800070AF3B6B5946404698477B6B98473B6BCA
:107290005946404698477B6B9847E5E75946404634
:1072A0003B6B98477B6B98474FEA880A0AF10A03C1
:1072B00023F00703ADEB030D02466C468AE700BFDF
:1072C0002DE9F04F83B00D9EDDE90F9C002E40DDCF
:1072D000DFF88480DF021D0388FB073B88FB05384D
:1072E0000E9BFF17ED17013B5200C5EB68150024FC
:1072F00000EB01084FF47A7E41F2301AA7EB6B17CE
:107300001E44411A01921AE008FB00FB59F82400C0
:10731000019A381890FBF2F00EFB00F090FBF5F0AC
:107320000EFB0BFB0AFB00F00C9A9E4202FB10B016
:1073300090FBF1F04CF8240004F1010409D013F89B
:10734000010F0028E0D19E424CF8240004F1010412
:10735000F5D103B0BDE8F08F1F85EB512DE9F04F5B
:1073600091460646850099B02A46DDE9244808463C
:107370008A460021139312F05AFA2A460021484601
:1073800012F055FA72000021229812F050FA32469B
:107390000021239812F04BFA2A464046002112F0B1
:1073A00046FA002E40F3A480229B221F0693239BC3
:1073B000CDE9079A0B9300230293279B1092C3EB0E
:1073C000C3732A445B0012920F93109B53F8041F5F
:1073D00010934FEA116BC1F307435B450D9100F227
:1073E0002181002201230392279A29989A400BFBBE
:1073F00002020492DDE927200BFB02020992029AA5
:1074000093400C93CBB20193C1F307230E930E99D3
:10741000019B994232DB099B4FF0010E5E18DC465E
:1074200005E0900667D4019B01398B4225DC16F8F4
:107430000129029B9A42F4D1049B089833F9112048
:10744000039C036802FB024401FB02330394079C84
:1074500003602368069D0CFB0233288823601044D8
:1074600028800B9803789342DDDAFF2AA8BFFF2219
:10747000019B01398B420270D9DDE346049A0F99D2
:107480000D9B0A4404922799099A0BF1FF3BC3F321
:107490000743521A5B450992B9DD069BB3F90020F8
:1074A00092B108980399036891FBF2F15B0293FB98
:1074B000F2F30360079803685B0293FBF2F3029A0E
:1074C0000360139B23F81210029B109A013302935E
:1074D000069B02330693089B04330893079B0433EF
:1074E00007930B9B01330B93129B93427FF46DAF79
:1074F00019B0BDE8F08F00234FF601701C464B4DCC
:1075000018AF95F800B047F8040D494D2898169526
:10751000059302F00F0500EB010A0A9245FA03F009
:10752000C20719D516AAD056279A604402FB00A0BC
:1075300013F9079010F809900EFA09F0D94540EABE
:10754000040009D2A04207D0059A044618A81044A6
:10755000013200F80C9C05920133042BDED10C9B08
:107560000A9A23423FF45FAF049B33F911B0D3066C
:1075700016D49DF808307370089A039813680BFBB3
:107580000B0001FB0B330390079813600368069C04
:107590000CFB0B33228803609344A4F800B042E74D
:1075A0004FF00009059B0DF153005A1E914500EB69
:1075B00003070DF1540A1846CDF844B01CDA09F15E
:1075C0000109484514DD54469AF800B00A9214F8AF
:1075D000013F9B452ABF1D465D465B4658F8252066
:1075E0000EFA03F31343A74248F82530EFD10A9A65
:1075F00091450AF1010AE2DB059BDDF844B0032B5B
:1076000009D0042B04D0022BB6D14FEA6B0BB3E7A1
:107610004FEAAB0BB0E74AF6AB2303FB0BFB4FEA99
:107620006B4BA9E70023039337E700BF1CA80100B9
:10763000000001FF0288014B1A807047B41500203A
:107640002DE9F0414DF2502C4DF6DA37184C069EDC
:1076500094F8008094F801E006EB410611F1FF3147
:1076600023D336F9024D002CF8D032F9114033F90A
:10767000115068B905F5807504F58074B8F1000FF4
:1076800001D0C5F50055BEF1000F01D0C4F5884406
:107690000CFB05F507FB04F42D14241422F81150FB
:1076A00023F8114011F1FF31DBD2BDE8F08100BFBA
:1076B000B41500202DE9F04F40F6FF7CDDE9097696
:1076C00040F6FE7849F6C43944F21F6EACEB060B67
:1076D0000344A8EB060AACEB070C10F1FF3020D3F3
:1076E00013F8014D002CF8D031F9105032F9104048
:1076F00009FB05F50EFB04F42D14BD424FEA2444AA
:1077000013DDAC4501DCA8EB0705B4420BDDA34556
:10771000D8BF544621F8105022F8104010F1FF3025
:10772000DED2BDE8F08F3446F4E73D46EDE700BF1A
:107730000288014B1A807047B8150020002370B4EE
:1077400010481149114AC0E90033C0E90233C1E9C8
:107750000033C1E90233C2E90033C2E902330C4C01
:107760000C4E0D4D03610B611361C6E9003333818B
:10777000C5E900332B81C4E90033C4E90233236136
:1077800070BC7047AC190020701900205C190020F3
:1077900084190020D4190020501900202DE9F04F41
:1077A000474C85B02578834600900F466078164692
:1077B0009A4609248DF80C500E9D01938DF80D000A
:1077C000DFF8108104F094FBDFF80C9112371236C9
:1077D0000BF1120B0AF1120A254432E019F80430B9
:1077E00004A91144013311F8041CDBB2994209F8D1
:1077F0000430DC46D64644D24FF000012A786300BC
:1078000008F8042009F80410BCF900102D48C152F2
:10781000B7F900102C48C152B6F900102B48C152DC
:10782000BEF900102A48C152013C631C05F8012929
:10783000ABF1020BA7F10207A6F10206AAF1020AB8
:1078400038D005F05BFB58B1B6F90030002B07DDEE
:10785000B7F90030B3F5007FBCBF01238DF80C30C1
:1078600018F804202B789342B8D14FF0000309F8A0
:1078700004306300009901EB030C019901EB030E46
:10788000C2E7D3B10F4B33F914106300ABF800100B
:107890000D4931F9141039800C4931F91410318037
:1078A0000B4931F91410AAF8001019F80410002936
:1078B000BAD1DFE705B0BDE8F08F6300A4E700BFF1
:1078C000B815002084190020AC1900207019002080
:1078D0005C190020D419002050190020F0B40C7855
:1078E0001A4D14B305EB8406B6F8446086421CDDDD
:1078F0000027661EF6B21F700E702F6C013FA74264
:1079000006DD05EB8406B6F84C60B04217DC0E7855
:10791000B44218BF14701A780132D2B21A70696971
:107920008A4200DD1970F0BC70472E6C013EA64201
:10793000F1DD05EB8406B6F84C60B042E7DD0020CF
:10794000661CF6B218700E70E2E700BF300500202A
:1079500001467422014811F05FBF00BF30050020CE
:1079600010B4002201240A490A4B087D03F58C71EA
:1079700043F8082C03F8042C03F8034C03F8020C1A
:1079800003F8012C43F81C2B8B42F1D110BC70473B
:1079900030050020F0270020F0B49DF8104024B3FB
:1079A0003B4F3C4D012C18BF00272C78012C21D0D7
:1079B000002C4BD1D7F800C0BCF1000F64DDBE88AD
:1079C000B04247DB23463A4605E016892346864205
:1079D00002F104023EDC5C1C6445F6D1DAB20A70A6
:1079E00007EB8303D888F0BC70472A4D2A4F2C78C8
:1079F000012CDDD1686991F800C0002816784FF09D
:107A0000000408DD05F1140202EB800052F8041FA7
:107A100082420C44FAD11878A0B300211F4A02EB2D
:107A2000800052F8043F90421944FAD107EB8603D4
:107A3000B44507EB8C07D888FB881BD91B1A01FBC0
:107A400003F191FBF4F1F0BC084470474FF47A70F5
:107A5000F0BC70470A78A242134608DD4FF0640C70
:107A60006D780CFB00F006FB05F6B042B7DCE2B225
:107A70002346B4E7C31A01FB03F191FBF4F1F0BC18
:107A8000401A70470146D1E722462346A7E700BFC8
:107A90008C050020300500207405002044050020DE
:107AA0002DE9F04FC600351AAD00904C05F11807CE
:107AB00087B004EB0709002900F0FE8004EB050EF7
:107AC000DEF810100A2940F3E480D3F800C0CDE9B5
:107AD0000332331A9B00109A04EB03088346E058E4
:107AE0001168D8F80430ACEB0000C91A0028B8BF00
:107AF00040420029B8BF494203F0D0FF4FF6FF7360
:107B00008342A8BF034698F8172005F1150A29F803
:107B1000123098F8173005900133DBB2012B88BF83
:107B2000002388F81730DFF8C881B9F80210E35B4A
:107B300098F800200B4405F114095B101635012A52
:107B40000293A144A244254400F0C88000222B46A1
:107B50000092494652460298FFF71EFFA6EB0B0320
:107B600004EB83031A6998F80C3007469A42C0F276
:107B700087800A22A6EB0B0304EB83031A61012022
:107B800052462B46009049460298FFF705FFA6EBA8
:107B90000B0304EB83031A6998F80C3082469A426F
:107BA00006DAD8F81030059A9342C8BFD8F808A072
:107BB000049BA6EB0B0203F1010997FBF9F7039B6A
:107BC00092001B68A11803FB07FC8868A358C7F53F
:107BD0007A75034405FB03C3DFF818C14FEAE37E5F
:107BE0008CFB03030398CEEBA3130360109BC868C0
:107BF0001B6803FB07F74B68184405FB00778CFBF9
:107C0000075E109DFF17C7EBAE172F6098F8023084
:107C1000029DAB4210DB0023C1E90233039BA6EBBC
:107C20000B061B68B600A351109B02981B682644E4
:107C3000736007B0BDE8F08F9AFBF9F98B68A05824
:107C4000C9F57A7A039A03FB0AF31268121A09FB40
:107C500002338CFB0302DB17C3EBA213C8688B60F3
:107C6000109B00FB0AF01B684A689B1A09FB03097A
:107C70008CFB093C4FEAE979C9EBAC13CB60CDE74B
:107C8000D8F81030059A93427FF773AFD8F8047094
:107C900075E70131CEF810100129D3F800C07FF448
:107CA00016AF4FF00008109944F805C00968CEF8E7
:107CB0000C80CEE9011808E74FF480700C4A05F1FA
:107CC000100352690291E1502344988002982544A0
:107CD000E975AA75E15107B0BDE8F08F2B46524611
:107CE00049460298FFF7FAFD30E700BFD827002089
:107CF00030050020D34D6210F8B505461A4C0146F8
:107D0000B022204611F088FD2E1D04F15C0C0FCE30
:107D1000ACE80F000FCEACE80F0096E8030005F1C9
:107D2000300704F188068CE803000FCF0FC60FCF91
:107D30000FC697E8030086E8030005F18807261DB3
:107D40000FCF0FC60FCF0FC697E803005C35303456
:107D500086E803000FCD0FC40FCD0FC495E80300D4
:107D600084E80300F8BD00BFBC1500202DE9F84FE2
:107D70009DF8288004460E4617461D4604F0B8F8C4
:107D8000B8F1010F43D0DFF810B1DFF8109105EB27
:107D900044050BF1300A14F1FF3438D335F9023DB4
:107DA000002BF8D056F82400DBF8583098424EDA11
:107DB000B8F1020F00B20CBF4946344903F0C4FECB
:107DC000DBF8583056F82420D21A00FB02F003EBFF
:107DD000A01346F8243057F82400DBF8003098420E
:107DE00017DAB8F1020F0CBF4946294900B203F077
:107DF000ABFEDBF8003057F82420D21A00FB02F06B
:107E000003EBA01347F8243014F1FF34C6D2BDE8C9
:107E1000F88FDBF82C30C0F5F0509842BBDAB8F19F
:107E2000020F00B20CBF4946514603F08DFE57F8D1
:107E30002420DBF82C30C2F5F052D21A00FB02F2FB
:107E400003EBA213C3F5F05347F82430A3E7DBF8A4
:107E50008430C0F584409842BDDAB8F1020F00B218
:107E60000CBF49460B4903F06FFE56F82420DBF89F
:107E70008430C2F58442D21A00FB02F203EBA21353
:107E8000C3F5844346F82430A5E700BF1816002048
:107E9000C015002044160020BC1500201C06002040
:107EA000F0B4847A464B0278012C1A7021D14288B2
:107EB0004449C2EB0232A1FB02120226120A5A8086
:107EC0008188414DC1EB0131A5FB0121890A9980CF
:107ED000C1888672C1EB0131A5FB0121890AD980D5
:107EE00002893A49C2EB0232A5FB0252920A1A8178
:107EF0000C70027C012A4CD012B90121334A117056
:107F0000827C304C9A74B0F81320D0F81B50C2EB2E
:107F10000232A4FB0212C2F30F22A3F81320B0F81E
:107F200015202B49C2EB0232A4FB0262C2F30F22DE
:107F3000A3F81520B0F81720C2EB0232A4FB0262AE
:107F4000C2F30F22A3F81720B0F81920C3F81B5072
:107F5000987FC2EB0232060900F00F073D0530059D
:107F6000A0EB0620A5EB0725A4FB0262A4FB056598
:107F7000A4FB0004587F1E7F00EB1424154806EB79
:107F80001525C2F30F220D800480A3F81920F0BC40
:107F90007047002502261A7481890B4CC1EB013110
:107FA000A4FB0121890A9981C2890674C2EB0232BD
:107FB000A4FB02120549920ADA810D70A0E700BF06
:107FC0006C160020B5814E1B49D6B9F2F430002062
:107FD000F0280020982A0020002370B4124D134A84
:107FE00013482B606B60AB60EB602B61114D124C42
:107FF000124E136053609360D3601361036043605B
:108000008360C36003612B606B602B8123606360BE
:10801000A360E3602361336073603381194670BCF1
:108020002822074811F003BC983100200C290020B9
:10803000842A002050290020B0310020F42800209C
:10804000CC260020C0F5FF630733002B2A4BB8BFB6
:10805000C0F57F621B78B4BF0E320246D3B110B4B4
:10806000264B1C8994422BDD002C39D0244A1288DF
:108070008A4235D8234A12888A4231D3DB7E012BCB
:1080800033D0022B2CD140F2FE71884294BF0220E3
:10809000012026E0194BD889904201DD022070476B
:1080A0009A7C02B3B3F817208A42F7D8B3F81900C4
:1080B000C0F57F600F308142CCBF022001207047A5
:1080C0009A7C52B1B3F817208A42CDD8B3F8192060
:1080D000C2F57F620F328A42C6DB012010BC7047B6
:1080E000022010BC70470120704740F2FE718842A8
:1080F0008CBF02200120F4E7F43000206C16002031
:10810000F0280020982A00202DE9F04F91B08346F6
:1081100007A8CDE901238A461A9E01F007FC9DF8C5
:108120002530022B00F0B780644B1B780593002BA1
:1081300000F0B1800024A146DFF89C81604AABF1D9
:10814000020BAAF1020A31783BF9027F3AF9025F89
:1081500018F8013B002941D0A9B2B8B2CDE90332E9
:10816000FFF770FF019B012833F914E0029B33F9FC
:1081700014C0DDE9033200F08A80022824D1115DA9
:1081800019BB4FF0010111555BBB4E494E4851F8E8
:10819000241020F81470481C01214C4F27F814506B
:1081A0004B4D25F814E04B4D25F814C03370454B6A
:1081B00043F8240001340A2C08F8011C06F10106DA
:1081C000C1D111B0BDE8F08F115D0129DCD0012BC8
:1081D00007D03C4B115D43F82490EBE7012B115580
:1081E000F7D1394B4FEA840C33F9141063007F1A2E
:1081F000002FB8BF7F423349972F51F8240017DC76
:10820000324931F914106D1A002DB8BF6D42442D5A
:108210000EDC2F28115D02DC11F0FD0542D0012992
:108220003ED1284B013086F8009043F80C00C1E79E
:108230004FF00201115505992F28C8BF00210846AB
:108240000221204D45F80C900028B3D01E4D1F4F41
:10825000E85E019DABF80000F85EAAF800001C483B
:10826000185E25F814001B48029D185E25F81400BE
:108270004FF001051648357023F80090124D15484F
:1082800025F8039027F8039023F8009092E74FF029
:10829000020111559BE711B0BDE8F04FFFF79CBEFE
:1082A0000020CEE7012903D0064840F80C50CDE766
:1082B000044D013045F80C00C8E700BF6C160020E3
:1082C00050290020CC26002098310020B031002019
:1082D0000C290020842A0020F4280020C0F5FF6328
:1082E0000733002B3C4B70B41D78BABFC0F57F64D8
:1082F0000E34044645BB9A7C002A51D0B3F81320B3
:10830000364E8A42367806D8B3F81520C2F57F6219
:108310000F32914257DD002E45D02522304D2D8859
:108320008D4240D82F4D2D888D423CD3A2423ADA5F
:10833000DB7E012B49D0022B35D140F2FE71884201
:1083400094BF022001202CE0244A1278A2B16429B3
:108350005A882BD8914232D89A7C52B1B3F8132064
:108360008A42DAD8B3F81520C2F57F620F32914203
:10837000D3DC70BC012070479A89A24213DC9A7C3E
:10838000002AF6D0B3F813208A420CD8B3F81500AF
:10839000C0F57F600F308842B4BF0220012000E0AA
:1083A000104670BC7047022070BC7047914206D8DE
:1083B0009A88A242D0DD252A28BF2522AEE7DA8896
:1083C000A242F8DCC8E72846EBE740F2FE7188429B
:1083D0008CBF02200120E4E76C160020F43000205E
:1083E000F0280020982A00202DE9F04F8BB0064697
:1083F00001A80F4601F09AFA9DF80D30022B38D0F3
:10840000204B1B7873B300244FF00209A0464FF0B5
:10841000010A149BDFF870B05D1E15F8013FDBB157
:1084200037F8141036F81400FFF758FF012816D05B
:10843000022805D11BF8043023B90BF804A003E08F
:108440001BF80430012B01D185F8008001340A2C7F
:10845000E3D10BB0BDE8F08F0BF80430F6E70BF872
:108460000490F3E7084A1360536013810BB0BDE832
:10847000F08F0022044B1A605A601A810BB0BDE8DD
:10848000F08F00BF6C160020002900202DE9F0417C
:1084900005460E461746984682B0089C0094FFF7A2
:1084A000A3FF43463A4631462846089402B0BDE849
:1084B000F041FFF729BE00BF01465422014811F0E8
:1084C000ABB900BFA40500200021044B03F17802E2
:1084D00099600C339342FBD1704700BF20310020DC
:1084E00030B40546064C6968AA68EB6800680FC49A
:1084F00028696969AA69EB690FC430BC704700BF7D
:108500008C1600202DE9F04F514ECBB0726800213F
:108510009200824611F08BF973683269581EA0EB05
:10852000630090477369984773685A1E0592002B41
:108530007CD0D6F800900AEB830AA3F1020849AC7C
:1085400088224FF0FF3106A811F071F9882200212E
:1085500028A811F06CF919F1FF39DDF814B02FD308
:10856000B36998470746BBF1000F6AD0706833695A
:10857000A8EB6000984719EB0B0F01D0736998477F
:10858000384606A927AA03680F68BB4202D20B60CF
:108590001F46036852F8045F04309D423CBF1D46ED
:1085A0001360D0F884300431BB4238BF41F8043C3A
:1085B000AB4288BF13609442E5D119F1FF39CFD2A5
:1085C000002727AA05A952F8040F51F8043F0744D1
:1085D0009442A7EB0307F6D11E4B4FF001094FF071
:1085E000040B039300234946CDE90193222228ABD3
:1085F0007220CDF800B0FAF717FC174BCDE900B99F
:108600000393002349460293222206AB7220FAF715
:108610000BFCD6F80090059B97FBF9F7013B0593FF
:10862000013308F1FF384AF8047D89D17368326953
:1086300003EBD3705B10C3EB600090474BB0BDE819
:10864000F08F73683269581EA0EB6300904792E781
:108650008C16002028A801003CA801000E4BF0B4A5
:108660005F68022F15DD00EB87070C3F04380246D8
:1086700000230A4900F10C0652F8045F11F9014B7E
:10868000964205FB0433F7D11B1140F8043F8742A3
:10869000EDD1F0BC704700BF8C160020981600206A
:1086A000DFF868C0F0B4DCF804600024002E0ADDB6
:1086B00001EB8606043E0B1F53F8045FAC42B8BFC3
:1086C0002C469E42F8D1DCF808304610A34214DA5A
:1086D000002818DD00236FF00045043951F8044FDD
:1086E000AC42B8BF1F4603F10103B8BF254698420C
:1086F000F4D1B81B1560F0BC704751F8263000204B
:10870000F0BC136070476FF00045F2E78C16002054
:10871000F0B40446074E00F1300735462068616822
:10872000A268E3681034BC4206F110060FC5F4D10C
:10873000F0BC7047AC1600202DE9F047DFF8E89058
:1087400002EB400599F82C3099F82D2082B0441E98
:108750000F468DF804208DF805304E464FF0000A84
:108760004FF0640800E0013C631C17D035F9023D6E
:10877000002BF8D0314637F9140003F0E5F9B5F9CC
:10878000003098423EDBD9F8282008FB03F302FBB7
:1087900000F29342C8BF4FF0020AE4E71F4B18787B
:1087A000BAF1000F13D11E4AC2F800A060B91D49EA
:1087B00099F82E400A680132A2420A6004DD0122C3
:1087C0001046C1F800A01A7002B0BDE8F087054657
:1087D000AAF10200B0FA80F04009854217D0104C8F
:1087E00002A92268014411F8041C01328A42226065
:1087F00011DD00221870226000220A4B1A6002B0BC
:10880000BDE8F0870020054B1D788542E7D10022A6
:10881000034B1A60F0E72846EEE700BFEC19002092
:10882000E0190020E8190020AC160020014B187058
:10883000704700BFEC190020034B1B781BB9034A9B
:108840001368013313607047EC190020E819002009
:108850000278014B1A707047F80500200022034B84
:1088600083F8F02083F8E421704700BFA82A002095
:108870000268014B1A607047DC1600200146B822DE
:10888000014810F0C9BF00BFE016002070B4D0E965
:1088900000250A4B8468017B867B1A605D60427B01
:1088A000C57B9C60047C19735A739E73D0E90512D2
:1088B000DD731C74C3E9051270BC7047E01600201C
:1088C0002DE9F0430746032200204FF0010803FB87
:1088D00007F6079D104C29448E5D94F80090DFF850
:1088E0003CE0DFF83CC006F00F0646FA02F4E4076D
:1088F0000CD512F90E4012F90C503C4403FB041441
:10890000645D4C453CBF08FA04F4204312F1FF3289
:10891000EBD2BDE8F08300BF20A8010050A8010001
:1089200058A801002DE9F04F8DB0199F054605901C
:1089300097F802B0F87888468345CDE90832DDF82B
:1089400074A04DDC0123B8461F9C0BFA03F20AFB0E
:10895000024204921E9A97F801900BFB0A2603FA32
:1089600005F28B40134303934FEA4A030693EBB29D
:10897000CDE90A13079298F800404C450CDD23E03E
:10898000FA0606D4079B834200F09780002800F087
:10899000B1800134A14515DB375DB906F9D51E9BC1
:1089A0001C9A0093214653465846FFF789FF039BC4
:1089B0008342E5D19DF81430335598F80190013485
:1089C000A145E9DA98F80300049B069A0BF1010B24
:1089D0001344584556440493CDDA4746DDF82880C1
:1089E0001A993B680846059A40F8223050F828301A
:1089F0009400C3F30741B1EB136F4FEA88003B606B
:108A000019DC94461E9B97F801900AFB01353B78D0
:108A100099450BD32B4413F8016B464504BF03F86B
:108A200001CC97F801905A1B9145F4DAFB7801319B
:108A30008B425544EBDA1B9B08F101011844099B5A
:108A40008B420FDD01279C461B9A059D161952F893
:108A50002550026807FA01F3134001311D438C458C
:108A60003560F6D100231B9A984542F8283040F330
:108A700083800122059F1B9802FA08F10444BC463A
:108A800002FA07F0CD4316461B9F06E002432A4038
:108A900047F82320013398456ED057F823200A4227
:108AA000F8D09C45F2DCF2DA226806FA03FE42EACC
:108AB0000E02226057F82320E9E79DF81430089849
:108AC0003355049B98F8019033F91420036804FB94
:108AD00002F103EB412303600BFB02F1169B1B68C1
:108AE00003EB412316990B60189B1B681344189ADB
:108AF00013604EE707F00F03CDF864800325984616
:108B000048FA05F3DB072FD51D4B1C9AEF561D4B7A
:108B10005F4415F903901E9BA144009338465346C9
:108B20004946FFF7CDFE039B83421DD11E9B0B9A46
:108B30000AFB0737049B07F80920325533F9142044
:108B4000089804FB02F1036803EB412303600BFB6D
:108B500002F1169B1B6803EB412316990B60189BCF
:108B60001B681344189A136015F1FF35C8D2DDF85D
:108B7000648098F801900CE70DB0BDE8F08F00BF5D
:108B800050A8010058A801002DE9F04F814293B090
:108B900005460C460B9298461C9F01DB04460D4689
:108BA0001E9B58F824A033F914201D9B57F82490DD
:108BB00033F814C002FB0AFE09FB02F602FB0CFCB0
:108BC0001D991E9B31F815B033F9153058F8250062
:108BD00057F8251003FB00EE03FB0BCC01FB0366EB
:108BE000AAEB00001344A9EB0101CDE90FC3CDF8B6
:108BF00034E00E9602F052FF209B834653F8242067
:108C000053F825309446D9B2D0B2884288BF61F378
:108C1000070CC2F30720C3F30721884238BF61F372
:108C20000F2CC2F30740C3F3074188424FEA136396
:108C300088BF61F3174CB3EB126F88BF63F31F6CEF
:108C4000269B239A0993259B0692229A0893249B9C
:108C50000592209A0DF1440E10A80FA907930EABB0
:108C6000CDE900310492CDE9020E0B9A0DAB2946F5
:108C70002046CDF844C0FFF755FE0DA80FC891FB64
:108C8000F3F190FBF3F092FBF3F24FEA840948F81A
:108C9000090047F809101D9966008A531E9A4FEA89
:108CA000450A9353219B33B19B5F9B45B8BF9B46BD
:108CB000219B23F806B01F9A1F9B115D5B5D00226C
:108CC0008B4238BF0B461F990B551E9B23F80A2079
:108CD00013B0BDE8F08F00BF2DE9F04FDFF8D0B042
:108CE0008FB09BF80C40189F002C5ED000285CDDF4
:108CF00000250D9337F9153005F1010A002B914637
:108D00008846064654464EDD564503DC4DE00134A8
:108D1000A64240D037F91430002BF8DD59F8243042
:108D200059F8250058F82510C01A4DF6DA3358F8CE
:108D30002420891A0029B8BF494203FB01F14DF2F2
:108D400050230028B8BF404203FB00F00914001470
:108D500002F0A4FEDBF814308342D8DD209B2146CC
:108D60000A931F9B324609931E9B284608931D9B1E
:108D7000013407931C9B06931B9B05931A9B04933A
:108D8000199BCDE902730D9BCDE900934346FFF794
:108D9000FBFEA642BED1554637F9153005F1010A52
:108DA000002B5446B0DC5645F5DC0FB0BDE8F08F23
:108DB000E01600202DE9F04F654C95B0247C1E9FF5
:108DC00034B3002824DD90468A4681464FF0000BDC
:108DD0000D9337F91B30BBB158F82B20249902F5BD
:108DE0008072521201FB02F65AF82B30259903F5D6
:108DF000807331445B12C95C56485945057825D0CB
:108E0000A94209D3880671D40BF1010BD945E0D1F1
:108E100015B0BDE8F08F7746269B4A460A93259BFE
:108E200058460993249B0893239B0793229B069300
:108E3000219B0593209B04931F9BCDE902730D9BFF
:108E4000CDE900835346FFF79FFEDDE74FF0FF308B
:108E50006FF0FE1C864603243D49CDF84CC089685E
:108E60000DF1480C11913C490E95129126991E97CF
:108E700001EB4601109159000F9113AE1EEB020E4B
:108E800018442BD4002829DB2399714526DD249929
:108E9000814223DD01FB0EF725990E9D3944095CC3
:108EA000A9421BD20F9D8B4505EB470716D0269D87
:108EB00035F907E06425109F05FB0EFE37F91370A6
:108EC000119D05FB07F7BE4508DD109D35F9100023
:108ED000AE46642505FB00F0B84237DC24B1013C06
:108EE00014F90CE0A057C9E71E9F8DE7209850F8B1
:108EF0002B00C0F307249C4224D0C0B298420BBF81
:108F0000032401244FF0020C4FF0000CBE4601F088
:108F10000F0025990B4440FA04F1C9070DD50F49FC
:108F2000249F61560E4E114407FB0131A657895DFF
:108F3000A94202D259457FF46EAF013C6445EADA9A
:108F4000774661E703244FF0020CDFE71E9F63E7DB
:108F5000E016002020A801000101FFFF50A8010039
:108F600058A801002DE9F04F83B0DDE90D4704FB5F
:108F700002FE07EB0E04E65C864245D08E4243D0EB
:108F800016F0200549D000250324AA464FF0010B16
:108F9000DFF8A4C006F00F069CF80090019307EBE1
:108FA000030C46FA04F7FB0715D5214F214BE75771
:108FB00014F903800D9B174403FB07C717F80880BB
:108FC0000BFA08F7C84547EA050704D2AF421CBFB1
:108FD0003D460AF1010A14F1FF34E2D2012202FAFD
:108FE00000F002FA01F10843A842019B19D0284081
:108FF00010D05B0003EB4E0E0F9B33F90E0090FB7D
:10900000FAF003B0BDE8F08F5B0003EB4E0E0F9B50
:1090100033F90E0003B0BDE8F08F284603B0BDE879
:10902000F08F934003EB4E0E0F9B33F90E00F1E7E8
:1090300050A8010058A8010020A801002DE9F04F18
:10904000B74CADB0E47B1D94002C00F00E810028DD
:1090500000F0038121930023CDE91B121293431EDC
:1090600016902093129B209A934280F2FE803A9BA6
:10907000129A194651F82230511CCB404FEA820215
:109080001E911792119300F05981169B19461E9B51
:10909000994240F3538110930023129A1F93369BF9
:1090A00003EB42031A930BE0109B119A0133520811
:1090B0001093119200F03E81169A9A4200F03A8184
:1090C000119BDB07F0D51B9B17991C4658581C9B1E
:1090D000109A1D4654F82240595855F82230051B65
:1090E0000E940F93CC1A85EAE573A3EBE5731893FE
:1090F00084EAE473A3EBE4731993369E1A9B36F962
:109100001220B3F90030002C40F0FF80002D40F019
:1091100018814FF4007BDDF874800E9E0F9F34465B
:109120003D4604FB03F402FB004405FB03F5134436
:1091300094FBF3F402FB015595FBF3F5389B179A6A
:109140009C469A5824941446CDE925610026109B2C
:1091500023905CF82330D0B2D9B2814238BF61F39A
:109160000704C2F30720C3F30721884238BF61F325
:109170000F24C2F30740C3F3074188424FEA136349
:1091800088BF61F31744B3EB126F88BF63F31F64AA
:109190002795230EC4F307459D422897CDE92966FC
:1091A0002B9600F3D48001331393E3B21493C4F3EA
:1091B0000723159329AF149C159A94425CDC9DF803
:1091C00048306E020D933346464698469DF840A0BF
:1091D00002F101093E9B2A4603933D9B51460293AF
:1091E0003C9B0D9801933B9B00932346FFF7BAFEEF
:1091F00000283DDDDDE90E324FEA442C0221ACEBC4
:10920000030E0EB30BFB0EF3A2EB6323A3EB0803D9
:10921000002BB8BF5B42B3F5007F09DAC3F50073DA
:1092200000FB03F357F8212002EB632347F82130BA
:10923000F1B1013923AB53F8213026AA52F821208D
:10924000ACEB030E002EDDD1A8EB02020BFB02F209
:10925000A3EB6223A3EB0C03DAE76FF00043314C7E
:109260003149324A23600B6010602DB0BDE8F08FA9
:1092700001344C45AED1B046139B01359D429AD185
:10928000DDE92A42DDE91801299B64259A42A8BF3D
:109290001A4605FB04F4154602F038FC2D2801DDC2
:1092A000C0F15A001E4A0CCA03FB00F3C0F12D00A6
:1092B00002FB00321E4B83FB0231D3170A44C3EB7F
:1092C000621305FB03F3A342BFF6EEAE3E9B169A74
:1092D0000A933D9B109909933C9B129808933B9BE2
:1092E00007933A9B0693399B0593389B0493379BCE
:1092F0000393369B0293219B01931C9B00931B9B22
:10930000FFF742FC1D9B1F93CEE6DDE91867BE42C6
:1093100017DA6D0295FBF4FBDDF87480FDE600BF03
:10932000E01600204406002048060020081A00200D
:10933000B7600BB61F9B002B7FF494AE1E9B12935D
:1093400090E6640294FBF5FB4FF00008E5E6DDE9EA
:10935000180102F0DBFB2D287FF7A6AE00252C4676
:109360009EE700BF2DE9F04FA54CAFB0A47B002CC9
:1093700000F03481002800F0318191461793389B2A
:109380004FF0000B023B189303EB400310934B4646
:1093900089469A460D901E2200211EA810F047FA19
:1093A00000211E2226A810F042FA964B4FEA4B01EC
:1093B00033F91B301391002B40F33681924B33F974
:1093C0001B30C3EBC3139B1214930D9B002B40F374
:1093D0002B8100278D4A189B8A180F928C4A12976E
:1093E0008A180E921D46CDF858B003E0109B013745
:1093F0009D4272D035F9022F002AF7DD0E9B0F989F
:10940000B3F9004059F827205AF82710B0F90000A6
:10941000611A801A02F042FB66243A9E7D4904FBE1
:1094200000F4F05D51F8046C02F08EFBA41280464B
:10943000794920B202F088FB0E9A15900F98B2F984
:1094400000C05AF82710B0F9002059F82700ACEBFB
:1094500001016B4B101A00299A6FB8BF49420028CE
:10946000B8BF4042D3F87CB0119202F04FFB2D28D8
:10947000C8BFC0F15A0000FB0BFB119AC0F12D00D0
:1094800002FB00B2654B664983FB023C139B94448C
:10949000595ED2170E44C2EB6C1208FB04F806FBAF
:1094A00002F6B04580F29D806420554BD3F88020B1
:1094B00000FB02F2424540F39480159B8B42129BC5
:1094C00003F1010280F28D800121D3B212931EAB11
:1094D000D955109B01379D428CD1129BDDF858B0B5
:1094E000012B40F2A1809DF87820002A40F0938162
:1094F0001EA913460D9C04E011F8010F002840F04E
:109500007D8101339C42F7D1199B9F004FEA4308AC
:1095100009EB07030F930AEB070311933B9B1F44CF
:10952000389B43441293399B98440026CDF84CB0A5
:10953000CDF83880DDF834B0DDF864801DAC1CADAA
:10954000002A3DD0B0453BD026AB9B5D419A002B15
:109550003C9B18BF00230A92409A059309923F9AB8
:109560004B4608923E9A314607923D9A40460692F3
:109570003B9A04923A9A0392389A0292179ACDE94A
:1095800000A25A46FFF700FB3868129B119A0F9908
:10959000B3F900301268096802904198CDE900548F
:1095A0000690409805903F9804903E98039040465E
:1095B00001F0A8F9DDE91C0102F070FA0E9B188099
:1095C0000136B3452ED01EAB9A5DB9E7109B0BF167
:1095D000010B023310930D9B5B4538D12FB0BDE8D2
:1095E000F08F149BA3427FF701AF0122129911441F
:1095F000CBB2129326ABDA551EABDA55F6E600BFB6
:10960000E0160020E029002014270020E030002090
:10961000C42700200817002030170020B7600BB6C1
:109620000C310020DDF84CB00BF1010BBBF10A0F3F
:109630007FF4B1AE5346CA4699460D9B002BCDDD53
:109640004FF0000B399B4C46DDF8E090109339F950
:109650001B3009EB4B02002B1892B7DD4FEA8B034E
:109660000AEB03021B93E3184FF000081A921993B8
:1096700040E02E4659464546419B0D9A0A93409B31
:10968000284609933F9B08933E9B07933D9B069377
:109690003C9B05933B9B04933A9BCDE90293179B1C
:1096A000CDE900435346FFF76FFA3B980E9F0F9B9F
:1096B000C059159A1699B3F90030126809680290DA
:1096C00041980690409805903F9804903E980390EA
:1096D00026A801901EA80090284601F013F92699AB
:1096E0001E9802F0DBF930800D9B08F1010843451C
:1096F0003FF46CAF39F918304FEA480509EB050221
:10970000002B0F92F0DDC345EED054F828205AF814
:10971000283054F82B105AF82B00891AC01A02F07E
:10972000BDF95AF82B3011905AF8280054F8281037
:109730001B1A54F82B2083EAE376A6EBE3763A9BD8
:10974000521A82EAE277394913F80B00A7EBE27765
:1097500002F0FAF93A9B1290344913F8080002F02B
:10976000F3F9334A3946D2F8B030139030461493A7
:10977000D2F8B46002F0CAF942F2107C4FEA8803D2
:109780002D280E935344C8BFC0F15A0016930E9B68
:1097900000FB06F6E3181593149BC0F12D0003FBA4
:1097A0000063234A109E2348D2F88470B6F9001053
:1097B00080FB0320129A184402FB017E3999139A08
:1097C00031F91810DB1702FB01E2C3EB6010119BAB
:1097D00002FB00F20CFB03FC399B94451D4483DA29
:1097E000C345FFF646AF189B41460F93199B5D4654
:1097F00015931A9B16931B9B0E933DE79F0009EB55
:1098000007010F910AEB070111913B994FEA4308B9
:109810000F44199384E6389BDDF8E480CDE911A369
:1098200000233B9FCDF83C9019937EE668170020FB
:10983000E0160020B7600BB684B038B5174D04AC05
:1098400084E80F00232240F21461154804AC00F0B4
:10985000C7F80FCC28606960AA6003CC1822286181
:10986000696128464FF4B871EB6000F0B9F80D4912
:109870004FF4606000F002F90B494FF4905000F093
:10988000FDF8642000F022FD632000F01FFDBDE81C
:109890003840602004B000F019BD00BFF42600205D
:1098A00050060020AC060020BC06002084B030B476
:1098B00002AC84E80F000A4B9DF808209DF80A10BE
:1098C0009DF812509DF813401A7099709D72DC72C9
:1098D00030BC184618224FF4B87104B000F0AAB892
:1098E000F4260020F8B500F0DDFA0446094E00F138
:1098F0002007354620686168A268E3681034BC42DE
:1099000006F110060FC5F4D12288A3783280B37017
:10991000F8BD00BF50060020034B187AA0F11000DC
:10992000B0FA80F04009704750060020F0B40746B6
:1099300005460B4E06F1200C34460FCC64452860DA
:109940006960AA60EB6006F1100605F11005F3D11D
:109950003288B37838462A80AB70F0BC704700BFBD
:109960005006002070B40446174D00686168A26874
:10997000E368164E0FC520696169154A03C573680F
:10998000A569207F51692B4373600870A37F657FB1
:10999000CB71E17F93680F480570197094F820002F
:1099A0000D49587094F821500C489D7094F822503D
:1099B000DD70D368A28DD4E909651A811E605D60EF
:1099C000086070BC704700BF1C2A0020FC08002003
:1099D00084080020581A0020C0270020499F00005A
:1099E000F8B5134B0C0A53F824606EB1F468CFB28B
:1099F000013C05E073681B5DFB1A002B05DA2C4661
:109A0000631C04F1FF35F5D1F8BD1546B368326823
:109A100033F81430014652F824002A4618440FF057
:109A2000FBFEB36833F814202A4423F81420F8BD51
:109A3000DC060020104BF0B40C0A53F824706FB110
:109A4000FB68CEB2013B05E07C68E45C341B002C73
:109A500006DA2B46591C03F1FF35F5D1F0BC7047EF
:109A6000BC68396834F8134051F82350A41A0146F1
:109A70002819F0BC0FF0D0BEDC060020044B000A11
:109A800053F820201AB9142898BF43F820107047C3
:109A9000DC06002000232DE9F043036069B3CE68A3
:109AA000D2B206F1804C06F100470CF1FF3C013FB9
:109AB00006F1FF3EB342A7EB0308AEEB0305ACEBA8
:109AC000030915D04C680133645D141BF2D40D6892
:109AD00055F82990B9F1000F07D08D6835F8185066
:109AE0002D1B002DE6DD0560A1444846BDE8F0834E
:109AF0004FF000094846BDE8F0838946F5E700BF0E
:109B00000023B1F5704F70B4C1F30724036028DA65
:109B1000132C1FD9144D06466A68E86889B2431EA3
:109B200002EB400204E032F8020D081A07D5234682
:109B3000581C03F1FF34F6D1002070BC7047AA68AE
:109B4000296852F8232051F82330121A3260184441
:109B500070BC7047054B8AB253F8241070BCFFF7F5
:109B600099BF1846E9E700BFCC060020DC060020BC
:109B700000B583B0014601A8FFF7C2FF044B18608F
:109B800008B1019B1844034B186003B05DF804FB57
:109B90004C1A0020501A002070B50E4E024635684F
:109BA0001DB10D4B1C68A54206D314460846002182
:109BB0000FF03DFE204670BD641B8442A8BF0446E2
:109BC00008462246294625440FF026FE35602046E9
:109BD00070BD00BF4C1A0020501A002070B50B4E0B
:109BE00035681DB10A4B1C68A54202D300242046EB
:109BF00070BD641B8442A8BF044628462246254403
:109C00000FF00AFE3560204670BD00BF4C1A0020E0
:109C1000501A0020B0F5C06F70B517D0234B1A78DA
:109C2000D20908D1B0F5047F18DC214B5B699BB1E8
:109C3000BDE87040184793F90020002AF5DAB0F526
:109C4000047FF2DD1A7802F07F0213E000291CDBAA
:109C5000184B1A78A02A25D0002070BD1A7802F07F
:109C60007F02140104F21124844217D893F90030C2
:109C7000002BDADA02F504728242D6DB43189A42EC
:109C8000D3DA00F03BF8012070BD084B1A78D209F6
:109C9000E4D093F90020002AC7DAD3E74518AC4294
:109CA000E4D8EEE7052201201A7070BD941C002054
:109CB0001C2A00207C070020024B1B6903B11847B7
:109CC000184670471C2A0020084B094A5B78DBB213
:109CD000012B137006D0022B03D10122054B5A70C1
:109CE00070477047044B1B68184700BF900700205F
:109CF000981A00207C0700201C2A002008B50A4B77
:109D00001B78012B0CD0022B02D10022074B5A707A
:109D1000074A137803F080036FF3C713137008BD6D
:109D2000044B5B689847F3E7981A00207C070020F3
:109D3000941C00201C2A00202DE9F843254EDFF852
:109D4000A8903378244DDFF89C80244F012B06D057
:109D5000022B1BD06A78934238D1BDE8F883D8F83B
:109D6000083098470446B9F1000F28D1D8F80430DC
:109D70009847D8F800309847DFF870906B783278C1
:109D8000DBB2934209D1002CE0D1E6E71A467C7899
:109D90006B78E4B2DBB29342F5D0012A12D0022AEA
:109DA00002D100220D4B5A700D4A69781378317038
:109DB00003F080036FF3C7131370BDE8F88309F154
:109DC000FF39DBE7074B5B689847EDE71A46012A46
:109DD000E5D1F7E7981A0020900700207C070020C3
:109DE000941C00201C2A0020FF2C0100FE2C0100E6
:109DF00038B5194C2378012B17D0022B0CD0174AF9
:109E00005278934206D0164A137803F080036FF31A
:109E1000C7131370002038BD124B104A597852787E
:109E2000022AF7D000225A70EDE70F4DAB68984731
:109E300018B16B6898472B6898470A4B07492278F6
:109E4000587849789142E5D0012A02D16B68984749
:109E5000D9E7022AE6D0D6E7981A0020900700201A
:109E6000941C00207C0700201C2A0020A023034A09
:109E700013701378A02BFCD0704700BF7C07002024
:109E8000014B1878704700BF90070020014BD8782D
:109E9000704700BF90070020014BD870704700BF8B
:109EA000900700200048704794070020014B9878E5
:109EB000704700BF90070020014B9870704700BFAB
:109EC0009007002008B5FFF793FF08B9014B186011
:109ED00008BD00BF901C00200A46F8B5094F0A4C87
:109EE0003B6826689B79B51803EB830103EB4103BC
:109EF0009D4200D9FFDE0146B86830440FF08CFC6B
:109F00002560F8BDD0070020901C002070B50D46DC
:109F10000646FFF711FF094A094C1378094963F017
:109F20007F0365F306038D80A5681370A660FFF7B5
:109F3000CBFEFFF701FFA56070BD00BF941C0020A1
:109F4000D0070020DC0700202DE9F04F89B00093F6
:109F50009DF860409DF868300746884691469DF818
:109F600064A001939DF86C503CB1FFF7ABFF002853
:109F700000F0148109B0BDE8F08F8D4B1E460293AE
:109F8000FFF7DAFE34600024A742CDE90444CDE9AE
:109F9000064440F3EC806B4203F00303159E854DAD
:109FA000039382E038F9142039F91400002900F0F5
:109FB000C180B5F90030934200F0F3804FF0010CFE
:109FC0009DF8103004EB0C016CF3010361F3850381
:109FD000022161F387138DF810309DF81330139927
:109FE00062F3071351F8241060F303031211C1F355
:109FF000072C8DF813308DF81120CBB2C1F3074236
:10A00000ACEB0303C2EB1162001193428DF8120016
:10A0100040F39F804D2101FB03F39B118DF8152028
:10A020008DF81430009B169933F914309DF81620E2
:10A030001B113F2BA8BF3F23095D63F305028DF879
:10A040001620002940F09080019B002B40F0A38057
:10A050009DF80C209DF817109DF8160062F38711EB
:10A0600063F38710149B6FF345111B5D8DF8171078
:10A07000102100228DF816000DEB01008DF819302B
:10A080008DF818A08DF81A20FFF726FF38F9143044
:10A0900031782B8039F914306B800134A742297153
:10A0A00006F1010605F1060561D033782979002B08
:10A0B0007FF478AF0029F0D001219DF810209DF8A1
:10A0C00017E09DF81AC0B5F9000061F3010263F3CF
:10A0D000871E9DF8131063F3030C63F3451E63F3AF
:10A0E000071CADF814308DF816308DF818308DF847
:10A0F0001930B5F9023060F3071163F303018DF8ED
:10A100001310102104F1010B00116BF3850262F0B2
:10A110003F028DF811001B110DEB01008DF810208E
:10A120008DF812308DF817E08DF81AC0FFF7D4FEC5
:10A130003178B2E74FF0010C9DF8103004EB0C01C0
:10A140006CF3010361F385036CF387138DF8103012
:10A1500043E74D2303FB02F2ACEB010192118DF8B2
:10A1600015108DF814205DE701231A4672E7029B53
:10A170001B68002B3FF4FEAE0F491C090A780F48FC
:10A1800002F07F0264F306020A708380FFF79CFDF1
:10A1900009B0BDE8F08F012302225BE7044B029374
:10A1A000F1E6B5F9023083427FF408AF75E700BFEE
:10A1B000901C0020981C0020941C0020DC0700202C
:10A1C00030B5094D83B02B780446834208D00B2369
:10A1D000022101A88DF805408DF80430FFF796FEA6
:10A1E0002C7003B030BD00BFDA1C002000B583B076
:10A1F0008DF804008DF8051001A80221FFF786FEF6
:10A2000003B05DF804FB00BFF0B4224C82B02578A7
:10A210008DF80720854202D002B0F0BC7047FF26BF
:10A220001D4802AD076B15F8012DBF681B48920051
:10A230000361C0E902151A4B3A81069A26701A602A
:10A240008A7822B30B7908784E7902FB003006F049
:10A250007F06144B06FB00F09F6838608B795BB17A
:10A260000022013B01EB83056D89013B2A445D1C03
:10A27000F8D102FB06023A60A0230B4A1370237840
:10A28000FF2BFCD00523137002B0F0BC70474A7856
:10A29000D8E700BFDC1C0020DC060020FC07002003
:10A2A000401A0020CC0600207C070020014BDB6810
:10A2B0005881704784080020034B1879A0F10100F1
:10A2C000B0FA80F040097047EC1C002000B583B064
:10A2D0000146202268460FF07BFA01230099064AC6
:10A2E000019802EB8102D2F8051083400B43C2F8BB
:10A2F000053003B05DF804FBEC1C0020014B18781E
:10A30000704700BFF808002070B4184A184B9060DE
:10A310001960827802B9427803790178457902FBA5
:10A32000013105F07F05134B05FB01F19E6831609B
:10A3300083795BB10022013B00EB83046489013B1C
:10A3400022445C1CF8D102FB05123260A024FF23DA
:10A3500009480A4A04700A49137002E00B78022B7C
:10A3600002D11378FF2BF9D070BC7047EC080020A5
:10A37000401A0020CC0600207C070020F8080020AE
:10A38000900700200246024B0068516803C37047E3
:10A390009817002000230B490B4A0C4810B4C1E960
:10A3A0000033C1E90233C2E90033C2E90233C0E934
:10A3B0000033074C0B6113610381C4E9003323812F
:10A3C00010BC704798190020C0190020FC1900200B
:10A3D000041D002009232DE9F04F324C85B065683B
:10A3E00024688646039530480294304FDFF8C090C9
:10A3F000DFF8C0A01A44009137E006784FEA430C1A
:10A400003EF91350002E36D039F913B0FC5CA5EBA1
:10A410000B010191029988460399002C18BF8846C8
:10A4200044460199E4B20029B8BF49428C422ADD72
:10A43000009931F913803AF91310A8EB0108B8F12B
:10A44000000FB8BFC8F1000844451CDD34462EF8A3
:10A4500013B03AF90C50009921F81350013B591CE4
:10A4600000F8014902F1FF3219D01478002CC4D150
:10A47000DC551478F2E7009929F8135031F913509C
:10A480002AF81350EAE7009929F80C5031F91340E3
:10A490004FF00101F9542AF80C401478DEE705B0BA
:10A4A000BDE8F08F98170020051A0020041D002039
:10A4B00098190020C019002030B40546044C0068EB
:10A4C0006968AA68EB680FC42869206030BC7047CF
:10A4D000A0170020014B1878704700BF0E1D002008
:10A4E0004FF0000C2DE9F04FE0464FF06409334F78
:10A4F00085B002923A69D7E901EA0192FA680392BB
:10A5000010F1FF3044D33A78002AF9D033F91040E3
:10A51000744544DD0E9D35F9105055453FDD4FF033
:10A52000010694460F9D2E547A78002AE8D0109A9E
:10A5300052F82060C6F307255FFA86FBC6F3074290
:10A54000A5EB0B05C2EB1662013501329542B5BF92
:10A5500009FB05F509FB02F295FBF2F292FBF5F21D
:10A56000019DAC42CCDD51F82040029DA4F5007461
:10A57000A4B2B4F5804F55F8205014D9039C9442EE
:10A58000BEDD4FF001040F9A145410F1FF30BAD21F
:10A5900060460B4B83F800C005B0BDE8F08F0F9A02
:10A5A00002F80080C0E7A5F50075ADB2B5F5E05F33
:10A5B000A6D9039C9442E4DCA2E700BFA0170020C8
:10A5C0000E1D00202DE9F04FC3F307461C0E8BB083
:10A5D000A642DDF85090DDE917E856DC06FB09FCE1
:10A5E00012B2A2EB46220292621CDDB209920AB2BA
:10A5F000079505926544159AC3F307276B1ED31878
:10A600000193169B089703EB4C0C4FEA4903013763
:10A610000693079B08998B422ADC029A019D002A27
:10A62000B8BF5242039204E08A0631D40133BB42E0
:10A630001ED015F8011F8142F6D13CF91340002CC1
:10A64000F4DD059AA2EB432181EAE172A2EBE1720B
:10A65000DEF80010013304FB0211CEF80010D8F828
:10A6600000200399BB4201FB0422C8F80020E0D17E
:10A67000069B01369C44019B4B440193029BA3F52E
:10A6800000730293099B9E42C3D10BB0BDE8F08FCB
:10A690000022159C01F00F0104EB030B049341FA17
:10A6A00002F4E3070BD5094C094B145712F903A028
:10A6B000344409FB04B414F80A40A04204D0013227
:10A6C000042AECD1049BB1E7049BB6E754A801002F
:10A6D0005CA80100F0B404460F46124E00F1300CA5
:10A6E000354620686168A268E3681034644506F165
:10A6F00010060FC5F4D13D46206861680A4F03C6B5
:10A7000005F130063C4628686968AA68EB68103590
:10A71000B54207F110070FC4F4D12868696803C770
:10A72000F0BC7047101D0020481D00202DE9F04F9F
:10A73000824693B01F46BDF98C30840007939DF884
:10A74000903088469146002122461C9806930FF0CF
:10A750006EF822461D9800210FF069F8BAF1000F3B
:10A7600072DD0024DFF898B102E00134A2456BD01D
:10A7700037F91430002BF8DD0025229E1E9B12A80D
:10A7800053F8243059F8242058F8241040F8245D58
:10A790000296219E04900196209E08A803900096A0
:10A7A00020460895FFF70EFFDDE9083237F914104F
:10A7B00093FBF1F392FBF1F11C9A42F824301D9BBC
:10A7C00043F82410069B012B41D058F82400594629
:10A7D000C0F30800B0F5807FC8BFC0F5007001F07D
:10A7E000B3F9064659F824004349C0F30800B0F510
:10A7F000807FC8BFC0F5007001F0A6F91D9B05461B
:10A8000053F824101C9B53F8240001F047F9DBF89F
:10A810002C3083424BDC4020064637F914C0DDE97A
:10A82000082302FB06F603FB00F34FEA8C1C96FBA1
:10A83000FCF693FBFCF31C9A42F824601D9A42F844
:10A8400024300134A24593D113B0BDE8F08F1C9B96
:10A8500058F8242053F8240059F82430C2F3080291
:10A86000C3F30803B2F5807FC8BFC2F50072B3F529
:10A87000807FC8BFC3F50073CDE90B010D920E9325
:10A880000A9401F00BF90022012104230F901B48C8
:10A8900037F91450079ECDE90220CDE90031082296
:10A8A0000AAB6420CDE91065F8F7BEFA5DE7DBF886
:10A8B0002830079A37F914C09A4202DC4020064635
:10A8C000ADE7C6F14003DBE90C12604600930023BC
:10A8D00001F0CEF8084B37F914C0D3E90C12C5F1DA
:10A8E0004003009306440023604601F0C1F837F9A5
:10A8F00014C0284493E700BF481D002060A8010051
:10A90000101D00202DE9F047002688B01C1EDDE94F
:10A910001087C8F800603E604FDD8A46169D08AB80
:10A9200043F8046D0295159D0DF1180C0195149DC9
:10A93000CDE903C30095129B91460696FFF742FEB0
:10A940001F4ECAF30800B0F5807FC8BFC0F5007085
:10A95000314601F0F9F8DFF86CA0C0F14003316B2B
:10A96000DAF83420054600932046002301F080F8F1
:10A97000C9F30809B9F5807FC8BFC9F50079054456
:10A980001049484601F0E0F8DAE90C12C0F1400342
:10A99000064600932046002301F06AF8DDE906230D
:10A9A000304403FB00F302FB05F0A40193FBF4F336
:10A9B00090FBF4F4C8F800403B6008B0BDE8F087B5
:10A9C000101D0020481D0020F0B40446094E00F17F
:10A9D0003007354620686168A268E3681034BC42DD
:10A9E00006F110060FC5F4D120686168A26807C699
:10A9F000F0BC7047B41700202DE9F84F061E33DD78
:10AA0000994690460F4600244FF0640B174DDFF82F
:10AA100060A002E00134A64226D015F8011B0029EF
:10AA2000F8D0134938F9140001F08EF8DAF8303014
:10AA300037F9141003FB00F00BFB01F139F814E0B7
:10AA40008142DAF828100BFB0EFE01FB03F1B4BFC4
:10AA5000002001208E45B8BF00220A9B1855B8BFC0
:10AA60001A550134A642D8D1BDE8F88F202900201C
:10AA7000B41700202DE9F84F071E2FDDDFF860B076
:10AA80009D1E0A9B941E4FF06408D94604EB4707AD
:10AA90008E1E03F1FF3A0BE001FB00F008FB03F30D
:10AAA0008342B4BF00200120BC420AF8010F15D038
:10AAB000494634F9020F01F047F8DBE90A3135F86D
:10AAC00002CF03FB01F208FB0CFC944536F9023F70
:10AAD000E2DA0020BC420AF8010FE9D1BDE8F88FA4
:10AAE000B417002000283BDD2DE9F043002637464F
:10AAF0008C1E04EB4008951E34F902EF35F902CFA5
:10AB00007745B8BF77466645B8BF66464445F3D13A
:10AB100000254FF06408A946124CD4E90DC404FB8B
:10AB200006F60CFB07F7079C013C04EB000E14F83B
:10AB3000010F78B131F915C008FB0CFCBC4505DBF1
:10AB400032F9150008FB00F0B04203DA84F80090F7
:10AB500003F80590A64505F10105E8D1BDE8F083AD
:10AB6000704700BFB4170020034610B4034C596867
:10AB70009A680068DB680FC410BC7047F0170020AB
:10AB80000023F0B4344A354D354C3648364F3749FA
:10AB9000C2E90033364EC2E902331361C5E900331E
:10ABA000344AC5E902332B61C4E90033324DC4E9AC
:10ABB00002332361314CC0E90033C0E90233036141
:10ABC0003B602F487B603B81C1E90033C1E9023320
:10ABD0000B61C2E900332B49C2E90233C6E90033F5
:10ABE00013613381284A294EC5E90033C5E9023390
:10ABF0002B612360264D6360A360E3602361254CD5
:10AC0000036043608360C36003610B6022484B6054
:10AC10008B60CB600B611360204953609360D360FD
:10AC2000136133601E4A736033812B60C4E90033C3
:10AC30006B602B81036043608360C36003610B60C2
:10AC40004B608B60CB600B6123811360536093601A
:10AC5000D3601361F0BC7047D41D0020E81D0020B4
:10AC6000101E0020C01D002020290020FC1D0020F7
:10AC7000941D0020AC1D0020801D00200C31002000
:10AC8000702A0020F8300020E02900202C27002026
:10AC90009C2A0020A01D0020E0300020C4270020B6
:10ACA000142700202DE9F04F440004F108058BB073
:10ACB000824625F00705073020F0070000AFADEB16
:10ACC000050D6E46ADEB000D6846FD6FF961E91D9F
:10ACD00021F00701ADEB010DBA61002152467B6105
:10ACE000BE60D7E920B378607B620EF0A0FD2A46F3
:10ACF0004FF0FF3168460EF09AFD2246796F3046DC
:10AD0000C7F810D00EF088FDBAF1000F7B6A67DD3E
:10AD1000BA6E002602F1FF3909EB0A027A6203E0FB
:10AD20007A6A013691455BD019F8011F0029F7D0E6
:10AD30007A6F002D32F916A0604A516801EB4A0A79
:10AD4000EEDD4FF0FF323A62D7F88C20C7F80C9056
:10AD50000024A2F10208994602E00134A54220D065
:10AD600038F9022F002AF8D03B6F59F8241033F934
:10AD700016C0FB6E5BF8242033F91600A1EB0C0122
:10AD8000101A00F08BFE4DF2502303FB00F000146C
:10AD90005045B8BF3C6204F10104B8BF8246A542E9
:10ADA000DED13A6A4B46511CD7F80C90B8D03969BD
:10ADB00089564A1C78D0BA6832F911008245AFDA58
:10ADC00000244FF0010C22F816A0386A3A69165494
:10ADD0007A68545402F806C07A6A01369145A3D1C4
:10ADE000002D5DDDD7E9246CD7E926E80022104666
:10ADF0003969013D0D444C1E7D6214F9011F4D1C43
:10AE00004AD05BF8225053F82290AA46FD6925F8F3
:10AE100011A0BD6925F81190D7F888501CF8029050
:10AE200035F812A07D6925F811A0D7F88C5035F9B6
:10AE300012A03D6D25F811A036F912A07D6D25F800
:10AE400011A0BD6D05F801901EF80290FD6D05F88A
:10AE50000190BD6F6A54D7F8A05035F912903D6E3D
:10AE6000AA4658F822504AF821507D6E25F81190D4
:10AE70004BF82200D7F8881043F8220021F812007E
:10AE8000D7F88C1021F8120026F812000CF80200F6
:10AE90000EF8020048F82200796A0132A142ACD1D2
:10AEA0002C37BD46BDE8F08F0121BA68386A22F818
:10AEB00016A03A6916547A68915531E7F0170020C8
:10AEC0002DE9F04F04469FB00AAFD7F890B0F96271
:10AED0000BF1070121F00701ADEB010D0AA9F960A3
:10AEE000BA6208465A464FF0FF317B600EF09FFC75
:10AEF000E31D23F00703ADEB030D0DF1280A2246F5
:10AF0000504600210EF093FC002293457A6452DDF6
:10AF1000BE6FC7F834A004E07A6C01325A457A64F7
:10AF200047DAD7F8A03033F91230002BF4DD0023D4
:10AF3000D7F8D0209C42C7E912237A6C40F3E08115
:10AF40004FF0FF3804E0FB6C0133A342FB6424DACA
:10AF500036F913100029F6DDF86AB96A31F91310D1
:10AF600030F91330D7F8980050F82250D7F89400F1
:10AF7000691A50F82200C01A00F090FD4DF25023DB
:10AF800003FB00F3BA6C1B149A4200F38081FB6C44
:10AF90007A6C0133A342FB64DADB4FFA88F30121B8
:10AFA000F868835401327B6B5A4503F808107A64C1
:10AFB000B7DBD7F834A0002C40F39E81D7F87C9003
:10AFC000013C0AEB04034FF000083B610AF1FF3A31
:10AFD000C7F8309008E03B6B08F1010802333B638F
:10AFE0003B699A4500F088811AF8013F002BF2D0A6
:10AFF000BB6FBBF1000F33F91890FB6AC7F84490A0
:10B0000033F91820BB6A09FB02FE33F918C07B68CC
:10B0100009FB0CFC33F81810D7F8843009FB01F158
:10B0200013F808303B62D7F8803013F808307B62A1
:10B03000D7F8CC3013F80830FB61D7F8883053F8D4
:10B04000285040F36181002472466046FB68C7F8CF
:10B0500008A05E1ED7F894A007F14C03BB617E6385
:10B060007E6B16F9013F43457E6340F0AE80D7F812
:10B070009860D7F8A03056F8246033F914307E6118
:10B080005AF82460994406FB03227E69C7F844906D
:10B0900006FB0300C7E90E202A46D7F89C6036F865
:10B0A00014C003FB0C11D7F8B0305FFA85FC53F8DD
:10B0B000243039645FFA83FEC3F30720F445C5F3F7
:10B0C000072188BF6EF30702C5F3074C8142C3F323
:10B0D000074138BF60F30F221B0E8C4588BF61F318
:10B0E0001742B3EB156F88BF63F31F6294465FFA94
:10B0F00082F9F14588BF6EF3070CC2F3072E86452F
:10B1000038BF60F30F2CC2F30740884288BF61F359
:10B11000174C1546B3EB126FD7F8C82088BF63F3FE
:10B120001F6C0992D7F8C42007F13C030892D7F8A6
:10B13000C02021460792D7F8BC200692D7F8B82045
:10B140000592D7F8B0200492BA69039207F144023D
:10B15000029207F14002CDE90032F86907F13803A5
:10B160005A46C7F84CC0FDF7DDFBD7F88430396A82
:10B170001A5D00239142B8BF1146D7F8A8207E6A15
:10B180003962115D4AF824300E437E62D7F8986028
:10B19000BA6B46F82430D7F89C60D7F8449026F86C
:10B1A0001430D7F8A060F86B26F81430D7F8A460F4
:10B1B000396C26F81430D7F8A8603355D7F8AC604E
:10B1C0003355D7F8B06046F824300134A3457FF4F6
:10B1D00047AF96468446D7F808A09EFBF9F69CFB3D
:10B1E000F9FC91FBF9F4D7F8C8300FFA89F9069306
:10B1F000D7F8C43007F148010593D7F8C03062464C
:10B200000493D7F8BC30F869CDE90253BB690091CB
:10B21000019331464B46C7E90E6C3C64FFF772FB65
:10B22000D7E9120100F03AFC662301224FF0000E2C
:10B230004FF0020C00B203FB00F33549386B9B1250
:10B240000391038011460346CDE9012ECDF800C0DD
:10B250007420F7F7E9FDBB6F23F81890FB6A23F819
:10B260001860BB6A23F81840D7F880301A4697F860
:10B27000243002F80830D7F884301A4697F8203086
:10B2800002F80830D7F8883043F82850A3E64FF08A
:10B29000000A01254FF0040952461E496D20BB6487
:10B2A000D7F84C80F7F70CFE1B4B2A46CDE902A3DA
:10B2B000294607F144030195CDF800906420F7F783
:10B2C000B3FD164B2A460393294607F14C03CDE9FB
:10B2D000015ACDF800906420F7F7A6FD104BCDE998
:10B2E000015A0393CDF800902A46294607F14803F6
:10B2F0006420F7F799FD4AE65437BD46BDE8F08F64
:10B300004FF0FF3398464AE607F14C03BB6164E710
:10B310008CA801006CA8010078A801007CA801009D
:10B3200080A801002DE9F04FB0F1000A91B0DDF8DE
:10B3300068B06BDD16460D4600245F460D9337F965
:10B340001430002B5FDD4FF0FF3B4FF00009DDF8BC
:10B350009C804C4513D037F91930002B0FDD56F87F
:10B36000241056F8292055F8240055F82930891A58
:10B37000C01A00F093FB4045BCBF8046CB4609F1A4
:10B380000109CA45E5D1BBF1FF3F3CD0259B5246A0
:10B390000A93249B59460993239B20460893229B9A
:10B3A0000793219B0693209B05931E9B04931D9B53
:10B3B000CDE902730D9BCDE900632B46FDF7E4FB5D
:10B3C000A34526DD259B1E9837F914C056F8242086
:10B3D00055F8241050F824000693249B02900593FE
:10B3E000239B0EA80493229B009003930FAB019321
:10B3F00020466346FFF786FADDE90E0100F04EFBBA
:10B400001B9B23F814000134A24598D111B0BDE86C
:10B41000F08F259B1E9837F91BC056F82B2055F846
:10B420002B1050F82B000693249B02900593239B2E
:10B430000EA80493229B009003930FAB01935846F0
:10B440006346FFF75FFADDE90E0100F027FB1B9B67
:10B4500023F81B00D7E700BF2DE9F04FB0F1000B38
:10B4600083B0DDE913C9DDF86CA0DDF8748050DD30
:10B4700000264FF0FF34DFF8A0E0019302E0013630
:10B48000B34546D01EF806000028F8D1013408EB79
:10B490000400019B02E00134A4453ADD077805462B
:10B4A0000130002FF7D06445019332DA159859F82E
:10B4B000247050F8240021F8167022F8160016980F
:10B4C00030F814701998005D23F81670179F0C9BC4
:10B4D00037F9147023F81670189B33F914700D9B0C
:10B4E00023F816700E9B98551A9B185D0F9B985564
:10B4F0001C9B28785AF8247033F91450109B43F899
:10B500002670119B23F81650129B98550136B345AF
:10B51000B8D103B0BDE8F08F202900202DE9F04F0D
:10B5200099464FF01F3304469DB018AFC7E9013369
:10B53000BB81BB6BCDE90B410E46391DD7F840A04E
:10B540000F930A91FB6B396FCDE9103A05917B6C33
:10B55000F96E12930491BB6CB96E13930391FB6C5B
:10B56000796EDFF8A0E1DFF8A0C114930D92BB6DF6
:10B570009046CDF838907A6D0291396E5F4801910E
:10B58000CDE908CEF96DDFF884C10091CDE906C0A0
:10B59000396D0A20FFF786FB594AD7F88C00D2E9AB
:10B5A000023200210092642200F062FA002860D08A
:10B5B000BB6F002B5DD0D7F88430002B59D0834669
:10B5C0003D1D3B6F1595D7F8885005931495FB6E7C
:10B5D000D7F8845004931395BB6ED7F8805003932B
:10B5E00012957B6EFD6F029311953B6EBD6F0193BB
:10B5F0001095FB6DFD6C0093396DD7E91523CDE9EE
:10B6000007680694CDF858B00F95BD6C0A200E95CA
:10B610007D6CCDE90CA5FD6B0B95BD6BCDE9099556
:10B62000FFF74EFCD7F88C301BB300233A1D0C9269
:10B63000D7F8882006930B92D7F884204B460A92BD
:10B64000D7F8802031460992FA6F20460892BA6FE7
:10B65000CDF834B00792FA6C0592BA6C04927A6C09
:10B66000CDE902A2FA6B0192BA6B00924246FFF753
:10B6700059FEE31D23F00703ADEB030D002C0DF184
:10B68000600C11DDBB6B0DF15F011D469A1E02EBD4
:10B69000440032F9023F002BD4BF00230123824231
:10B6A00001F8013FF5D1BD63FB6B07940C93BB6BB5
:10B6B000FC6CCDE90A937B6F109406933B6FBC6CD6
:10B6C0000593FB6E0F940493BB6E7C6C03937B6EAF
:10B6D000396D02933B6E0A200193FB6DCDF844C097
:10B6E0000093D7E91523CDF834A0CDE908680E946E
:10B6F000FFF7B2FE1437BD46BDE8F08FFC1D0020F9
:10B70000F0170020801D0020101E0020202900209E
:10B710002DE9F04F4FF0000883B08246894601932F
:10B7200044460F9D574E584ADFF878B12BE000236E
:10B730002354002963D13AF91430544F22F81430BD
:10B7400039F91400524927F814003AF91400514B02
:10B750002BF8140039F91400371921F81400019955
:10B76000287831F9141023F814100E9B33F91410B3
:10B77000494B387023F8141008F1010801340A2CE1
:10B7800005F1010537D02B78311900914348315D1F
:10B79000002BCCD14148DFF8F8C0DFF80CE10029DC
:10B7A000ECD0215C3BF81470013149B2DEF800E0C6
:10B7B000215422F814703CF81400344F714527F8D6
:10B7C0001400DBDD31192CF814303548DFF8C4C023
:10B7D0000B70314922F8143027F814302BF814304C
:10B7E00020F814302CF8143021F8143001340A2CCD
:10B7F00005F10105C7D1404603B0BDE8F08F234FE6
:10B8000032F9143039F914C037F914103AF9140028
:10B81000ACEB0101C01A009200F040F9204B3BF95B
:10B8200014C023F814003AF91430009AA3EB0C0C5E
:10B83000174903EB6C0322F8143039F9143031F94D
:10B8400014C01448A3EB0C0C03EB6C0327F8143062
:10B850003AF9143095F800C02BF8143039F9143047
:10B8600021F81430019B311933F9143081F800C0EC
:10B8700020F814300E9B33F91410074B23F81410E2
:10B880007AE700BF20290020FC1D0020101E0020A8
:10B89000E81D0020C01D0020AC1D0020941D0020CC
:10B8A000801D0020D41D0020F01700202DE9F04F4E
:10B8B0004FF0000983B0CDE9001298465F4D604B10
:10B8C000824695E8070003C34C460E9EDFF89CB104
:10B8D0001A803BE000215A4F9E42DFF880E1DFF8FA
:10B8E00084C15848584A395565DB3AF91430574FE6
:10B8F000A15CEB53009B564F33F91430EB533AF9EC
:10B900001430544F25F80B30009B33F9143025F8D0
:10B910000E30019B33F914E04F4B25F80CE038F959
:10B9200014C027F805C00C9F17F804C004F800C025
:10B93000385D814238BF0146A1540D9A32F9142076
:10B94000EA5209F1010901340A2C30D038F91420E7
:10B95000404BB2424FEA440533F91430BADC9E4200
:10B960003E4A3F49EFDA364F35F80B003B5D096838
:10B9700001335BB23B55354F35F802C0E8533448CC
:10B980008B4225F800C0DEDD00233649AB526B52F6
:10B990002C4A2D492B52A3542E482F4A635401346C
:10B9A0000A2C25F80B30EB534353AB52CED148460B
:10B9B00003B0BDE8F08F264B009FEA5E234B37F9BA
:10B9C0001410EB5E3AF91400891AC01A00F066F8F8
:10B9D000254B35F90B1058533AF914301F4A591AB0
:10B9E00003EB61031949A85E6B5237F914301D4906
:10B9F000181A03EB600316482B523AF91430114819
:10BA000025F80B3037F91430124FAB52019B0E4A18
:10BA100033F914306B5238F91410A35C79530C9934
:10BA2000095D21540C99085D0B49834238BF0346D8
:10BA3000A3540D9B33F914306B5282E7941D002000
:10BA4000A01D00209C2A00202C270020E030002090
:10BA5000C4270020E029002014270020F83000200F
:10BA6000F01700200C310020801D0020702A0020DB
:10BA7000884210DB904210B40ADA441A0198521A34
:10BA8000C01A04FB00F494FBF2F210BCD01870470B
:10BA9000019810BC70471846704700BF81EAE173F7
:10BAA000A3EBE17318B30028B8BF4042F1B198424C
:10BAB0001FDA820192FBF3F2402AA8BF402211490B
:10BAC0008A5CC2F15A028AB10F4910B4C2F15A0419
:10BAD00031F8122031F8141003FB02F300FB01F0DF
:10BAE0001B1403EB2043184610BC7047034618464E
:10BAF00070479A0192FBF0F2402AA8BF4022014908
:10BB00008A5CE0E770A90100B4A9010088420ADB61
:10BB100040B1890191FBF0F04028A8BF4020094BBB
:10BB2000185C7047704751B1800190FBF1F14029DA
:10BB3000A8BF4021034B595CC1F15A007047084629
:10BB4000704700BF70A9010070B40E680C89022E06
:10BB500025DDA04223DB0B460125013E02E08442A5
:10BB600006DC15466A1C96429C8903F10403F6D153
:10BB700001EB8505AE88ED88A6420DD001EB820170
:10BB8000CB88001B5D1B00FB05F0A41B90FBF4F4AD
:10BB90001C4420B270BC704728B270BC70470025AE
:10BBA0000122E5E77F280CDC402824DA0F2824DC7A
:10BBB000082827DA022829DB0428B4BF0120022044
:10BBC0007047B0F5806F08DAB0F5007F1CDAB0F589
:10BBD000807FB4BF072008207047B0F5805F05DA8A
:10BBE000B0F5006FACBF0B200A207047B0F5005FC6
:10BBF0000CDA0C207047062070472028B4BF0420C0
:10BC000005207047032070470920704700207047C7
:10BC10002DE9F04F056887B0144665B12C4E2D4DC7
:10BC2000314600226020F7F74BF92246294664206E
:10BC3000F7F746F9F4E7284A074613680846013340
:10BC4000884613600DF0D8FD386020B1234B00EB1F
:10BC500008029A422CD90025DFF888B0DFF888A0C6
:10BC6000DFF88890494600226420F7F729F9042676
:10BC700001223868114600EB080C04AB0490CDE9B2
:10BC8000025B019500966420CDF814C0F7F7CCF85C
:10BC9000012200961146CDE9025A019505AB6420B8
:10BCA000F7F7C2F8002221466420F7F709F9D9E72F
:10BCB0000B4A2B46114602E00133322B05D051F8D6
:10BCC000044B002CF8D142F8230007B0BDE8F08FF8
:10BCD00020A9010024A90100EC1E00200C3E002038
:10BCE000241E002058A9010064A9010044A90100F4
:10BCF0002DE9F04D0746006886B08846B8B1244D5E
:10BD000000232A4602E00133322B18D052F8041BDC
:10BD10008142F8D1002445F823400DF075FD1D4AFD
:10BD20003C601368013B136006B0BDE8F08D0A4625
:10BD300064201949F7F7C4F806B0BDE8F08D002477
:10BD4000DFF85CB0DFF85CA0144E314600226420BE
:10BD5000F7F7B6F8042501223B6811460593CDE9B3
:10BD6000024B05ABCDE900546420F7F75DF841467E
:10BD700000226420F7F7A4F80A220095CDE9024AD0
:10BD800001941146024B0020F7F74EF8DDE700BFA3
:10BD9000241E0020EC1E0020C4A80100E4A801001D
:10BDA00068A901000CA901000D4B1B68002B15DDD3
:10BDB00070B500260B4D0C4C84B021460022642047
:10BDC000F7F77EF801220423CDE902650093019282
:10BDD0001146034B6420F7F727F8EEE7704700BFE2
:10BDE000EC1E002088AA01006CAA010010B50446D0
:10BDF000FCF744FD04F1F00104F1B800FEF76AFC21
:10BE000004F59470FBF778FF04F5EC70FBF712FC77
:10BE100004F5EE70FEF750FB04F5F870FCF778FCC3
:10BE200004F51770FEF7D0FD04F52670FEF79CFEB2
:10BE300004F52A70FCF71CFD04F2813002F0ECF8E6
:10BE400004F2AE20FCF704FD94F8AE320BB9FCF717
:10BE500005FD04F52C70FCF72FFB04F54170FBF792
:10BE600077FD04F55E70FEF78DFA04F5617001F060
:10BE70003DF80023044C194623604FF48862BDE866
:10BE8000104002480DF0D3BCE4190020902C002093
:10BE900038B9064A136801338B4205DD1060012072
:10BEA000704700231846014A13607047E4190020C8
:10BEB00008B5FBF743FCFEF76DFAFEF761FEFCF7F1
:10BEC000CDFCFCF701FBFBF74BFDBDE8084002F0A1
:10BED0009BB800BF0022014B1A607047F01E002083
:10BEE000024A136801331360704700BFF01E002040
:10BEF000014B1868704700BFF01E00202DE9F04F7D
:10BF00000024DDE90A67A246A646A14640F6FD7870
:10BF1000DDF830C0013E16F8015FBDB131F814B054
:10BF2000ABF5007BBBF5406F10D232F814B00BF1CB
:10BF3000FF3B1FFA8BFBC34508D833F91490F1453A
:10BF400058DDCE46A946099D35F914A001340A2CC6
:10BF5000E1D100263546A7F1020807F23E474146E7
:10BF6000002205E0262B00D901350132222A0AD011
:10BF700031F8023F062A03F113039BB2F2DC262BB1
:10BF8000F3D90136F0E708F144084745E7D1002727
:10BF9000ACF102030CF10A0C33F9022F9C45174453
:10BFA000FAD100220D9B0D99023301F11A0C33F9DD
:10BFB000021F9C450A44FAD143F698230E9949681A
:10BFC000994213D8B32D11DC4A2E0FDCA0B1B9F180
:10BFD000000F1FD0BEEBEA0F1CDD114A1368032BC4
:10BFE00005DC013313602046BDE8F08F0B242046AA
:10BFF000BDE8F08FA946A9E7952F02DD962AA8BFD4
:10C000000B24074B1A68002AF1D0002220461A6040
:10C01000BDE8F08F0022024B20461A60BDE8F08F89
:10C02000081F0020024B0A201978FEF7DFB800BF76
:10C0300014090020002001220249034B08601A70F5
:10C04000704700BFFC1E0020F41E0020014B187832
:10C05000704700BFF41E002019B10E4B1860FFF7A7
:10C06000E1BF0C4B30B41C680B4D84422A680DD0E4
:10C070000A2C14BF28210221914203DD01322A60DB
:10C0800030BC704730BC1860FFF7CCBF02B12960EC
:10C0900030BC704714090020F81E002070B586B02F
:10C0A0000C9CDDE90A56029401960F9C0E9E0095A9
:10C0B0000D9DCDE9046403950E4D2C68FFF71EFF1E
:10C0C00001210D4AE31782FB0462C3EBA20303EBD9
:10C0D00083030A4AA4EB430301FA03F311680A2815
:10C0E00014BF0B4321EA0303013413602C6006B034
:10C0F00070BD00BFFC1E002067666666041F00203E
:10C10000034B18680028D4BF00200120704700BFEF
:10C11000041F00202DE9F04FDFF84CA187B09AF8FA
:10C120000040169E002C35D0B42404FB06F4484D84
:10C13000DFF8388185FB045BE417D8F80050C4EBC6
:10C14000AB14AC4249DA434C074624688C460A2CAF
:10C150009646994621D14FEA460B0BEB0604A542C1
:10C160001BDB06EB8606B5EB860F3B4E02DA346826
:10C17000A3454ADC0021394B39481A6801238A4219
:10C18000D4BF00220122013502708AF80010C8F8DD
:10C190000050336007B0BDE8F08F159B61460593F2
:10C1A000149B72460493139B38460393129B2A4EAA
:10C1B0000293119B0193109B00934B46FFF79EFE49
:10C1C0000021FFF749FF0123D8F800500135C8F8D6
:10C1D0000050336007B0BDE8F08F159E0596149EA1
:10C1E0000496139E0396129E0296119E0196109E2F
:10C1F0000096FFF783FE1B4AAC42136840EA030037
:10C2000010601ED00123144EE0E7159C0594149C89
:10C210000494139C0394129C0294119C0194109C0E
:10C220000094FFF76BFE0B2808BF00234FF00001BE
:10C2300008BF3360FFF710FF3368D8F800500133B0
:10C24000C4E7044B1860FFF7EDFED8F80050D9E7BB
:10C25000D34D621014090020001F0020041F00208D
:10C26000F51E002018090020F41E0020FC1E0020EE
:10C27000014B1878704700BFF51E002038B50D4CF3
:10C2800030B123680A2B03D00A232360FFF7CAFECC
:10C2900000230A220849094D0B60094809492B600F
:10C2A00003600B60084D094809492B700370226038
:10C2B0000A6038BD14090020F81E0020041F002069
:10C2C000001F0020FC1E0020F51E0020F41E002090
:10C2D000180900206E20704738B500240B4B0C4D18
:10C2E00021464FF42A72C3E90044C3E90244C3E97A
:10C2F000044408482C600DF09AFA2146BDE8384005
:10C300004FF4A07204480DF092BA00BF1C23002025
:10C31000141F0020181F0020C02100202DE9F04F1D
:10C3200000279A460D4695B00BAC0DF11C088146CE
:10C3300016463946222220460797C8E90177C8F8F1
:10C340000C700DF074FA4FEAAA034D4A142BB8BFD3
:10C350001423BD42C2E90077C2E9027717616CDDA0
:10C36000C446C9EBC9714900CDE901774FEA490ECE
:10C370000091691E0597049706EB0E0208EB050A6B
:10C380000391B9F1000F16DD00210098ACEB080B0A
:10C39000101830F9025B9D4207DD9CF800700E5DBD
:10C3A000013701368CF800700E55212937DD904297
:10C3B00001F10101EDD10CF1010CD4457244E0D141
:10C3C000019B002B58D1059A9DF82C609DF81C30DC
:10C3D000002A4DD1002528462F4629460DF11D0281
:10C3E0000BB1012528448B42C4BF19460127944252
:10C3F00002D012F8013BF3E7002F36D195BB0021A4
:10C400000B460DF131020EB101210B44944202D0D2
:10C4100014F8016FF7E711BB15B0BDE8F08F029E6D
:10C42000BBF1000F2E44029604DD039E5E4501DD44
:10C4300005290BDD01250195B9E700253B463E4660
:10C4400028462F4629460DF11D02C9E7049F012603
:10C45000AF42B8BF2F46059604970196A7E7084A52
:10C460009360D9E7064B1860C9E7054B5960C5E7EB
:10C47000034A04991161ADE7014B029ADA60A2E721
:10C48000002300202DE9F04F95B000AF7B61D7F875
:10C4900094300028BB60D7F89830C7E90621D7E967
:10C4A0001ECED7E92C51D7F8B8407B60386240F3F4
:10C4B0007D819146DFF83083C44ED8F800204000DB
:10C4C00002EB021206EB8202A9F10203B246F86007
:10C4D000023A1E1833F9020F9E4222F8020FF9D1D8
:10C4E00023683B61FB69002B17DD7B69D8F800806E
:10C4F0009E1E3346B64AF86902EB481206EB40002E
:10C50000023A33F9028F834222F8028FF9D13B6A53
:10C51000002B40F36D81AD4B9A460022C7F8B8401E
:10C5200047F6FF765446C7F8B410DFF8C082B96901
:10C530007A6200234FEA420B786A04EB0B09C3448A
:10C5400039F944ABCB455344FAD182467862A148CD
:10C5500080FB0309DB17C3EBA9031BB2002B21F8F7
:10C560001230994602DD5046184478629E42A8BFB8
:10C570001E469C450CDAB5F808902B6809F10109B4
:10C58000A5F8089031F91290A9EB0C0A53442B60DE
:10C59000CE450CDDB5F80A906B6809F10109A5F8E4
:10C5A0000A9031F91290A9EB0E094B446B60022AF4
:10C5B00040F32D813B6A01329342BADCD7E92D1456
:10C5C0003A69AE811546844B786A83FB0553A3EB29
:10C5D000E2732360E3683A6A3B61FB6990FBF2F027
:10C5E000002B40F3EE807B699E1E6FF001054FF03B
:10C5F000000E47F6FF7CFB69754A03EB0508C7F898
:10C600002480D7F80490D7F808807861104600237A
:10C6100002F5A07B30F920AB83455344FAD16D4835
:10C6200080FB03A0DB17C3EBA0031BB29E45B8BF82
:10C630009E469C45A8BF9C46434526F8023F09DD1F
:10C640000B89086801330B81B6F90030A3EB080AA7
:10C6500050440860994509DD4B89486801334B8196
:10C66000B6F90030A3EB090A504448600B2D23EAC9
:10C67000E37000F291803B69013503443B61E36064
:10C680007B6A0232AB42C1D178690FFA8EFE0FFA93
:10C690008CFCFD68A1F80EC02B46083323F007037D
:10C6A000ADEB030DFB69A1F80CE0A3F1040C3B6AB0
:10C6B0006946002B38DDBB6900269A1E154440F2FE
:10C6C0004458A946A1F1020E32F902AF256AAAEB3D
:10C6D000000323EAE3731BB2AAF1970AAB421FFAE5
:10C6E0008AFAC8BFC4E90763C2452EF8023F06F1C3
:10C6F000010602D8A3690133A3619145E4D1B1F9E0
:10C700000030002B10DDA36A3A6A1A441046013348
:10C7100004E031F9022F002A40F39C8098421D4624
:10C7200003F10103F5D1A06247F6FF703B690326D0
:10C73000984293FBFCF1B8BF18460023274AC7E98B
:10C740000E33C7E91033C7E91233254D254BA160DD
:10C7500000B207F12801C7E90C23C7E90A65FFF712
:10C76000F3F9E2686369012A1146B8BF01219B0110
:10C7700093FBF1F323EAE373984209DAE369B342E6
:10C7800006DD41F287339A4202DC012384F824302B
:10C790005437BD46BDE8F08F6369013503446361DA
:10C7A0007B6A0232AB427FF431AF6DE723683B61B5
:10C7B000FB69002B3CDD3B6ADFF82C805B00FB60F3
:10C7C00093E647F6FF7C4FF0000E62E7181F00204B
:10C7D000C02100206766666656555555E80340003F
:10C7E000F4013200D0074000141F0020C0210020B7
:10C7F00047F6FF72AA813A69174B104683FB000384
:10C80000A3EBE2732360E36800203B61EDE631F9BE
:10C8100012903869D7F8B830B9F1000FA8BF484472
:10C820005B6838619944D7F8B830C3E90009C1E6BC
:10C8300047F6FF70FA69084BA2F1040C3A69A88127
:10C8400083FB0263E068A3EBE273044A2360386170
:10C85000CA6069E7A56267E7565555550000FF7F36
:10C860000020A2F1040C2DE9F047E046064647F609
:10C87000FF77DFF858E1DFF858918D1E10605060A7
:10C880009060D0601061043135F9023F002B3ADD31
:10C8900098B2441E092C39D81C461E449E45B8BF88
:10C8A0009E469F42A8BF1F468D4248F8044FEBD1D9
:10C8B0004348BEF57A7FC1791CDA012F3B46B8BFE9
:10C8C00001231BB29EFBF3F3052B13DD91B93D4D04
:10C8D0000E4602F108015CF8043F312B06DD85FBB2
:10C8E0000374DB17C3EBA403CCF8003061451E448E
:10C8F000F1D1C179344B116183FB0613A3EBE673CD
:10C90000D360BDE8F08700242346C7E7A0F10B04FD
:10C91000092C11D9A0F1150ABAF1090F1C4612D839
:10C9200003EB43035B00A9FB0303DB0803339BB268
:10C930001C461BB22644B1E75B10053398B204468F
:10C9400003B20644AAE7A0F11F0ABAF1090F0ED9F3
:10C95000A0F1290ABAF1090F11D8DB00A9FB0303E2
:10C96000DB08043B9BB21C461BB2264496E7C3EB94
:10C97000C303A9FB0334E408264423B28EE7A0F1E5
:10C98000330ABAF1090F04D93D3827280CD91E44BF
:10C9900084E703EBC303A9FB0303DB08093B9BB25A
:10C9A0001C461BB2264479E7C3EBC3035B00A9FB1B
:10C9B0000303DB08263B9BB21C461BB226446DE7F3
:10C9C0001C23002067666666565555550080FFFF9C
:10C9D000CDCCCCCC84B02DE9F0470024814609A809
:10C9E00080E80E003D4D9DF848603D4FDFF8148112
:10C9F000DFF814A115F8013BABB90F9B122B02DC39
:10CA0000B9F1000F28D00EB3002236494920F6F7BD
:10CA100057FA002305F8053C0134042CEAD1BDE89F
:10CA2000F04704B0704707EB4403099A1B899A4208
:10CA30004FF0000202DD0B9B1E2B29DC41464920F2
:10CA4000F6F73EFA002305F8053CE5E732462649AD
:10CA50004920F6F735FADFE74A4624494920F6F738
:10CA60002FFA109B062BD7DD7EBB0E9BB3F57A7F8A
:10CA700025DD139B052B22DC119BB3F5FA7F1EDA13
:10CA800032461B494920F6F71BFA05F8056CC3E747
:10CA900051464920F6F714FA012305F8053C46B142
:10CAA000002214494920F6F70BFA002305F8053C4B
:10CAB000B2E7324610494920F6F702FAACE7002205
:10CAC0000E494920F6F7FCF9A6E74A460C494920E9
:10CAD000F6F7F6F905F8059C9EE700BF2023002035
:10CAE00098AA01006CAB0100A8AB0100C0AA01002C
:10CAF00010AB0100F8AB010028AC010034AB010021
:10CB0000E8AA010038AC0100DCAB010082B010B42F
:10CB100001A981E80C00DDE90234012B18D0A0B195
:10CB2000511001EB4201994202DCD11E032907D9C1
:10CB3000023B032B09D8012C07DD023A042A04D852
:10CB40000022074B5A709A70DA7010BC02B070471E
:10CB5000042AE4DC0022024B5A709A70DA70F4E77F
:10CB60001C23002030B400250124104B181D1A7915
:10CB700019786AB979B1597A0131C9B20A29597259
:10CB800001D91C715A7201338342F0D130BC704715
:10CB900019B15D73F7E75972F5E75A7B0132D2B2EA
:10CBA0000A2A5A7384BF19715973ECE71C230020B9
:10CBB00084B030B49DF8484002AD85E80F00002CE9
:10CBC00031D0109BB3F5FA5F14DD2E4A13680133A0
:10CBD000052B36DD052101231160002201202A4D9D
:10CBE0002A4C2B492A6022602A4A087030BC1372F2
:10CBF00004B07047119B642BE7DC254803781BBB0E
:10CC0000244A9179D3790B4335D01F491D480B68CD
:10CC10000133052BC8BF05230B6000231B490360AC
:10CC20000B600223E2E7194B174A1C6002231460D1
:10CC300017481449174A04700C60137230BC04B0D2
:10CC4000704713600223C8E71E241049114A0B687D
:10CC500001330B609C42BABF00230C6002234FF0EB
:10CC60000001B8BF0370074C07482160016030BC69
:10CC7000137204B0704705490B240B6801330B6035
:10CC8000E8E700BF14230020342300200C1F0020FD
:10CC9000182300201C23002000212DE9F0473B4FE2
:10CCA00092463A46994601250B468EB09DF8A080E3
:10CCB000189E1A9C364842F8041B12F8011B31B921
:10CCC00030F813108E4202DD1E2CC8BFFD54013314
:10CCD000042BF2D16C461BAD0FCD0FC495E80F00AD
:10CCE00084E80F0018AD95E80E004846FFF772FE85
:10CCF00025AB93E807008DE8070023AC94E80C000F
:10CD000049465046FFF702FF00234FF0010C42F264
:10CD1000107026994BB3032B32D05A1C042A01D031
:10CD20000133F7E740F2DC539E4206DC43F69823DA
:10CD30009942CCBF01230023BB706E4607AFFFF7BB
:10CD400011FF0FCCCDF830800FC723681CAC3B60BF
:10CD50000FCC0FC694E8070086E8070095E80F009F
:10CD6000FFF726FF0EB0BDE8F08797F800E001223C
:10CD7000BEF1000FD4D18142C8BF07F803C0CDE790
:10CD8000FA78002ACED10422F5E700BF1C23002048
:10CD900098AA0100034B187AA0F10100B0FA80F0C4
:10CDA000400970471C23002020B90C4B9A7952B1DE
:10CDB0000320704701280FD1084B1B7A002B14BFAA
:10CDC0000420052070475A790AB10220704718796B
:10CDD000003018BF01207047002070471C2300203E
:10CDE0002DE9F04FA3B00025DDE93C876E46814672
:10CDF0008B4617AC149220462C2200219DF800A1EE
:10CE000015930CF014FDCDE90F74CDF838800DF1B9
:10CE1000D40C0DF11C0EBCE80F00AEE80F009CE82E
:10CE200007008EE807000DF1B80CBCE80F00C8F849
:10CE30000050C8F80450C8F80850C8F80C50C8F89A
:10CE400010503D607D60BD60FD603D610FC69CE897
:10CE500007002D9B86E8070059462C9A4846194E34
:10CE6000FFF710FB0DAFCDF848A00FCE0FC7366807
:10CE70000FCC3E6002AE0FC60FCC0FC694E8070081
:10CE8000159B86E807002D990F4C01912C99149A57
:10CE9000009148465946FFF7FFFE23682C9901335D
:10CEA0000A2B18BF1D4648463E9A2560FFF7D8FC5E
:10CEB0003E9B3F9ADB6850469382FFF775FF23B095
:10CEC000BDE8F08F00230020141F002030B9064B6E
:10CED000187810B10138C0B2187070471423024A94
:10CEE00018461370704700BF101F002001464FF412
:10CEF000A67201480CF090BC00180020014B187875
:10CF0000704700BF5D2300202DE9F04F0026B9B027
:10CF1000CDE90A23894B8A4C1E708A4D8A4B8B4A75
:10CF20008B49266082464B9C0DA81E602E601660C1
:10CF30000E60FCF7FBFC3146882216A80CF077FC4B
:10CF400004F10F0009902F68B346304621257E4B2F
:10CF50007E4A7B4C1268D3F800807E4B7C49049259
:10CF600093F902302268CDE90666D1F800E0089610
:10CF7000059202930DF1DC09774B4FEA450C03EB68
:10CF80000C02A3F588639C44CDF804C0099C844638
:10CF90001DE04FF0010B9E44D844CDF818B0052D8C
:10CFA000A2F144020FD00298591D83420BDA207877
:10CFB0000CF1010C0390D9F8000001440398C9F862
:10CFC00000101F2817D0019B013C9A421DD0B2F9D6
:10CFD000FC33534504BF2F4601260A2BD9DC13F13D
:10CFE0000A0FDCDA012007900498013004900598BC
:10CFF00018440590D3E74A980028E4DD0898013CDE
:10D000001844019B08909A42E1D1013D6B1C604697
:10D01000A9F10409B0D1079B002B75D1069B002B09
:10D0200040F08780BBF1000F02D0494BC3F800E00D
:10D030000EB1444B1F60474B22229988B3F906601A
:10D04000B3F90840429F212314E007EB4202B2F8F3
:10D0500056205AB18A4209D238AA02EB830252F80A
:10D06000882CB24202DA089AA24212DC5D1E8BB111
:10D070001A462B46052BE8D1B7F86030002B4AD072
:10D080008B4248D21A9B9E4245DD089A0423A24255
:10D09000ECDD01230A9AB2F57A6F48D9429A118BD6
:10D0A0005A2994BF0021012140F2EE22429C248E95
:10D0B00094423AD9429CB4F84C40944294BF002226
:10D0C0000122012B2AD1429C248B142C26D91E2804
:10D0D00024DD0B98052821DD01BBFAB99DF83A1033
:10D0E00001F0FF00D1B91B491C4C0D7813494C9E2F
:10D0F0000B70216835448D42D3BF18460131216041
:10D10000226039B0BDE8F08F104B049A1A600C4BC6
:10D11000059A1A6082E704230325A9E7002318462D
:10D120000E4A136039B0BDE8F08F0022C9E7002134
:10D13000BAE7054BC3F8008074E700BF4423002022
:10D140004C23002058230020502300204823002097
:10D150005423002000180020902C002038230020A9
:10D16000F0B58DB0BDF954509DF890609DF8947065
:10D17000C0B9B9B93D4C2178C9B1132A55DC139A0D
:10D18000632A52DC133350DB129B092B4DD8384BEA
:10D19000384AD9691368994260DD01210B44136054
:10D1A000217024E00022314B1A700DB0F0BD23999C
:10D1B000104609912199CDE90A67089120990791B4
:10D1C0001F9906911D9905911C99CDE903511B9951
:10D1D00002911A9901911E9900911946DDE91223D5
:10D1E000FFF792FE207010B12348FAF723FAFCF7FC
:10D1F00059FE2478054624B3204C214E23883278EA
:10D2000001331BB22380002ACFD1632BCDDD1D4B10
:10D210001B78002BC9D002210920FCF7E7FF01236E
:10D220006422AB7733702280BFE7114B1399B3F9B7
:10D2300018209142ACDC002201210E4B21701A60B3
:10D24000D5E70F4E0D4A33781480002BADD0032163
:10D250000920FCF7CBFFAC773470A6E700230A481F
:10D2600013602370FAF7E6F9C1E700BF5D230020E1
:10D27000001800204023002004D101005E2300207C
:10D280005C2300204423002008CF0100054A92F8C7
:10D290004E30834204DA8B42B4BF00200120704735
:10D2A00001207047001800203228CCBF0020012048
:10D2B000704700BF2DE9F04F91B004460E4602932F
:10D2C000FCF7E4FD012801D0002C4BD000232124E1
:10D2D0009E4698469B469946184619461F469A46CA
:10D2E0009C46CA4ACA4D1360CA4A1360CA4A1360B0
:10D2F000CA4A1360CA4A136005F5886207E04FF016
:10D30000010A0CF1010C1F44443AAA4212D0B2F9AE
:10D31000FC33B34204BF214601200A2BEFDC13F19A
:10D320000A0FF1DA4FF0010E443AAA42F346F144F3
:10D330009844ECD1013C631CA2F10205DCD1BAF1A6
:10D34000000F40F0D381002840F0D681BBF1000FE0
:10D3500002D0B14BC3F80090BEF1000F02D0B04B29
:10D36000C3F80080029991F8295091F8283091F87B
:10D370002B805B1B05EB6305032D2A46A8BF032208
:10D38000039391F82A3052B2A3EB080308EB630829
:10D39000B8F11E0F049300F3BD800C2D00F3C6807E
:10D3A000B8F1020F4FF0030C00F324810121634612
:10D3B000AA4205F1FF3405F1010740F3C2800023C2
:10D3C00000933C2E1CDD914B1A9A1B6832F91330E6
:10D3D000012BB8BF012396FBF3F3022B10DD8E4B1C
:10D3E00090481B68C3EB431203EB820380FB0320CE
:10D3F000884ADB171268C3EB6013934200F3248161
:10D400000023019300290CBF04230323BC4205938E
:10D4100000F3108100200446DFF814A205EB051C80
:10D4200008EB4C0CAAF1480E08F1FF3B0EEB4C0E3A
:10D4300008F10109CB450BDC03223AF91C700EEB15
:10D44000000131F9023F013AA3EB07031C44F8D174
:10D450004430CC28EED1C4F100090FFA89F902F06A
:10D46000B9FA072809DD029AB2F924301146772B60
:10D4700003DC136A142B00F203810027242200210D
:10D4800007A80CF0D4F94FF4C87164234FF4167256
:10D490004FF4BE7E40F27D1C4FF0050B4FF0C80AE2
:10D4A000ADF82610484606A9ADF81E30ADF820307C
:10D4B000ADF82230CDF818B0ADF824A0ADF828E0D2
:10D4C000ADF82A20ADF82E20ADF82CC0FEF73CFBBD
:10D4D000554BB3F90A30B3420BDA7C2E09DC1A9BA8
:10D4E00033F91830312B00F3C080049A062A40F239
:10D4F000DB80019B13B9002F00F0A0804B4A1E99DE
:10D5000013688B427BDB012700233846136011B080
:10D51000BDE8F08FC8F121030C2D5BB264DC032B56
:10D5200000F0DD804FF0030C012141E7C5F10F0C45
:10D53000B8F1020F4FFA8CFC5CDC032301216C1E56
:10D540006F1CCCF11000A8427FF739AFB8F1030F80
:10D55000C646A8BF4FF0030EC6453FF730AFC3F134
:10D56000220040457FF72BAFAA1AAC4462453FF733
:10D5700026AF0020DFF8B89003EB080B009002EB19
:10D5800002130CF10100059009EB830008F101037F
:10D59000A8EB0E0A08F1FF3C0BF1010E0193D345F5
:10D5A0001BDBC1465346A8460CE0019D9D420BDBA8
:10D5B00030F91350093502DA009D01350095013329
:10D5C000734508D06345F0DAA242F8DBBA42EFDDDA
:10D5D00001337345F6D14546C846059B01329A4250
:10D5E00000F14400DBD1ECE6C5F10F0C032B4FFA40
:10D5F0008CFCA3D1022D6BDC03230121D8E600278C
:10D6000038460133136011B0BDE8F08F5823002075
:10D61000922800205023002048230020542300207B
:10D620004C2300201F85EB51E40D00203C230020FB
:10D63000902C00204FF000094C4610E73846304B44
:10D640001F6011B0BDE8F08F2E4B2F481B6800689B
:10D65000002BB8BF5B42B0EB430FBFF6D1AE092A37
:10D66000D4BF002301230193CCE61B9A32F9152085
:10D67000272A3FF73EAF049A062A3FF63AAF13E057
:10D68000536992686433B3EB520F7FF6F6AECB8BDF
:10D69000502B7FF6F2AE40F6B7331B4A17689F4215
:10D6A000CCBF00270127E9E6039A062A3FF621AFFF
:10D6B000009A05998A42FFF61CAF643404DA029A94
:10D6C00052688242FFF41AAF002B3FF712AF15E702
:10D6D0000322BCEB020118BF0121134668E6022DAC
:10D6E000CABF002101211A469C4661E6074BC3F8D8
:10D6F00000C0054B1F6026E6054B196026E600BFFB
:10D700003C2300204C2300205423002050230020E1
:10D71000582300202DE9F04F013883B000280191F3
:10D720006CDD012872D04FF000094FF0010C09EBBD
:10D73000000303EBD3735B1032F9131032F910407E
:10D740004500A14204DD22F813400C4622F81010D7
:10D7500032F919104FEA490BA14202EB0B0A04DD22
:10D7600022F81940515332F9191032F913408C4202
:10D7700005DD22F8131022F80B4032F9134006465B
:10D780000BF10201555E02EB4C0E22F8135054527D
:10D7900032F90B503EF9028F0CF1010CA845F9DB70
:10D7A000711E02EB410301E00E4601391F4633F9B9
:10D7B0000249AC42F8DC8C4507DCAEF80040A7F823
:10D7C00000800E46BAF90050E4E7019B22F80B40B6
:10D7D0008B423D8018DBE14616DD48450EDD09F140
:10D7E000010C8445A3D102EB49094000B9F900308E
:10D7F000115E8B42C4BFA9F800101352019B32F98D
:10D80000130003B0BDE8F08FB01EE6E7914602209A
:10D81000ECE700BF2DE9F04F013800EBD07383B087
:10D820005B10002801936CDD012872D04FF00009D5
:10D830004FF0010C09EB000303EBD3735B1031F9DC
:10D84000132031F910404500A24204DD21F81340B5
:10D85000144621F8102031F919204FEA490BA24251
:10D8600001EB0B0A04DD21F819404A5331F9192064
:10D8700031F91340944205DD21F8132021F80B40C3
:10D8800031F9134006460BF102028D5E01EB4C0E9E
:10D8900021F813508C5231F90B503EF9028F0CF1E4
:10D8A000010CA845F9DB721E01EB420301E01646AC
:10D8B000013A1F4633F90249AC42F8DC944507DCD3
:10D8C000AEF80040A7F800801646BAF90050E4E729
:10D8D000019B21F80B4093423D8018DBE14616DDA9
:10D8E00048450EDD09F1010C8445A3D101EB49093E
:10D8F0004000B9F900300A5E9342C4BFA9F8002085
:10D900000B52019B31F9130003B0BDE8F08FB01E3C
:10D91000E6E789460220ECE7831A042B10B413DDF6
:10D92000DC1EB1F90430002A0B804B8031F9143031
:10D9300008DD4000A0EB42020A44014421F8023D08
:10D940008A42FBD110BC70475C1E032C08BF9C1E92
:10D95000E7E700BFF0B40446049E0846DDE9055140
:10D96000A642DDF81CC019DD04F10044AF1E013CE5
:10D9700007EB460705EB44058E1C06E09C42B8BF4A
:10D980001C46BD4226F8024F08D035F9024F94429A
:10D99000F4DD1446BD4226F8024FF6D1F0BC6246D3
:10D9A000FFF7BABFF0B400280F46DDE90561DDF8E6
:10D9B0001CC014DB013006EB40048D1C06E09842CD
:10D9C000B8BF1846B44225F8020F08D034F9020D4A
:10D9D0009042F4DD1046B44225F8020FF6D13846E5
:10D9E000F0BC6246FFF798BF2DE9F043B1F9009013
:10D9F00002284FEA4918DDE90767C2E90088DDE936
:10DA000009CE21DD8C1E5B0176017F01043204EB1F
:10DA10004000023103E0A84631F9029C0432B1F91A
:10DA20000050B1F9024006FB05F503FB04541568EC
:10DA300002310CFB054407FB094408FB0E448142FC
:10DA40004FEAA4245460E6D1BDE8F0832DE9F0410B
:10DA5000884684B04C00083404AFBD6B24F0070442
:10DA6000ADEB040DBE690395FD6904AC019500960C
:10DA700002947D6BFFF76EFF3B6B21460293FB6ABE
:10DA800003950193BB6A40460093D7E90823FFF74B
:10DA9000ABFFBD46BDE8F0812DE9F041884684B07A
:10DAA0004C00083404AFBD6B24F00704ADEB040D4B
:10DAB000BE690395FD6904AC0195009602947D6BE7
:10DAC000FFF770FF3B6B21460293FB6A03950193BE
:10DAD000BB6A40460093D7E90823FFF785FFBD46A0
:10DAE000BDE8F0812DE9F04F8FB00AAF7D6D9A4609
:10DAF0001B1A023300F103088B465919FB6B18EB14
:10DB0000050804461646FB6000F0AA804FEA880923
:10DB1000002934D109F10A0929F00709C7F808D00A
:10DB2000ADEB090D08953E6D0DF128090796FE6CC9
:10DB300013460696BE6C5A4605967E6C4146049680
:10DB40003E6C0396BE6BCDF80890CDE900A6FFF7BA
:10DB5000A3FF002C0DDBFE680235013409EB8509BB
:10DB600006EB440459F8043B5B1124F8023DA6423D
:10DB7000F8D1D7F808D01437BD46BDE8F08F8B0038
:10DB80000A3323F00703C7F804D0ADEB030D089563
:10DB90003A6D0AAB0792FA6C09F10A090692BA6C5F
:10DBA00029F0070905927A6C04923A6C0392BA6BD9
:10DBB000CDE900A2BB605A4602933346FFF746FF09
:10DBC000ADEB090D0895396D0DF128090791F96C38
:10DBD00033460691B96C5A460591796C20460491FA
:10DBE000396C0391B96BCDF80890CDE900A141469D
:10DBF000FFF752FF631C9A4511DDFE68BA68E91C05
:10DC0000B31E02EB810103EB4A0A06EB440251F812
:10DC1000043B5B1122F8023F5245F8D1FE60002C14
:10DC20000DDDFE68E91C09EB810106EB440251F8A9
:10DC3000043B5B1122F8023D9642F8D1FE60BB68BE
:10DC4000023559F8252053F825301344FA689B1102
:10DC500022F81430D7F804D01437BD46BDE8F08F51
:10DC60008B000A3323F00703E946ADEB030D08955B
:10DC70003E6D0DF128080796FE6C13460696BE6CA5
:10DC80005A4605967E6C04963E6C0396BE6BCDF8A4
:10DC90000880CDE900A6FFF7D9FE544512DAFA68EC
:10DCA00004F10044013C0335931E02EB440608EBEB
:10DCB000850803EB4A0A58F8043B5B1126F8023F3B
:10DCC000B245F8D1CD461437BD46BDE8F08F00BF50
:10DCD0002DE9F04788B099464FEA430808F1080457
:10DCE00024F0070408AFADEB040DD7E90D563C6BEB
:10DCF000CDE90656BD6AFE6A059403953C6A7D6AC5
:10DD0000049608AECDE901650094FD6BFFF7EAFECD
:10DD1000B9F1000F10DD023CA044A6F1020A34F96B
:10DD2000023F3AF9022F9B1AAB42CCBF5B1B03EABE
:10DD3000E37344452380F2D1BD46BDE8F08700BFC0
:10DD400070B40024254601F58866B1F90630B1F9B2
:10DD50000800002BB8BF5B420028B8BF4042834296
:10DD6000B8BF034644310A2BC4BFED1801348E42BC
:10DD7000EBD100231846194609E01C2BC8BF32F925
:10DD8000136003F10103C8BF8019222B07D0042BB5
:10DD9000F3DC32F913600133222B3144F7D1072C25
:10DDA00001DD782D02DC70BC002070472829FADDE7
:10DDB00070BC0128B8BF012091FBF0F10229D4BF4B
:10DDC00000200120704700BFF0B50D4685B0074622
:10DDD0001B49642014460022F5F772F80026012240
:10DDE000042118482B460091039011466420CDE988
:10DDF0000166F5F719F80120134AE91B490900905B
:10DE00000392CDE901663B4620226420F5F70CF829
:10DE1000294651F8043BA342FBD000220124C5F15E
:10DE20001F030A481944CDE90122039049092B46F2
:10DE3000009420226420F4F7F7FF05B0F0BD00BF86
:10DE400064AC010078AC010084AC01009CAC010022
:10DE50000B68934209D070B50D461446064622461B
:10DE600029463046FFF7B0FFF9E770472DE9F0414A
:10DE700000258CB00790081A2E46049309952B466E
:10DE8000CDE905218410129D06E00133B4EB830F28
:10DE90004FF00106C0F28A8051F80429AA42F4D05A
:10DEA000002E40F09E8000274FF0040801224E4BC8
:10DEB000861B1146CDE901770393642007ABCDF8AB
:10DEC00000800A96F4F7B0FF01221446474B484EF3
:10DED0001146CDE901770393642006ABCDF80080AD
:10DEE000F4F7A2FF224621460297CDE9008409AB50
:10DEF00064200396F4F798FF3E4BCDE90147224694
:10DF000021460393CDF800800AAB6420F4F78CFF20
:10DF1000049C3946A446059C0997A4EB0C07BF1046
:10DF2000ACF104020B4605E00133B7EB830F4FF071
:10DF3000010147DB52F8040FA842F5D000294DD16A
:10DF40000025042701222C4BA4EB0C04C1EBA404F4
:10DF50000393114605ABCDE90155009764200B945E
:10DF6000F4F762FF01221446244B11460393CDE9D6
:10DF7000015504AB00976420F4F756FF09AB224625
:10DF8000214602950097039601946420F4F74CFF14
:10DF90001B4BCDE9014503930097224621460BAB6D
:10DFA0006420F4F741FF0CB0BDE8F081642000224A
:10DFB00014490993F4F784FFDDE90640099B201A10
:10DFC0009E0070E70F49002264200993F4F778FF60
:10DFD0000999059C8900DDF810C0B1E70993990003
:10DFE000AEE709939E005EE7BCAC0100C8AC01003F
:10DFF00078A80100D4AC0100E8AC0100F4AC010049
:10E0000000AD0100B0AC01000022024BC3E90022C8
:10E010001A817047D82300200278014B1A7070478C
:10E020004C190020314B1B78002B5AD02DE9F04FB2
:10E0300016462F4A87B08946804600242D4F136824
:10E04000DFF8B4B0DFF8B4A0013E14E03D5D38F96C
:10E050001410022D2BF8101005F1010E39F91410CF
:10E060009CBF5FFA8EF53D55032D2AF8101017D08E
:10E0700001340A2C0CD04FEA440C0CEB0401C818F4
:10E0800016F8011F0029E1D1395501340A2CF2D1CB
:10E090000133022BC8BF0023136007B0BDE8F08F27
:10E0A0000CEB04035B000BEB030108685344029084
:10E0B0001868B1F804C09B88049002A92846019210
:10E0C000ADF81430ADF80CC0FFF7A4FB04A928F894
:10E0D00014002846FFF79EFB019A29F814001368E4
:10E0E000C6E7044AC2E90033138170474C19002087
:10E0F000E4230020D8230020602300209C2300205C
:10E10000F0B483000A3323F00703002800AFADEB1F
:10E11000030D30DD6B4600260439B20002F1804267
:10E1200092F880C292F8815292F8824292F8832249
:10E130005FFA8CFCEDB2E4B2D2B2013683F800C0D3
:10E140005D709C70DA70BCF1000F03D00CF1FF3CE5
:10E1500083F800C0202D9CBF01355D700CB1013CDF
:10E160009C700E2A9CBF0132DA7053F8042BB04227
:10E1700041F8042FD1D1BD46F0BC704792F822304F
:10E18000002B39D1F0B5002889B00E46054614465B
:10E190000FDD936942189A420FDB00231A4684F878
:10E1A0002130237D93429CBF012384F8203009B0A5
:10E1B000F0BDF2D1D3698B42EFDD94F8213000221B
:10E1C000013384F821300D496420F4F779FE0020F2
:10E1D0000121042202900A4B94F821706420CDE9B9
:10E1E00000210393032205AB069607950597F4F7E4
:10E1F0001BFE94F82120D4E7704700BF20AD01003A
:10E2000048AD01002DE9F04F98468BB0DDE914537D
:10E21000012DA946B8BF4FF00109012B9C464FF0D4
:10E220000004B8BF4FF0010C169E07923788B6F86D
:10E2300004E01268D8F8006005FB072503FB0E66B2
:10E24000002895FBF9F596FBFCF6CDE908442ADD9C
:10E25000A446A146A246023901EB40000694CEF145
:10E26000000B059031F9023F5A1B22EAE272334457
:10E2700003EAE37397420EEB030403DC0120D21B95
:10E28000069092445B4505DC4FF0010C002CB8BFB2
:10E290006442A144059B9942E4D1069B002B3AD1EC
:10E2A000BCF1000F3AD1012400260425079F1D4B25
:10E2B000224621460393CDE901463B460095642062
:10E2C000F4F7B2FD184B224621460393CDE90146EF
:10E2D000434600956420F4F7A7FD144B22462146DF
:10E2E0000393CDE9014608AB00956420F4F79CFD4B
:10E2F0000F4B22460393CDE9014609AB0095214619
:10E300006420F4F791FDDDE908233A60C8F8003095
:10E310000BB0BDE8F08FCDF820A0C1E7CDF8249078
:10E32000C1E700BF58AD010068AD010078AD010044
:10E330008CAD010070B19A4215DC0F4A1368C72BEF
:10E3400001DC013313600D4B187808B181F0010036
:10E3500019707047084B1A68C72AF4DD1860074B1C
:10E360000120197070470022034B1A60034B187884
:10E370000028EDD0EAE700BFF423002002240020AB
:10E3800078B1187870B16FF4D2700144B1F5B85F0C
:10E3900007D843F2F661A2F5DC728A429CBF0022E4
:10E3A0001A70704741F6A600D239814204D843F66C
:10E3B000B001DB3A8A42F4D901221A70704700BFDB
:10E3C00030B108785AB1022808D801300870704777
:10E3D00023B10B78022B9CBF01330B707047002BCD
:10E3E000F1D10028FAD00138087070472DE9F04FBC
:10E3F000C64DADF2EC4DDDF8304517932B7832A8C1
:10E400001A93231C18BF0123CDE918121B930DF199
:10E41000EC09FBF78BFA1E22002122A80BF007FA69
:10E420000DF5607A3C22002148460BF000FA782274
:10E43000002150460BF0FBF91E2200212AA80BF008
:10E44000F6F93C2200214AA80BF0F1F959A83C2228
:10E4500000210BF0ECF90023DDF83005CDE91D3388
:10E46000CDE91F332193002840F0E7824FF02208C6
:10E470001027DDF82835A4AA0793DDF82C3586A9E6
:10E4800006932AABCDE90093C2AB0393CDF808A065
:10E490004AABCDE90478F8F761FF0123002400932B
:10E4A0009B4B4246394603936C20DDF82C35CDE971
:10E4B0000144F4F7B9FCC2AB0493DDF82835DDF86C
:10E4C00030050893DDF82C35A4AA079359ABCDE9A4
:10E4D00002A32AABCDE9009386A94AABCDE9057822
:10E4E000FAF768FCC2AB0493DDF82835DDF8300597
:10E4F0000893DDF82C35A4AA079359ABCDE902A304
:10E500002AABCDE9009386A94AABCDE90578FAF7A5
:10E5100095FDC2AB0493DDF82835DDF8300508938E
:10E52000DDF82C35A4AA079359ABCDE902A32AAB99
:10E53000CDE9009386A94AABFEAECDE90578FAF79E
:10E54000CBFB0DF58E652146782230460BF06FF936
:10E550002146782228460BF06AF96E4BDDF830052B
:10E560001A68DDF854355278B3F924300892DDF892
:10E57000282507930692DDF82C254B460592CDF809
:10E5800010800397CDE90065CDF808A0A4AA86A95C
:10E59000FCF7CCF8DDF830350DF5D07BA3420DDD6E
:10E5A0005F4655F8041B56F8040BFDF777FADDF8C3
:10E5B00030350134A34227F8020BF2DC1024222567
:10E5C000DDF85425DDF82815B2F924201846CDE9E8
:10E5D0000912DDF82C25CDE906450892C2AA05925C
:10E5E00059AACDE903A22AAACDE901B24AABA4AA4D
:10E5F00086A9CDF80090FAF7B5FE00230120214648
:10E60000434CCDE900032A46CDE902346C20DDF805
:10E610002C35F4F709FC9DF8D130DDF83005009376
:10E62000A4AA4B4686A9F9F7A1FBDDF8300500281E
:10E630000CDD5A4666240BEB4001B2F9003004FBB6
:10E6400003F39B1222F8023B8A42F6D122ABCDE9BA
:10E6500000B3A4AA4B4686A9CDF808A0FBF740FF5B
:10E66000FEF74CFC002840F072819DF8CE30002B64
:10E6700040F056811A9B012B04D19DF8E730002B06
:10E6800040F0F8810026DDF85C3577AC03F51770B3
:10E69000FCF79AF9DDF830352660B34200F35F816C
:10E6A0000126002504201C4B32463146009003937E
:10E6B0006D200DF5A663CDE90165F4F7B5FBDDF836
:10E6C0007075199A1597DDF8287507921497DDF87B
:10E6D0002C75189A1397C2AF1097DDF8187506922B
:10E6E0000F971DAF0E97DDF8207559AA0D97DDF82D
:10E6F0002475179B0C97DDF81C75CDE904A20B97C8
:10E70000DDF814752AAA0A9708E000BF541000200B
:10E71000A0AD0100A8060020D8AD0100DDF81075FD
:10E72000039222AADDF830054FF022080893CDE9C4
:10E7300001B2CDF80090099710274AAA134686A97E
:10E74000A4AACDF848801197FCF7E8FEBE48CDE9B1
:10E750000155039000966C2042463946DDF82C3571
:10E76000F4F762FBDDF83005A8422ADDDDF8142558
:10E77000179BA2F10208DDF81025B146AB46DFF881
:10E78000E8A2971E9E1E01E0A8421ADD38F9021F7A
:10E7900037F9023F36F8022F2560C4E9011301352D
:10E7A000E260002BF0D004224120CDE902BACDE98D
:10E7B000002923460121F4F737FBDDF83005A84294
:10E7C000E4DC14231DAA189DDDF864800192DDF8B5
:10E7D0002425414600920293DDF81425DDF810351A
:10E7E0002846FDF763F8179EDDF81835DDF8142587
:10E7F0000093DDF8101533460A20FCF73BF9DDF8ED
:10E800001835DDF814250093DDF8101533460A207D
:10E81000FCF7F2F8DDF81835DDF810250093DDF887
:10E820001415DDF81C350A20FCF75CF9DDF8183505
:10E83000324603931DAB0293DDF824354146019324
:10E84000DDF8143528460093DDF81035FCF760FF3D
:10E85000DDF810352A4600930A2143460020F8F7D8
:10E86000EFFE41462846DDF81825FFF7DBFBFEF7F3
:10E8700045FB1A9B2E46022B08BF40F00100C3B295
:10E880001793DDF8183506F11409704DDFF8DCA197
:10E890006F4F08F1140803F109061FE02A78317858
:10E8A0001CAB0094F9F7FCF81C9B2168B0F5C87FFD
:10E8B00017F801299BF80000C8BF0022A9F8003012
:10E8C000179BA8F800102946FFF77AFD16F80139C2
:10E8D000013D8AF800305F4B9D4277D039F9020D37
:10E8E00038F902CD014662463B461C903078C4F8A8
:10E8F00000C0FFF745FD584A1AF8013DA81AB34673
:10E9000033B9337823B13B7813B14FF003032B7045
:10E91000179B002BC2D04FF0000300222B70BEE7E4
:10E920009DF8CF30002B7FF4A5AE4A465946DDF85E
:10E930003005F9F701FFDDF87435187000283FF451
:10E94000A1AEDDF85C3503F50870FCF73DF877AC57
:10E950000026DDF830352660B3427FF7A1AEDFF840
:10E9600010810022414670200125F4F7A9FA042302
:10E9700002273A4A2946CDE9026200932A462346F5
:10E9800070200195F4F750FA2368354A2946CDE9FD
:10E9900002620BEB43032A46702001950097F4F7BF
:10E9A00043FA23682F4A09EB4303CDE90262CDE91C
:10E9B00000752A4629467020F4F736FA2368DDF8F8
:10E9C00030252B4493422360CBDB69E60024199E5B
:10E9D000189D9DF8CD30DDF818250293CDE900246F
:10E9E000DDF81435DDF8102531462846F8F7D6FE57
:10E9F000DDF8182531462846FBF7ECFC9DF8D130B0
:10EA00002946022B0CBF22460D22DDF81835019253
:10EA1000009432460A20F8F74DFEDDF818352846F6
:10EA20000093DDF81025DDF814353146F9F72EFD99
:10EA30001B980DF2EC4DBDE8F08F5146FFF760FBDF
:10EA4000DDF8300512E500BFA0AD01000D24002067
:10EA5000F1230020032400200424002078A80100D2
:10EA6000C0AD0100CCAD0100E4AD010002240020E6
:10EA7000A8AD01002422002178A80AF0D8FE1125B3
:10EA80001E2077ACFA214FF416724FF496774FF0B0
:10EA9000320C4FF03C0E2581A081642546200526CE
:10EAA0004FF028080223C4E90B50E781A4F810C0F6
:10EAB000A4F814E02046E18061816282E28226604F
:10EAC000C4F82880C4E90D33FBF77EFF40E700BFA0
:10EAD0002DE9F04FC7B2C0F3072883B04745019036
:10EAE0000C992BDC9DF806A052000AF100499DF814
:10EAF00007B009F1FF390AFB023301EB490901EBC9
:10EB00004B0C0D9908F1010801EB470EDA4518D8B6
:10EB100049461C460C4D34F9170031F9026F854205
:10EB2000B8BF05468642B8BF08808C451444F2D170
:10EB30002DB2013747452EF8025BE7D103B0BDE89F
:10EB4000F08F014DF5E700BF0080FFFF2DE9F04F8A
:10EB500005468FB04FEA410A08AF18463A6088462A
:10EB6000524600216C007B60D7F844900AF05FFEAB
:10EB70002246386C00210AF05AFE002D67DD0AF1AA
:10EB800008033E6C23F0070B4FEAA803FB603B68C9
:10EB90003119B9609C1EC7F814D0ADEB0B0D08AB52
:10EBA000A51C1846294652460AF036FEF968024668
:10EBB0004046FEF7AFFDB8F1000F014653DD0020DF
:10EBC0002246034632F902CF8C4508BF184601336E
:10EBD0009845F7D10522ADEB0B0D15234FF0290E0B
:10EBE00007926FF4247240F23E6CCDE903E3069283
:10EBF00008AA02930095CDF814C03A610192BD6C49
:10EC0000FA6C43468A1A2944FEF76CFF3B697A681E
:10EC10009D1E0AEB040134F9023F35F9020F1B1A5D
:10EC2000A3EB0903002B238006DD10889BB2184458
:10EC300010803088034433808C4202F10202EAD112
:10EC4000BB6802369E42D7F814D00C46A3D10023ED
:10EC50003A68C8EBC8084FEA48081C3722F8083061
:10EC6000BD46BDE8F08F6FF424724FF0050E1523FA
:10EC700040F23E6C2920ADEB0B0DCDE9062E08AA23
:10EC8000049302930095CDF814C003900192B86CE0
:10EC9000FA6C43468A1A01440020FEF723FF04EB76
:10ECA0000A01CDE72DE9F04F9FB08A0008AF7A61E5
:10ECB000083222F00702ADEB020DB8614E0008A841
:10ECC00000297963B860FE6119DD4FF4004E47F604
:10ECD000FF7C0025B11ED7F884200144D7F88C00B2
:10ECE000023A96190DF11E04023822F8025FB24270
:10ECF00021F802EF20F8025F24F802CFF5D1B969BC
:10ED0000786B4A0000FB02F2083222F00702ADEBFA
:10ED1000020D08AA00297A6040F3E3807A64002299
:10ED20003A6300EBD07222F00102043B0A32D7F8BA
:10ED30008010BB6322F007033B617B690439CB1869
:10ED4000F9603B653B69C7F82CD0ADEB030D08AA11
:10ED5000ADEB030D08ABBB647B6BFA64002B40F397
:10ED60003981D7F890200023013A144647F6FF79FD
:10ED70007A629046D7F88C209A46951E7A6CC7E93D
:10ED80000F33CB46FE68D7F838E0A2F1020C3C62A4
:10ED90000BE0FC6C4A4524F8130002DA0146814678
:10EDA000FB633A6D0133964221D056F8040F5EF8AA
:10EDB000042F35F8021FC2EBA0121144298018F865
:10EDC000014F10B2E4072CF8020F4946C7F854B0BF
:10EDD000DFD4BC6C5A4524F81A0003DA8346786500
:10EDE000C7F840A03A6D0AF1010A9642DDD1C7F892
:10EDF00028A015254FF0000B05266FF4247840F26B
:10EE00003E694FF0290AFA6C3C6A0092F86B643153
:10EE1000CDE9066B0395CDE9015A4FF00042CDE9EB
:10EE20000498FEF755FFCDE902A5CDE9066BCDE9C3
:10EE300004980195BE6C4FF000420096796DBB6A54
:10EE40006431386CFEF744FF796B7B6AFD6C0B44D0
:10EE5000594618467B6C14F8012F0233D2074BBF7A
:10EE600035F81B2036F811200BF1010B01318442DB
:10EE700023F8022CEFD17A6CF9693B6B0A447A646F
:10EE80007969BA6B01330A44BA63BA693B639A423F
:10EE9000D7F82CD07FF456AFD7E90C897A68FB6994
:10EEA000A2F1020CBA6800269E4692469D1E1544A9
:10EEB000B9F1000F11DD29466046AAF1020230F9CE
:10EEC000023F31F9024F9C42B8BF0B8032F9024F2A
:10EED0009C42C8BF1380AA42F1D101364645F44492
:10EEE000E6D17B6B002B71DDBB68D7F888109C1EC8
:10EEF0002646FA69881ED7F88C10A2F1020CD7F8C2
:10EF00001880023903EB0C0500EB020E35F8023FC6
:10EF100036F8022F9B1A20F8023F31F9023F704564
:10EF200093FBF8F30B80F1D1D7F88430991E0A4691
:10EF3000BB6803EB0C0534F9023F32F9020F002BDA
:10EF4000B8BF5B42984200DA1380A542F3D1BB6898
:10EF5000084663449C46FB690B441A463CF9023F51
:10EF600030F9024F002BB8BF5B429C42B8BF038010
:10EF70009042F3D16FF00044D7F890302646581EE7
:10EF80007B6B03449C46034604E09442A8BF1446AE
:10EF90009C450AD013F8015F31F9022FED07F4D434
:10EFA0009642A8BF16469C45F4D1D7F8842010F8A5
:10EFB000015F118815F0010FA1EB04050ABF891B41
:10EFC00015801180834202F10202F0D15C37BD4608
:10EFD000BDE8F08F0024152505266FF4247840F253
:10EFE0003E694FF0290AFB6C2046009307942346A4
:10EFF000CDE90586CDE90359CDE9015A4FF000422C
:10F0000048F26301FEF764FECDE90664CDE9049899
:10F01000CDE902A50195BB6C204600934FF000425C
:10F02000234648F26301FEF753FE24E7002824DD5F
:10F03000F0B400258E1EAC464FF0FF3700E01D46B1
:10F0400036F9024F6B1C944203DD6445C4BFA446ED
:10F050002F469842F3D17B1C11D07B0031F9170069
:10F060001FB1CA1832F9022C1044AF4203DA194416
:10F07000B1F902301844F0BC7047002070470020FE
:10F08000F0BC70472DE9F04F1D468046460006F162
:10F09000080A91B02AF0070A06AFADEB0A0DC7E9DE
:10F0A00002213B6D00927A6F06AC049301920B46ED
:10F0B0000395014602941A220220D7F858B0D7F8D7
:10F0C0006890FFF7EFFD7A6D796F4046FFF7AEFF6E
:10F0D0003B6EADEB0A0DB8F1000F18600DF1180A88
:10F0E00040F39080AAF102031946023DA81935F9B0
:10F0F000022F002AB8BF5242854221F8022FF6D1D2
:10F100005A46514640467B60FFF790FF00227B6ED7
:10F11000023E186010467B680AEB0605C9F800201D
:10F1200033F9022F934505DAD9F800101044013164
:10F13000C9F800109D42F3D1FB6E264418600023ED
:10F14000023C34F9022F9342B8BF1346A642F8D1CD
:10F1500001240426062100254FF0020B386F304AA7
:10F160000360BB68CDE90141039221464246009607
:10F170006220F3F759FE2B4AFB68CDE9025259464B
:10F180004246CDE900647220F3F74EFE264A53460C
:10F1900021460392CDE901454246CDF800B04E200C
:10F1A000F3F742FE21487B6F424621460390CDE9AA
:10F1B0000145CDF800B04E20F3F736FE2A461C4933
:10F1C0006E20F3F77DFE3A6E1A4B126821467A6183
:10F1D0007A6E6E201268BA61FA6E1268FA61D9F816
:10F1E00000203A623A6F126803937A6207F11403BF
:10F1F0000096CDE901450522F3F716FE2C37BD46F2
:10F20000BDE8F08F5A4651464046FFF70FFF0022F7
:10F210007B6EF96E1860C9F8002013460A6097E704
:10F22000FCAD010008AE010014AE01002CAE0100DF
:10F230003CAE010068AE01002DE9F04F8246164653
:10F24000524600258BB000AF8846386D5200002131
:10F250003C6E9946BB61C7F808A00AF0E8FA0AEBD1
:10F26000DA7323F001030A3323F00703ADEB030D38
:10F27000C7F820D0AA45ADEB030D2561C7F81CD017
:10F2800025606560A560E56084F811A0257440F3F1
:10F29000F980504647F6FF7E7A6DCC46013A7A6097
:10F2A0009246321F02EB80037B613B6DAB46714699
:10F2B000A8F10408A3F102097D623C6611E07345E0
:10F2C000A8BF7346D7E9084524F81500A8BF18461B
:10F2D0007C6A86467869013490427C620CF1010CAC
:10F2E00031D0B86952F8043F20B19CF8000000FB0F
:10F2F0000333DB1158F8040FBD6DC3EBA01347F6C1
:10F30000FF708342A8BF034661480E468342B8BFE0
:10F31000034618B229F8020F1AF8014F2C57002C97
:10F32000CDD18B42A8BF0B46FC691E4624F81B00BA
:10F33000A8BF184601467869734690420BF1010B4D
:10F340000CF1010CCDD1D7E918429342A8BF134666
:10F350009642A8BF16461BB2524236B29342B8BF7D
:10F3600013469642B8BF164632464FF0000C4FF097
:10F370000040FE60FE6D7968D6E900E9BE683B6139
:10F380000E44B346B7F9106012B27E61E0464E46B5
:10F3900063466FF00045BA617862D7F8509041E05B
:10F3A0003A6A786932F91820002A5ADB002802DB11
:10F3B0003869121A12B229F8132008F101087245AF
:10F3C00018DDB4F808A022680AF1010AA4F808A020
:10F3D00039F913A094F91100AAEB0E0A52442260E5
:10F3E00094F910209842C8BF63749A42B8BF23743E
:10F3F00039F9132096420ADD628960680132628120
:10F4000039F91320A2EB060A8244C4F804A0786AF2
:10F4100001339042B8BF10469542A8BF15468B45B0
:10F42000786227D011F8012FB86D8256002AB7D123
:10F43000FA69B86932F91C20002A09DB002802DBCE
:10F44000F868121A12B229F813200CF1010CB6E771
:10F450000028F5DA121A02EAE27212B229F8132031
:10F46000F3E70028A4DA121A02EAE27212B229F8CB
:10F470001320A2E72DB203B22C37A381E581BD464C
:10F48000BDE8F08F2B464FF000404FF0FF35F3E71B
:10F490000080FFFF2DE9F047824686B00620DDE9B7
:10F4A00012781C460E4691461425F5F7B1FBF5F788
:10F4B0003FFF159B31460493149B029003930F9BCF
:10F4C0004A46CDE9004305950E9B5046FFF7B4FE32
:10F4D0000025012102261548234603905246692043
:10F4E000CDE901150096F3F79FFCAA4528460EDDED
:10F4F000A31E03EB4A0A33F9021FCA1B002AC8BF26
:10F50000AD18B1EB080148BF40185345F3D1109B2B
:10F51000AB4207DB119B8342D4BF0020012006B021
:10F52000BDE8F087012006B0BDE8F087FCB001001F
:10F53000002820DDF0B48E1E06EB4006B14218D044
:10F54000571C38460B46B1F9004033F9025FAC4214
:10F5500007DD0D801C8092F9004090F90050157075
:10F560000470B34200F10100EDD10231B1423A46DC
:10F57000E6D1F0BC704770472DE9F04F804645005A
:10F5800005F1080485B000EBD07A24F007040730B9
:10F590002AF0010A00AF20F00700ADEB040D08F1DE
:10F5A000090424F00704EB46ADEB000D0AF10A0054
:10F5B00020F007006E46ADEB040D6C46ADEB000D80
:10F5C000E946C7E902210AF1020A08F102021F21F5
:10F5D00020467B600AF02BF95246484600210AF08B
:10F5E00026F9B8F1000F7B6807DD324606EB08000C
:10F5F000911B02F8011B8242FAD14FF0FF3A2A46D2
:10F60000F96858467B600AF007F959463246404689
:10F61000FFF78EFF023D08F1FF3E7B6806EB0E010F
:10F62000AB44013EB14218D03BF9025911F901290E
:10F630009D4202F1010C10DBA05C22441F2892784D
:10F6400060D01E2860D81E2A96BF4FF0FF3204F803
:10F650000C0004F80C20B142E6D1B8F1020F04F11D
:10F66000010113DD0B46FF20A64402E00133734580
:10F670000CD05A781F2AF9D11A781E2AF6D89A780F
:10F6800001331E2A98BF18707345F2D1B8F1000FEC
:10F690002EDDFB6804EB0806F96004E00134A642A5
:10F6A00003F1020323D06278FF2AF7D1257894F87A
:10F6B00002C039F8150039F81CE08346704528BFB0
:10F6C000F346B3F90020B96B0A449345E6DA704576
:10F6D00038BF7046013465458CBF29F81C0029F8F5
:10F6E0001500A6420AF1FF3A03F10203DBD1F968E3
:10F6F0004246B8680AF090F80AF101001437BD4696
:10F70000BDE8F08F1F2A06D01E2A88BF6FF069025D
:10F7100004F80C2086E70AF1010A04F80CA029F885
:10F720001A507FE7FFF728BF00487047700100209C
:10F73000024B1A680260187D704700BF70010020FC
:10F74000024B5A680260587D704700BF700100206C
:10F7500030B44FF0804300220F21212022251024B5
:10F7600083F8082183F80A2183F8090183F80B1133
:10F770001A739A735873D9731D725C72DA7793F89F
:10F78000211041F0010183F8211093F8211062F358
:10F79000410183F8211030BC704700BF10B44FF016
:10F7A000804485B00DF1100C0CE90F00BDF800305D
:10F7B0002382BDF802306382BDF90430A382BDF913
:10F7C0000630E382BDF808302383BDF80A30638336
:10F7D000BDF80C30A38305B010BC70474FF08043D8
:10F7E000988370474FF08043988B70474FF0804369
:10F7F00083F82000704700BF0123002110B50A4A9A
:10F800000A4C2377917210B94FF08042D3704FF0B9
:10F8100080430122987000211A700A2000F088F9B4
:10F820000022024B1A7710BD102400200000105057
:10F8300001234FF08040102110B4034A034CA372FF
:10F84000436010BC11607047200900201024002084
:10F8500001234FF08040102110B4044A044C63721D
:10F86000C0F8043110BC1160704700BF20090020AF
:10F8700010240020E0220021014809F0D8BF00BF79
:10F8800080010040F0B50546174B184885B06A1E48
:10F8900013F8011B834202F8011FF9D101242B4602
:10F8A000002702262A681248D11780FB020211485D
:10F8B000C1EB222243F8242B214622460390CDE9B6
:10F8C000014700966220F3F7AFFA0B48CDE90147F4
:10F8D0000390009605F12603224621466220F3F7A5
:10F8E000A3FA05B0F0BD00BF28000040540000405E
:10F8F00079787878D0D80100A8AE010070B5E02200
:10F90000064600210B4809F092FF002401234FF026
:10F910008042094D09492B770A208C729370214649
:10F92000137000F005F92C773046BDE87040FFF702
:10F93000A9BF00BF8001004000001050102400202B
:10F9400010B50446FFF79EFF31234FF0804004F1CD
:10F95000500203F1600150F82110013B212B22F8E5
:10F96000021DF6D14FF0804004F19C0203F16001CA
:10F9700050F82110013B22F8021D591CF6D110BD90
:10F980004FF0804270B5037909B201FB03F1948B0B
:10F990008B11A342B8BF234601250024022106880B
:10F9A0009BB24380A2F80C61A2F80E31074E084BBF
:10F9B000357709205C7282F8035182F802112146E2
:10F9C000A2F8005100F0B4F8347770BD0000105078
:10F9D000102400204FF0804393F81401704700BFBB
:10F9E0004FF0804393F81701704700BF0023094A86
:10F9F00082F832305064916472B6012382F840304C
:10FA000000BFB2F852309BB2002BFAD062B6B2F807
:10FA100050007047000010502DE9F04710222020C0
:10FA20004FF0300A502160244FF040094FF0010898
:10FA30004FF4807E4FF4007C4FF480674FF40066F3
:10FA40000825124B83F8002383F8040383F808A3E6
:10FA5000DFF83CA08AF8234083F8032383F805935A
:10FA600083F8091383F80A1383F80B1383F80F4301
:10FA7000C3F800801A601860C3F800E0C3F800C043
:10FA80001F601E601D60BDE8F08700BF00E100E060
:10FA900000ED00E04FF40042034BC3F88020BFF3B9
:10FAA0004F8FBFF36F8F704700E100E0002201210C
:10FAB000034BA3F86E20A3F86A20A3F868107047E0
:10FAC0000000105010B5174C84B094E80300029069
:10FAD00002A88DF80C1000F0ADF800F0B5F8FFF7B3
:10FAE0009BFF62B600F07CFAA36804A840F80C3DC6
:10FAF00000F070FA00F0B8FA00F0D4F900F028FB3A
:10FB0000094B1A6922F004021A61BFF34F8F0721D3
:10FB1000064A82F824105A6942F010025A6104B071
:10FB200010BD00BF309A010000ED00E00000105051
:10FB300008B500BF72B6084A135C3BB900BF30BFBE
:10FB400062B600BF72B6135C002BF7D000231354CB
:10FB500001B1884762B608BD1024002000200A4B7E
:10FB60000A4913F8012B10448B42C0B2F9D1064B5D
:10FB70001A78AA2A01D000207047DB7B181AB0FA45
:10FB800080F04009704700BF800040008F004000B7
:10FB90002DE9F041142000F09FFC0028B8BF073089
:10FBA000C51000234FF0A04001E08D4228DB027E0B
:10FBB0000133591E002AF8D10126B046194F0023FF
:10FBC0004FF0A04402E0A942267406DCA27E013375
:10FBD000591E002AF7D0BDE8F08172B6BFF34F8FEF
:10FBE0004FF6FE724FF6FF733A877A877B873B8723
:10FBF000BFF34F8F00F0FEFF84F8118062B6DEE79E
:10FC000072B6BFF34F8F4FF6FE714FF6FF72054B82
:10FC1000198759875A871A87BFF34F8F00F0EAFF79
:10FC200062B6C9E7000010504FF0A04301225A7499
:10FC3000704700BF0246034B0068127918601A71C2
:10FC4000704700BF2024002070B5FFF787FF012216
:10FC50000021334BD9705A72DA7200285CD0314AD5
:10FC6000D278D2B21A72002201242F492C4B8D78FF
:10FC70009A725A731D734D780E781E751D77CD7864
:10FC8000097983F8215083F820105A749A741C74EF
:10FC90009A7018B3234A51781A78C9B2D2B28A42FC
:10FCA00008D08A42B4BF013202F1FF32D0B28A4298
:10FCB0001870F6D11B4B1A491A794B78D2B2DBB2C5
:10FCC0009A420AD09A4203F1010096BF03F1FF3332
:10FCD000C3B2DBB29A424B70F4D170BD1A78D2B283
:10FCE000B02A08D0AF2AD4BF013202F1FF32D1B21C
:10FCF000B02A1970F6D10A4A5378DBB2082BECD03F
:10FD0000072B03F101018ABF03F1FF33CBB2DBB252
:10FD1000082B5370F4D1E0E7E0221A72A3E700BF8A
:10FD200000001050800040002024002007490B787C
:10FD3000DBB2834208D09842CCBF013303F1FF33DA
:10FD4000DAB283420A70F6D1704700BF000010504B
:10FD500008B5FFF703FF48B3154A5078D179C0B210
:10FD60009379882843EA01230FD0CE280CD1C3F51C
:10FD70009C432033002B07DD0E4AD81782FB032358
:10FD8000C0EBA3103238C0B208BD44F620629342E3
:10FD9000FADDA3F59C43084A203B82FB0312D817E7
:10FDA0001344A0EB63107838C0B208BDB02008BD82
:10FDB0008000400091739F5D43082184014B1878B7
:10FDC000704700BF00001050084A5378DBB28342EE
:10FDD0000AD0984203F1010196BF03F1FF33CBB281
:10FDE000DBB283425370F4D1704700BF0000105063
:10FDF000014B5878704700BF0000105010B5044602
:10FE0000FFF712FF4FF0A04320686168A26807C3A4
:10FE100010BD00BF38B54FF0A044E37DDBB2042B2A
:10FE200028D0082B19D0022B09D00123184A1370AF
:10FE300000BF4FF0A042137300BF537338BD154D80
:10FE400015496079F9F7CAFE61792868F9F734FF36
:10FE500062792B6813442B60E7E7104BD0E9051259
:10FE600059609A60236A5BBA0A4A18461360F9F728
:10FE70007FFEDAE7074D0A492079F9F78DFE2179EF
:10FE80002868F9F7C7FE22792B6813442B60CCE76A
:10FE9000102400202824002020000050581A0020A0
:10FEA000240000501021264B0020D3F8802042F07F
:10FEB0000102C3F880201A6C22F001021A641A6849
:10FEC00042F001021A60D3F8802022F00202C3F847
:10FED00080201A6C22F002021A641A6842F00202B0
:10FEE0001A60D3F880200A43C3F880201A6C0A43B2
:10FEF0001A641A680A431A60D3F8802022F020029C
:10FF0000C3F880201A6C22F020021A641A6842F0AA
:10FF100020021A60D3F8802022F04002C3F880202B
:10FF20001A6C22F040021A641A6842F040021A6009
:10FF3000C3F80801C3F80411C3F80011704700BFEB
:10FF40000000025038B572B64FF0405401256420CD
:10FF500084F8245000F0EAFA00F048FA00234FF445
:10FF60007A7084F8253084F8815000F0DFFA00F0D0
:10FF70003DFA62B638BD00BF10B572B64FF04054BE
:10FF80000123642084F8253000F0D0FA00F02EFA26
:10FF9000002384F8243084F8813062B610BD00BF9D
:10FFA0000122002110B5094C86B02478084806AB20
:10FFB000029103F8014DCDE9002103901146642020
:10FFC000F2F732FF9DF8170006B010BDB7004000F1
:10FFD000BCAE01000268014B1A6070472C2400205F
:10FFE00038B5FFF7BBFD0F23F0B94FF040524FF08B
:10FFF0000104D9B2013B072B82F82B1082F828406C
:020000021000EC
:1000000082F82800F5D1042382F82F304FF04053B6
:100010000121002283F8281083F828204FF47A70F9
:10002000BDE8384000F022BB4FF0405101250024CC
:100030000C4806E081F82B20013B81F8285081F81C
:100040002840027A0E2A8EBF0F22027AD2B2934241
:10005000DAB2EFDA4FF04052024B5B7ADBB282F851
:100060002F30D3E780004000F8B5FFF777FD4FF061
:10007000405401250026074684F825604FF47A7025
:1000800084F8205084F8275000F0F0FA642084F8B7
:10009000255000F0EBFA84F82450642000F0E6FAD2
:1000A00084F8256007BB06231C4D84F82730EB78C5
:1000B00084F826302B7884F842304FF040540123E6
:1000C0000022697840F24C4084F8461084F84420BD
:1000D00084F8453084F8413084F8403000F0C6FAA6
:1000E000AB7884F84430F8BDFFF75AFF0C4B9B7A8D
:1000F00088B94FF04052DBB2084D84F82730E978D8
:10010000074B82F82610DB7A29780B440B3BDBB2D5
:1001100082F84230D1E7053BEBE700BF2C240020FA
:100120008000400020B9064A064B106018607047F6
:1001300003490548034B054A08601A60704700BF31
:10014000342400203024002045FF000079FF000007
:100150004FF04053F0B40624012200250A26FF2068
:1001600083F8D64093F8D7100F2764F3030183F880
:10017000D710042183F8D86083F8402183F8D00099
:1001800083F87F5093F88C000526104383F88C0089
:1001900093F88C0040F0020083F88C0093F89100F3
:1001A00064F30300032483F8910083F8901083F82C
:1001B0008D1083F8A02093F8A10065F3010083F867
:1001C000A10083F8947093F88800104383F88800A6
:1001D00093F88900104383F8890083F8F12083F8AD
:1001E000874083F88E4083F8D22083F8D52083F8A7
:1001F000AB6083F8AD5083F8AC400224072083F84D
:10020000AE1083F8AF1093F88B1064F3061183F8E7
:100210008B1083F8930083F8B020F0BC704700BFC8
:10022000014B1870704700BF3D24002070B5194C79
:100230008AB02368184D092BCCBF0A23013301A8CB
:100240002360F9F773FB2B7813B3144B1B78FBB1C6
:100250002368092B1CDD9DF8133003F0FF06BBB9A2
:1002600000F0BAF80E4B1B68A3EBD30290420FD9F3
:10027000A3EB131398420BD22E70266072B600F0D7
:100280001DFA08490848094B094A08601A6062B615
:100290000AB070BD382400203D2400203E240020F8
:1002A00040240020041100209D060100B810002009
:1002B0003146000000230249024A0B701360704768
:1002C0003D2400203824002010B501248AB001A864
:1002D000F9F72CFB074B1C70F9F7D8FD28B9064B32
:1002E0001B7813B9054B1B680BB10AB010BD044B4A
:1002F0001C70FAE73E24002050100020B8100020A7
:100300003D24002070B50024124D1349134A2B6878
:100310008AB00C7014708BB1114E336873B101A8A0
:10032000F9F704FB2C60F9F7B1FD38B90D4B1B78D8
:1003300023B99DF8133003F0FF020BB10AB070BD72
:100340003260F4F7DBFC78200AB0BDE87040F4F7C7
:10035000C1BC00BF041100203E2400203D24002029
:10036000B81000205010002070B50C4D0C4C2B78AC
:1003700022789A4209D0002B0CBF05260426F9F7F3
:1003800085FD28B12B78237070BD0028F3D1FBE7E1
:1003900031460920F9F72AFFF4E700BF3E24002088
:1003A0003C24002000220721034B04481A605860B7
:1003B0009A601960704700BF10E000E0FFFF0F0077
:1003C0000022044B98681A60C0F57F2000F6FF7089
:1003D000704700BF10E000E0034B9868C0F57F2035
:1003E00000F6FF70704700BF10E000E0002382B00D
:1003F00000280193B8BF0730019BC010984206DD6A
:1004000000BF019B01330193019B8342F8DB02B0E3
:10041000704700BF30B583B072B600250E4C256022
:1004200062B6142000F058F801950028B8BF0730D4
:10043000019BC010984206DD00BF019B0133019370
:10044000019B8342F8DB2368002B02DD0122034B72
:100450001A7003B030BD00BF402400203E240020AD
:10046000054A0649937CD27801335B00934000FB38
:1004700003F091FBF0F070470000105000B4C4048A
:10048000054A937AD27ADBB20AB101339840034B22
:1004900093FBF0F0704700BF0000105040420F0087
:1004A000054A937AD27ADBB22AB10122134402FAC6
:1004B00003F390FBF3F0704700001050054A00EB87
:1004C0008000937CD27801335B009340000190FB65
:1004D000F3F070470000105041F28833124A00FBDD
:1004E00003F0137B0001DBB25A1E062A0DD9082B3C
:1004F00012D0092B15D0A3F10B02032A0ED90F2B12
:100500000CBF01234FF0FF3300E00133064AD278DD
:10051000934090FBF3F070470A23F7E7063B9B00FC
:10052000F4E70C23F2E700BF00001050124B00EB81
:1005300080001B7B0001DBB25A1E062A0DD9082B56
:1005400012D0092B15D0A3F10B02032A0ED90F2BC1
:100550000CBF01234FF0FF3300E00133064AD2788D
:10056000934090FBF3F070470A23F7E7063B9B00AC
:10057000F4E70C23F2E700BF00001050034B044ADD
:100580005B7C03F0010352F8233018470000105041
:10059000C8AE0100134B1B7BDBB25A1E062A0DD9D5
:1005A000082B18D0092B1BD0A3F10B02032A14D956
:1005B0000F2B0CBF01234FF0FF3300E0013309493B
:1005C000094AC9788B4000FB03F382FB0320DB1749
:1005D000C3EB601070470A23F1E7063B9B00EEE790
:1005E0000C23ECE70000105067666666034B044A74
:1005F0005B7C03F0010352F82330184700001050D1
:10060000C0AE010038B50024064D21460320EC7031
:10061000FFF78EFA21460320EC70FFF789FA024BB0
:10062000186838BD102400204024002070B5012235
:100630000024042686B00B4D06AB43F8040D11468A
:10064000CDE90124009603956420F2F7EDFB064BFB
:1006500005985C7100F07EF821460520FFF768FAE6
:1006600006B070BDD0AE01001024002008B5FFF721
:1006700085FFBDE80840FFF7D9BF00BF08B5FFF709
:10068000B5FFBDE8084000F01DB800BF08B5FFF792
:10069000ADFFBDE8084000F02DB800BF08B57A20D6
:1006A000FFF7A4FFBDE8084000F03CB8002000F0D0
:1006B00081B800BF012000F07DB800BF00F062B833
:1006C00000F06CB8012830B44FF000024FF0020483
:1006D00038BF01200121054B054D1A702A719C700D
:1006E0009860DA605A70197030BC7047000008508A
:1006F00010240020012830B44FF000024FF0020413
:1007000038BF01200121054B054D1A706A719C709C
:100710009860DA605A70197030BC70470000095058
:100720001024002001284FF000024FF0010138BFD3
:10073000012010B4054B064C1A7022719970986014
:10074000DA605A70197010BC704700BF0000085082
:100750001024002001284FF000024FF0010138BFA3
:10076000012010B4054B064C1A70627199709860A4
:10077000DA605A70197010BC704700BF0000095051
:1007800010240020012000220249034B08711A7036
:10079000704700BF102400200000085001200022F4
:1007A0000249034B48711A70704700BF10240020A3
:1007B0000000095010B40B4A0B4983B0CDE9001278
:1007C00002AB03EB800353F8082C9378DBB2012BC8
:1007D00004D10021054C04302354117003B010BC27
:1007E000704700BF0000095000000850102400208E
:1007F000034AD2F8803023F00103C2F880307047FA
:1008000000000250034AD2F8803043F00103C2F8DE
:100810008030704700000250034BD3F88000C04383
:1008200000F00100704700BF000002504FF48072DA
:10083000DCF808301A617047002823DDF0B5DCE9E8
:10084000013ED3F8013000241E7E0CE0DCF800707D
:100850003F5D07FB055503FB05F35B1242F82430AF
:100860000134A0420DD051F8045BDEF81030002EA8
:10087000ECD103FB05F39B1042F824300134A04275
:10088000F1D1F0BD704700BF4FF48072DCF8083042
:100890001A617047002821DDF0B5DCE9013E002433
:1008A0001E7E0CE0DCF800703F5D07FB055503FB86
:1008B00005F35B1242F824300134A0420DD051F808
:1008C000045BDEF81030002EECD103FB05F39B1027
:1008D00042F824300134A042F1D1F0BD704700BF8E
:1008E0004FF48072DCF808301A617047002823DD6D
:1008F000F0B5DCE9013ED3F8013000241E7E0CE0A7
:10090000DCF800703F5D07FB055503FB05F35B1248
:1009100042F824300134A0420DD051F8045BDEF8D7
:100920001030002EECD103FB05F39B1042F824306D
:100930000134A042F1D1F0BD704700BF4FF4807286
:10094000DCF808301A617047002823DDF0B5DCE9D7
:10095000013ED3F8013000241E7E0CE0DCF800706C
:100960003F5D07FB055503FB05F35B1242F824309E
:100970000134A0420DD051F8045BDEF81030002E97
:10098000ECD103FB05F39B1042F824300134A04264
:10099000F1D1F0BD704700BFDCF80430F0B4D3F8FB
:1009A000013093F821409CB900280FDD9B68DE8858
:1009B0009D8851F8043B013403FB06F393FBF5F3E8
:1009C000A0424FEA831342F8043BF2D1F0BC7047D7
:1009D0000028FBDD9B68DCF80040DF88013C9E8836
:1009E000204414F8015F51F8043BA04205FB033397
:1009F00007FB03F393FBF6F34FEA630342F8043B70
:100A0000EFD1F0BC704700BF704700BF00280BDD7E
:100A100010B4002451F8043B01349B01A04242F879
:100A2000043BF7D110BC7047704700BFF0B50E46CD
:100A300087B00221074601206546F3F727FE002311
:100A40001946043806F5086406F6081C059350F8A4
:100A5000046FA4F50862B60952F8883B9B1B9442C8
:100A60001944F9D10434A4450591F0D191FBF7F173
:100A7000AB6805911A88002A40D05888121A1202D1
:100A8000091A92FBF1F1B1F5DC7FA8BF4FF4DC71DC
:100A900019616A684FF0020CD2F8012000269068B4
:100AA00001228488042701FB04F10912FF29A8BF51
:100AB000FF211446C1801348CDF800C011460390B1
:100AC000CDE901666420F2F7AFF90F4B22462146CB
:100AD0000393CDE9014605AB00976420F2F7A4F932
:100AE000AB680A48CDE901460390009710332246CF
:100AF00021466420F2F798F907B0F0BD4FF48071F9
:100B00001961C6E7BCAF0100D8AF0100E4AF010036
:100B1000F4F7DCB808B5F4F70BF9BDE8084000219C
:100B20000120F3F7B3BD00BF30B595B020220021FE
:100B30000CA808F07CFE294C29492A4D2A48CDE909
:100B40000854CDE90A01294A294B0E9293F88120D5
:100B500002AC8DF83C2093F881308DF83D30F6F7EB
:100B600073F98DF83E00F6F775F98DF83F00F6F74A
:100B700077F98DF84000F6F779F98DF84100F6F72E
:100B80007BF98DF84200F6F77DF91190F6F780F9C0
:100B90001290F6F783F9ADF84C0008A8F8F7E2FEDA
:100BA000F6F77CF9F9F782FB002303220293A38274
:100BB000C4E90133C4E903338DF81D20FBF78AFB38
:100BC00006ABADF81E0093E803008DE8030094E83F
:100BD0000F00F8F731FE15B030BD00BF0508010069
:100BE0006D060100F1070100190801006E3816FAC0
:100BF0000000105070B5002301223F21482608252F
:100C0000022484B001A8CDE9013303938DF8076075
:100C10008DF808508DF809208DF80F208DF80A40C6
:100C20008DF80D10FFF7EAF804B070BD02FB01F279
:100C30001212FF2AA8BFFF22028070472DE9F0435D
:100C40002D4E95B02D4D0FAC08AF904699460A91A8
:100C500096E80F0084E80F001CABC4E9027520463B
:100C600013A91393EFF70CFB96E80F00244E0BAD7E
:100C700085E80F002146C5E902762846EFF700FB1C
:100C80000520F3F7C5FF0521D0F801200990D2E92E
:100C900002309A8814AEDA8006F8401D089031467A
:100CA0000120F3F765FF0221164B44F0010445F0E3
:100CB00001050846CDE906450593CDF81090F3F7F8
:100CC000E5FC04468822002108F0B1FD23463146A8
:100CD00040462222F6F7E8F80625012104200A4AB8
:100CE000009003922346CDE9011522226420F2F7F9
:100CF0009BF815B0BDE8F0833C9A01002D08010077
:100D000039080100CD6600000CC501002DE9F04353
:100D10002D4E95B02D4D0FAC08AF904699460A91D7
:100D200096E80F0084E80F001CABC4E9027520466A
:100D300013A91393EFF7A4FA96E80F00244E0BAD16
:100D400085E80F002146C5E902762846EFF798FAB4
:100D50000620F3F75DFF0627D0F8013014AE9A683D
:100D600009939188DB68D18006F8407D31460120E7
:100D70000893F3F7FDFE174B44F0010445F001051D
:100D8000022103200593CDE90645CDF81090F3F735
:100D90007DFC04464022002108F049FD23463146EF
:100DA00040461022F6F780F8012104200A4ACDE9D6
:100DB000000103920297234610226420F2F734F8D0
:100DC00015B0BDE8F08300BF3C9A0100890801001E
:100DD00095080100F56600000CC501002DE9F04200
:100DE000214E90B0214D0BAC04AF9946CDE90521C1
:100DF00096E80F0084E80F0016ABC4E902752046A0
:100E00000FA90F93EFF73CFA96E80F00184E07ADC5
:100E100085E80F00C5E9027621462846EFF730FA4B
:100E2000059B144FD3F8013044F00104D3E90223A9
:100E3000918845F00105D180169A0221042004937F
:100E40000092CDE902450197F3F720FC88220021AA
:100E500008F0EDFC2222034669464846F6F724F8DE
:100E600010B0BDE8F08200BF3C9A0100E10801002B
:100E7000ED080100E16600002DE9F042214E90B03E
:100E8000214D0BAC04AF9946CDE9052196E80F0042
:100E900084E80F0016ABC4E9027520460FA90F9332
:100EA000EFF7EEF996E80F00184E07AD85E80F0052
:100EB000C5E9027621462846EFF7E2F9059B144F73
:100EC000D3F8013044F00104D3E90223918845F0BE
:100ED0000105D180169A0221052004930092CDE9E4
:100EE00002450197F3F7D2FB4022002108F09FFC56
:100EF0001022034669464846F5F7D6FF10B0BDE814
:100F0000F08200BF3C9A01003D090100490901003F
:100F100009670000054B0649013810F8012F01331D
:100F200003F8012C8B42F8D1704700BF00008360AA
:100F3000200283602DE9F041304E90B0304D0BAC73
:100F400004AF8846069096E80F0084E80F0016ABC1
:100F5000C4E9027520460FA90F93EFF791F996E8BF
:100F60000F00284E07AD85E80F002146C5E902763F
:100F70002846EFF785F90120F3F74AFE0590022095
:100F8000F3F746FE02210020F3F780FB4FF40862DE
:100F90000021074608F04BFC0122059B10AED3F858
:100FA000013010469B6906F8402D31460493F3F753
:100FB000DFFD059BDFF864C0D3F8013031469A6845
:100FC000114EB2F804E03B46A2F806E0404644F079
:100FD000010445F001054FF40872CDE90245CDE961
:100FE00000C6F5F761FF094B09481B6909490A4A20
:100FF00003610B61136110B0BDE8F0813C9A010000
:101000002D0A0100990901007D450000E40D002032
:10101000200B0020000C0020B80C0020CD4C00005C
:1010200038B505460C4601200221F3F72FFBD5F811
:10103000013004F188059B68D9889A8854F8043BEC
:1010400003FB01F393FBF2F3A54240F8043BF5D117
:1010500038BD00BF2DE9F041804684B00220F3F78F
:10106000D7FD022106460120F3F710FB02220546B8
:10107000D6F8013004AC9B68012099880E4FD980C6
:1010800004F8102D2146F3F773FD2846882200212D
:1010900008F0CDFB094ADFF82CC0094E009221462A
:1010A0002B4640462222CDE901C70396F5F7FCFE08
:1010B00004B0BDE8F08100BF090A0100110B010076
:1010C0000D0A0100150B010083682DE9F04F9C8883
:1010D0000D4602FB04F42412FF2CA8BFFF248968EC
:1010E000DC808A780F788BB0A7EB42070497D0F8A2
:1010F00004E09A7806461878D5F804C0A0EB4202BE
:1011000005929EF802809CF80200B1F806A0804586
:1011100091F8089093F808B040F0B18030682968E1
:1011200000780978884240F0AA809EF806009CF872
:101130000610884240F0A380974200F0A980012267
:101140004FF00008022117465548063300910390DE
:1011500011467120CDE90188F1F766FEB368514868
:1011600008333A4639460390CDE90188712000974B
:10117000F1F75AFE04204C4B3A463946009003934F
:10118000712005ABCDE90178F1F74EFE0222AB6884
:101190004648009239463A4606330390CDE9018825
:1011A0007120F1F741FEAB68414808333A463946B1
:1011B0000390CDE9018871200097F1F735FE0422F4
:1011C0003C4B009203937120CDE901783A463946B1
:1011D00004ABF1F729FE049800FB0AF0002854D074
:1011E000059BA4B203FB04F409F10E09A9EB0B0B58
:1011F00004FA0BF494FBF0F402214046F3F746FAAC
:10120000E517061F00F67C0C56F8040FC117CDE950
:101210000801DDE9088908FB05F7A8FB040104FBC8
:101220000977820B394442EA81428B13CDE90823C6
:10123000DDE90823B4453260E6D102210120F3F74D
:1012400025FA061F00F1840C56F8042FD317CDE9B8
:101250000623DDE9062302FB05F704FB0377A2FB67
:1012600004233B44900B40EA83409913CDE90601E7
:10127000DDE9062366453260E6D1012005E0642001
:1012800000220D49F1F71CFE02200BB0BDE8F08FE3
:10129000642000220949F1F713FE0020F5E700BFA2
:1012A0000CAF010034AF010058AF010064AF010082
:1012B0008CAF0100B0AF0100D4AE0100F0AE010070
:1012C00030B583B0FFF730FCF5F778FAFFF792FC02
:1012D000FEF72AFAFEF7F6FBFEF73AFA00230C496E
:1012E00000931A460D68022001210A4CA847FFF717
:1012F00091F80120FFF738F800F050FB2568FEF761
:101300005DFDA8702468FEF773FDE07003B030BD8A
:1013100084DA0100A80600200246034B51680068E9
:10132000926807C3704700BF442400202DE9F04FA6
:10133000964683B0544E9DF834709DF830C0984660
:10134000009763460D46B6F90620B6F90410044628
:1013500070469DF83870FAF78BFB3378800290FB6B
:10136000F8F0002B4BD0A91C96F801904B002A46B0
:1013700004EB030E03F10208B9F1000F50D13EF85F
:10138000069C05F1FF3C24F80890A3F108053EF8FF
:10139000043C254424F8113061892389618023802D
:1013A000531ED2B31A4602F1010B4FEA4B0104EB74
:1013B000010A063134F801903AF8028C34F81B30F7
:1013C000C84407FB08F9BAF8048096F903B043440F
:1013D0000BFB0398BAF8023096F90290624509FBBC
:1013E00003834FEAA31300FB03F34FEA2343635243
:1013F00046D0012AD4D1E38800226380D3E765B1C7
:10140000A91C04EB4101043431F8022D00FB02F267
:101410008C424FEA22428A80F6D103B0BDE8F08FB9
:1014200000236380238024F8113024F80830002D35
:10143000F3D07F0004EB450131F802E996F903503F
:10144000B1F808C00B88CA889C4538BF9C469645B1
:1014500038BF96460CFB07F36A000EFB02338D88FB
:1014600096F902208C4205FB02324FEAA21200FBE1
:1014700002F24FEA22420A81DED103B0BDE8F08FCA
:101480002B88AEF800308BE74424002082B0F0B502
:1014900091B005460E4607A816A981E80C00F8F79A
:1014A00045FA9DF822301BB19DF82330002B5FD008
:1014B0003C4C169823461799189A07C394F90330A1
:1014C00094F90270C3F12003E17AC7EB4307A37AD2
:1014D000C7F347076A6905F12C00CDE901170093AE
:1014E00010212223FFF722FF05F15400617A237AAD
:1014F00004466A69CDE90117009322211023FFF702
:1015000015FFFEF7B7F9204631234FF0804403F171
:10151000600230F8021D013B212B44F82210F6D165
:101520004FF0804405F1A00232F8020D03F1600192
:10153000013B44F82100591CF6D10120FEF75CF96B
:101540002846FEF79FF9B4F84C301BB2336094F88C
:101550005030337294F85130737294F85230B37241
:1015600094F85330F37211B0BDE8F04002B0704708
:10157000B5F92430B3F5827F9ADA47F22E526B68C0
:10158000A3F5EA43313B934292D86B8BB42B8FD9AE
:10159000054A044C04AB07CA83E8070084E8070047
:1015A0008CE700BF442400204C9A010038B5042287
:1015B0000125124B124C1D712260FFF777F8F8F7E6
:1015C00071FC837E2BB90F4B1B6813B10E4A15704B
:1015D00098470E4BD3F80021120708D500220825A2
:1015E0000B480C49C3F880510270C1F84021012119
:1015F0001023094AD160236038BD00BF10240020A9
:1016000020090020B41000207010002000E100E04C
:101610001C09002000000250000008500122052192
:1016200038B50D4B0D4C5A712160FFF743F80C4B48
:10163000D3F80021120708D50022082509480A49D5
:10164000C3F880510270C1F8402101211023074ADC
:10165000D160236038BD00BF102400202009002085
:1016600000E100E01C0900200000025000000950C9
:101670000321012238B5144B144C154DDA7021604A
:10168000FEF722FE2B78D3B901232B70FEF78AFEDA
:10169000104B1B6803B19847F8F704FCC37E03F0B6
:1016A000FF052BB90C4B1B6813B198470B4B1D70F2
:1016B000002110230A4AC2F84011236038BDFEF70A
:1016C0007FFE084B1860DFE710240020200900206F
:1016D0001C09002004110020B81000207010002008
:1016E000000002504024002001234FF060501021E0
:1016F00010B4034A034CE372836210BC116070475C
:1017000020090020102400200F21124A124B1160E2
:101710005B6F84B00193019B23F4FF6323F0070305
:101720000293019B23F07F030393029BB3F5800F89
:101730000AD0039A094B9A4206D0019A084B9A4262
:1017400002D20122074B1A700122034BA3F86C202E
:1017500004B07047200900200000105080FF0100F5
:1017600000FC01005024002008B5FFF7A9FD00F09F
:10177000BFFC002008BD00BF704700BF30B50A4D58
:101780000A4C83B0294620464FF0CD32FCF71CFBB3
:101790004FF0CD32204600922B46054A0549FCF712
:1017A00065FB002003B030BD0C3E00200C32002051
:1017B000005600200C3E0020704700BF10B5084BBB
:1017C000084C1A6821466320F1F77AFBF3F770F8AA
:1017D000054B2146BDE810401A686320F1F770BB45
:1017E000A004002014B00100A40400200021012066
:1017F000F2F74CBFF0B5194B194C83B01A6821466B
:101800006320F1F75DFBF2F75BFF0220F3F700FACC
:10181000064601A8FDF78CFF02210120F2F736FFF2
:101820000746104B02A91B880F4D21F8083D0220E6
:10183000F3F79EF90220FFF70DFC28460221FFF77F
:1018400079FB2A6939463046FFF7EAFB074B214608
:101850001A686320F1F734FB03B0F0BDA004002048
:10186000F4AF0100589A0100E40D0020A404002008
:101870002DE9F0430220ABB0F3F7CAF902210120B1
:10188000F2F704FF002107460120F2F7FFFE0646AB
:1018900007A8FDF74DFF0546274C8822002120466A
:1018A00007F0C5FF079AEDB219A80DF1200C0492BC
:1018B000CDE901C003940097294633461A2202203D
:1018C000FDF7F0F95DB1204604EB4502B0F90030B8
:1018D000002BB8BF5B4220F8023B9042F6D10124B6
:1018E0004FF0040906214FF00008144A3B46CDE9A9
:1018F0000141039221462A46CDF800906220F1F77B
:1019000093FA0F4A3346CDE90282CDE900942A4684
:1019100002217220F1F788FA02200A4B009003930B
:10192000CDE9014821462A46034B6920F1F77CFAAC
:1019300001482BB0BDE8F08338270020FCAD010042
:10194000ECB00100F8B00100022300B583B002A999
:1019500001F8043D0120F3F70BF9F3F7B7F9F3F7BA
:10196000E7F903B05DF804FB30B585B00446FEF737
:10197000EFF901220023074D07490444CDE9013363
:1019800003912B460092114664202C70F1F74CFA1B
:1019900005B030BDD404002058A201000148F6F77C
:1019A0009FBD00BFFC0500202DE9F04F8BB004AFB8
:1019B000FEF7CEF9012400250426DFF834C207F132
:1019C000180343F8140D2246CDF80CC0CDE90145AB
:1019D000214600966420F1F727FA784807F11803AA
:1019E000DFF8109243F8105D22460390CDE90145DF
:1019F000009621466420F1F717FAD9F804107B68A5
:101A0000CA1DB86822F00702ADEB020D0344A942DB
:101A10000DF1100B7B600EDD5A4601EBD170A3EB8C
:101A20006003DBB20BEB010002F8013B824203F1E1
:101A30000103DBB2F8D189000A3121F00701ADEBD7
:101A4000010D0DF110084046F6F75CFD00225C49DF
:101A50006420F1F735FA414607F11002D9F8040085
:101A600001240025F6F71CFE0426564B07F1180A40
:101A70004AF8040D2246CDE90253CDE9006421461F
:101A8000514B6420F1F7D0F9504BD9F8042003935F
:101A900021465B46CDE9015500946420F1F7C4F975
:101AA0004B49D9F80420009643460391CDE90145FE
:101AB00021466420F1F7B8F9464B07F11002009671
:101AC000039321461346CDE9014522466420F1F7F0
:101AD000ABF9414A5346214600960392CDE90145B0
:101AE00022466420F1F7A0F94046F6F7B7FD2A46F2
:101AF0003A496420F1F7E4F9D9F8043007F10C0C05
:101B0000023B624641461846C7E90353F6F7C8FD53
:101B1000334A786107F1100000960346039221468C
:101B20002246CDE901456420F1F77EF92D493A6955
:101B30000BEB04030391CDE9015521460094642089
:101B4000F1F772F922493A694346CDE90251CDE9EC
:101B5000006421466420F1F767F91E4BCDE900646B
:101B6000CDE90253224607F10C0321466420F1F728
:101B70005BF9194A5346CDE90252CDE90064224689
:101B800021466420F1F750F97A697E68164BDFF838
:101B900068C01B681644154AF6B29E70214603922F
:101BA000CDE9015500946346224664208CF800601C
:101BB000F1F73AF91C37BD46BDE8F08F30B00100AF
:101BC00040B001006CB001000006002078B00100B8
:101BD00084B0010080B0010090B00100A0B001000D
:101BE000D8B00100E0B00100A806002058A2010012
:101BF00024B00100FC050020D404002010B5084BDF
:101C0000084C1A6821466320F1F75AF9FFF7CCFE19
